:100000000C94CC230C94FD230C94FD230C94FD2321
:100010000C94FD230C94FD230C94FD230C94FD23E0
:100020000C94FD230C94FD230C94FD230C94FD23D0
:100030000C94FD230D94CF570C94FD230C94FD23B9
:100040000C94FD230C947DF60C94FD230C94FD235D
:100050000C94FD230C94FD230C9444F30D948557CC
:100060000C94FD230C94295D0C941F5D0C94FD23CE
:100070000C94FD230C94FD230C94FD230C94FD2380
:100080000C94F5400C94FD230C94FD230C94FD235B
:100090000C94FD230C94FD230C94FD230C94FD2360
:1000A0000C94FD230C94FD230C94C7400C94FD2369
:1000B0000C94FD230C94FD230C94FD230C94FD2340
:1000C0000C94FD230C94FD230C94FD230C94FD2330
:1000D0000C94FD230C94FD230C94FD230C94FD2320
:1000E0000C94FD23084AD73B3BCE016E84BCBFFD78
:1000F000C12F3D6C74319ABD56833DDA3D00C77FF8
:1001000011BED9E4BB4C3E916BAAAABE0000008090
:100110003F05A84CCDB2D44EB93836A9020C50B91F
:10012000918688083CA6AAAA2ABE000000803F004B
:100130000C9493980C949E9B0C94898C0C946A98C4
:100140000C948E8F0D9433510C94C7980C94EBC97A
:100150000C94D5B70C94B0BE0C9422910D94A05180
:100160000C94C1C90C9476400C9416DC0C94A591A7
:100170000C94CF970C94CDC90C944A910D94525085
:100180000D94DB2E0D94CE500D9468500C94BF91BD
:100190000D944D500C94BB970C94FF8E0C942795A6
:1001A0000D9479500C94BCB00D94D5510C944C9195
:1001B0000C94CDD30C94F28C0C94A59B0C94615DA3
:1001C0000C94E15D0D94FD510D94A8510C9466932F
:1001D0000C94408F0C9433B60C9479950C947B8FCF
:1001E0000C9435C00C94019C0C9470930C940DA04D
:1001F0000C94948C0C94FFB40C94E5C90D94955018
:100200000C94C28F0D9475510C94C9920C94EEAE5F
:100210000C94929B0C94DACD0C94CE910C9427DE26
:100220000C94899B0C94C2DA0C9484D30C946A933A
:100230000C9468930C94D1A60C94C75D0C9475959E
:100240000C9451900C947F900C94688F0C94DFB7B1
:100250000C94A29A0C947D950D9407510C94C3971D
:100260000D94082F0C9429900C94A9C90D94A350B7
:100270000C94318F0C948F9B0D9473500C945B40B5
:100280000C9412990D94DF510D94B3500C94C3DA71
:100290000C94598F0D940C510D947D500C94C8BC46
:1002A0000C94959B0C9455930C9478260C94AEDC8E
:1002B0000D946D510D9464500C941B950C941993EE
:1002C0000C94F9980C945E910C9487920C94A98FDD
:1002D0000D9499500C94D6A60C94D1910C94995DE0
:1002E0000C94DCA30C94DBA60C9468900C94B5C918
:1002F0000C94C9DF0C94B35D0C94D4910D941851F7
:100300000D9491500C94B9390C94F2910D94E951DB
:100310000C946E930C94D7970C9442900C94CE5DF1
:100320000C94B7970D9407520C9402240C943699B0
:100330000C9440DA0D9484510C94D9C90C94C9B929
:100340000C947E9B0C94D58F0C94A89B0C94AB9B27
:100350000D9414610C94EC8C0C94D2DE0C94649388
:100360000D94BC510D94F6600C9468910D94285135
:100370000C948B980C9413A90C9450A70D949F5037
:100380000C94D7910C9484AC0C9499B10C94A39BCD
:100390000C946C930C944F260C94EE8F0C948ACA98
:1003A0000C946D910D9483500C9416900C94914084
:1003B0000C94BBC90C94C7970C9484AF0C94C35D88
:1003C0000C94A3D30D9498510C94CCA60C94A3C96F
:1003D0000C94C2DD0C945FAB0D948B500C949F4336
:1003E0000C9496900C94BBC50C942B990C942DDD19
:1003F0000C94E2930D94F3510C9466C10C949B9B66
:100400000C94A85D0C94979A0C94E3DD0C94FF2354
:100410000C9459910C9401270C94DFC90C94D89238
:100420000C94FFDE0C948C9B0C94F7B70C9424D3A3
:100430000C9443D30C9450CA0C9405240C94389E0D
:100440000C9423B00D94A4600C940EAE0D948750C0
:100450000C94668C0C9463910C9407900C94ED951D
:100460000C94AFC90C948A5D0C94869A0C948E9A65
:100470000C9442DE0C94AF5D0C94D3C90C94B397EA
:100480000C94D3970C94BB5D0C9418A10C94188F0A
:100490000C94B75D0C94AC400D94B2510C94D38C79
:1004A0000C94D95D0C94BF970C94049C0D941E5130
:1004B0000C94989B0C94C7C90D946C500C94CB97DA
:1004C0000C94809A0C94D8C70C9437910C944ADD04
:1004D0000D942A2F0D947A510C94BF5D0D94705099
:1004E0000C94D1D20C94DA260D94C6510C94B2D24D
:1004F0000C942B910C9472930C940AB30D948E511E
:100500000C94C0DE0C944E910C94E0980C941F9CBB
:100510004E414E494E495459494E46CDCCCC3D0AE8
:10052000D7233C17B7D13877CC2B329595E6241FCB
:10053000B14F0A000020410000C84200401C462084
:10054000BCBE4CCA1B0E5AAEC59D7400407A10F357
:100550005A00A0724E18090010A5D4E80000E876F1
:1005600048170000E40B54020000CA9A3B00000048
:10057000E1F505000080969800000040420F000061
:1005800000A08601000000102700000000E8030022
:100590000000006400000000000A000000000001EC
:1005A00000000000002C76D888DC674F0823DFC1EC
:1005B000DFAE59E1B1B796E5E3E453C63AE65199A7
:1005C0007696E8E6C28426EB898C9B62ED407C6FD0
:1005D000FCEFBC9C9F40F2BAA56FA5F490055A2A87
:1005E000F75C936B6CF9676DC11BFCE0E40D47FE93
:1005F000F520E6B500D0ED902E0300943577050088
:1006000080841E080000204E0A000000C80C33330E
:1006100033330F986E12831141EF8D2114893BE61D
:100620005516CFFEE6DB18D1844B381BF77C1D90A6
:100630001DA4BBE424203284725E228100C9F1240F
:10064000ECA1E53D27434F4D4D554E49434154499B
:100650004F4E0044525952554E004552524F52533C
:1006600000494E464F004543484F004572726F7235
:100670002077726974696E6720746F204545505207
:100680004F4D210A0053544F505045442E200050E6
:1006900072696E7465722073746F70706564206423
:1006A000756520746F206572726F72732E204669B3
:1006B0007820746865206572726F7220616E6420A4
:1006C000757365204D39393920746F2072657374E4
:1006D0006172742E202854656D7065726174757234
:1006E000652069732072657365742E2053657420CC
:1006F00069742061667465722072657374617274C6
:10070000696E67290A004E6F20436865636B7375D5
:100710006D2077697468206C696E65206E756D62F6
:1007200065722C204C617374204C696E653A200010
:100730004E6F20436865636B73756D2077697468CD
:10074000206C696E65206E756D6265722C204C613F
:100750007374204C696E653A2000636865636B733F
:10076000756D206D69736D617463682C204C6173C5
:1007700074204C696E653A20004C696E65204E7598
:100780006D626572206973206E6F74204C617374A2
:10079000204C696E65204E756D6265722B312C2080
:1007A0004C617374204C696E653A20004D313130D4
:1007B0000053657269616C20737461747573206D88
:1007C00069736D617463680A00776169740A005324
:1007D000442072656164206572726F720A00486F0E
:1007E00074656E642049646C652054696D656F752D
:1007F0007400486F74656E642049646C65205469A8
:100800006D656F75740A002121204B494C4C2063A3
:100810006175736564206279204B494C4C20627588
:1008200074746F6E2F70696E0A002121204B494C41
:100830004C2063617573656420627920746F6F204A
:100840006D75636820696E6163746976652074698B
:100850006D65202D2063757272656E7420636F6DF7
:100860006D616E643A20004D656469612052656D6A
:100870006F766564004D6564696120496E736572C9
:10088000746564004D313030305300627573793ACD
:100890002070617573656420666F7220696E707573
:1008A000740A00627573793A20706175736564200B
:1008B000666F7220757365720A00627573793A20EB
:1008C00070726F63657373696E670A00506C65615F
:1008D0007365205265736574005052494E544552F9
:1008E0002048414C5445440025533A20255300707C
:1008F0006F7765726F6666004B494C4C45442E20FD
:10090000005072696E7465722068616C7465642E43
:10091000206B696C6C28292063616C6C6564210A0A
:100920000053544F505045442E20005072696E744D
:1009300065722073746F70706564206475652074CF
:100940006F206572726F72732E204669782074680A
:1009500065206572726F7220616E64207573652008
:100960004D39393920746F20726573746172742E39
:10097000202854656D7065726174757265206973A5
:100980002072657365742E2053657420697420612C
:10099000667465722072657374617274696E67291A
:1009A0000A006563686F3A004572726F723A0042DE
:1009B000696C696E656172204C6576656C696E67FD
:1009C00020477269643A0A0021212053544F502075
:1009D00063616C6C65642062656361757365206F2B
:1009E0006620424C546F756368206572726F722086
:1009F0002D20726573746172742077697468204D5C
:100A00003939390A0021212053544F502063616C39
:100A10006C65642062656361757365206F66204252
:100A20004C546F756368206572726F72202D20724E
:100A30006573746172742077697468204D3939392F
:100A40000A005072696E74696E67204F626A65634E
:100A500074002553202569002F2F616374696F6E20
:100A60003A00737461727400656E6400486F746557
:100A70006E6420746F6F20636F6C640A0053656E40
:100A800064204D31303820746F20726573756D6548
:100A90000A00496E736572742066696C616D656EDB
:100AA0007420616E642073656E64204D3130380AA5
:100AB0000052656865617420446F6E650052656818
:100AC000656174696E672E2E2E00526568656174CB
:100AD000004865617465722054696D656F757400B6
:100AE00053656E64204D31303820746F2068656125
:100AF00074206E6F7A7A6C650A004E6F7A7A6C6534
:100B0000205061726B65640070617573656400509C
:100B10006175736500726573756D65640052657308
:100B2000756D696E67004732362043616E63656C90
:100B30006564004732362048656174696E67204EEF
:100B40006F7A7A6C65004732362048656174696E49
:100B500067204265640057616974696E6720666F3B
:100B600072206865617475702E0A00466978656444
:100B7000204C656E677468205072696D6500446F23
:100B80006E65205072696D696E67004D616E7561AA
:100B90006C207072696D696E672E2E2E004C656137
:100BA00076696E6720473236003F53706563696629
:100BB00069656420582C5920636F6F7264696E6197
:100BC0007465206F7574206F6620626F756E647334
:100BD0002E0A003F28522965706561742076616C89
:100BE0007565206E6F7420706C61757369626C65D9
:100BF0003B206D757374206265206174206C6561A3
:100C0000737420312E0A003F53706563696669650D
:100C100064206E6F7A7A6C652074656D70657261A0
:100C200074757265206E6F7420706C617573696283
:100C30006C652E0A003F53706563696669656420C0
:100C400066696C616D656E742073697A65206E6F7C
:100C50007420706C61757369626C652E0A003F5375
:100C60007065636966696564207072696D65206C82
:100C7000656E677468206E6F7420706C617573693F
:100C8000626C652E0A003F5370656369666965642E
:100C9000206E6F7A7A6C652073697A65206E6F7446
:100CA00020706C61757369626C652E0A003F526535
:100CB0007472616374696F6E204D756C7469706CC9
:100CC000696572206D757374206265207370656349
:100CD00069666965642E0A003F53706563696669D9
:100CE00065642052657472616374696F6E204D751E
:100CF0006C7469706C696572206E6F7420706C61C1
:100D0000757369626C652E0A003F5370656369668E
:100D1000696564206C6179657220686569676874CB
:100D2000206E6F7420706C61757369626C652E0A39
:100D30000043292E0A003F53706563696669656444
:100D4000206265642074656D70657261747572658A
:100D5000206E6F7420706C61757369626C652028F9
:100D600034302D00473236207374617274696E67B7
:100D70002E2E2E0A004F46460A0046616465204822
:100D800065696768742000426564204C6576656C0F
:100D9000696E6720004661696C656420746F206528
:100DA0006E61626C6520426564204C6576656C6995
:100DB0006E670A00496E76616C6964206D657368C0
:100DC0002E0A0050726F62696E6720506F696E74F0
:100DD0000025532025692F2569002E0A002F005079
:100DE000726F62696E67206D65736820706F696EDF
:100DF000742000202844525952554E290047323958
:100E0000204175746F20426564204C6576656C697D
:100E10006E67003F20284C2C522C462C4229206F14
:100E20007574206F6620626F756E64732E0A003FC2
:100E30002856296572626F7365206C6576656C2033
:100E4000696D706C61757369626C652028302D3432
:100E5000292E0A00426164205A2076616C75650A69
:100E6000004E6F2062696C696E65617220677269FD
:100E7000640A00446576696174696F6E0025533AAF
:100E80002025730046696E6973686564210A003A1B
:100E9000207A3A2000206F662000476F696E672035
:100EA000746F3A20580043570A00206469723A0070
:100EB00020616E676C653A005374617274207261D0
:100EC000646975733A004D343820506F696E740050
:100ED00025533A2025642F256400506F7369746987
:100EE0006F6E696E67207468652070726F62652E20
:100EF0002E2E0A003F4C656773206F66206D6F765B
:100F0000656D656E7420696D706C61757369626C76
:100F1000652028302D3135292E0A003F2028582CF5
:100F20005929206F7574206F6620626F756E647327
:100F30002E0A0050726F6265206F7574206F6620F4
:100F4000626F756E6473003F53616D706C652073E2
:100F5000697A65206E6F7420706C61757369626C5C
:100F6000652028342D3530292E0A004D3438205A7A
:100F70002D50726F6265205265706561746162699F
:100F80006C69747920546573740A003F285629658A
:100F900072626F7365206C6576656C20696D706C2C
:100FA00061757369626C652028302D34292E0A0022
:100FB0005374616E6461726420446576696174691A
:100FC0006F6E3A20002052616E67653A2000204D16
:100FD00061783A2000204D696E3A200020536967FD
:100FE0006D613A20004D65616E3A2000205200414B
:100FF0006363656C65726174696F6E3A2050005767
:1010000041524E494E4721204C6F77205A204A6565
:10101000726B206D6179206C65616420746F20753E
:101020006E77616E746564207061757365732E0AE6
:101030000020204D61783A2000200020204D696E6C
:101040003A2000536F667420656E6473746F70731A
:101050003A20004D32342053256C642054256C64B2
:10106000004739322E392045257300473120462567
:1010700064004739322E39205A2573004731205AEF
:101080003020463230300047312058257320592512
:1010900073204633303030004D34323020532569D0
:1010A000205A2573004D31303620502569205325B4
:1010B00069004D32303020442573004732385230B9
:1010C0005859004739322E39204530205A300A47C6
:1010D000315A2573004D31303920532569004D3187
:1010E000393020532569004D343230205330205A96
:1010F000300020496E76616C696420657874727581
:10110000646572200047322F47332062616420708B
:101110006172616D65746572730A00536C65657008
:101120002E2E2E005A2050726F626520506173740B
:10113000204265640A005A2050726F626520506137
:10114000737420426564004732384C30004D3131B1
:10115000372050726F6265206661696C65642E0A83
:101160004732380A0070726F62655F726577697026
:101170006500473239205265747279696E67005094
:10118000726F62696E67204661696C6564004D31FB
:10119000313720426564206C6576656C696E672026
:1011A0006661696C65642E0A4730205A31300A4DF9
:1011B0003330302050323520533838300A4D3330F8
:1011C00030205035302053300A4D333030205032EB
:1011D0003520533838300A4D3330302050353020E8
:1011E00053300A4D333030205032352053383830A8
:1011F0000A4D333030205035302053300A473420E8
:1012000053310070726F62655F6661696C6564007E
:101210004D31313720426564206C6576656C696EAE
:101220006720646F6E652E00205A3A200020593ADC
:10123000200042656420583A20004D657368207094
:101240006F696E74206F7574206F662072616E67AF
:10125000650A004D302053746F70004D3120537477
:101260006F7000436C69636B20746F2052657375F7
:101270006D652E2E2E004E6F204D6F76652E00452B
:101280006E642066696C65206C6973740A0042653F
:1012900067696E2066696C65206C6973740A004E1C
:1012A0006F206D656469610A00526573756D696EC2
:1012B0006720534400286E6F2066696C65290043DF
:1012C000757272656E742066696C653A20005072A2
:1012D000696E742074696D653A20000A53746174F4
:1012E000733A2046696C616D656E74207573656430
:1012F0003A20002C204C6F6E67657374206A6F6211
:101300003A2000546F74616C2074696D653A200056
:1013100053746174733A20002C204661696C6564D3
:101320003A20002C2046696E69736865643A200093
:101330005072696E74733A200053746174733A206A
:1013400000436F6F6C696E672E2E2E0048656174C6
:10135000696E672E2E2E0045202553006F6B006F9F
:10136000666600660661065A06530645064445420F
:1013700055473A004D3131332053004265642043D4
:101380006F6F6C696E672E2E2E0042656420486573
:101390006174696E672E2E2E00537550655220437E
:1013A000522D3230204F46462E002F2F004D313423
:1013B0003520533C696E6465783E206F7574206FEC
:1013C000662072616E67652028302D31290A004D34
:1013D00032303620580046523A0020466C6F773A39
:1013E00020003A200020536572766F2000206F7530
:1013F00074206F662072616E67650A0053657276AD
:101400006F200020643A0020693A0020703A0049B9
:101410006E76616C69642065787472756465720AB1
:101420000020643A0020693A0020703A004C43449E
:1014300020436F6E74726173743A200064697300A4
:10144000656E0043290A0061626C656420286D693D
:101450006E2074656D702000436F6C642065787435
:1014600072756465732061726520004D34323120DD
:10147000696E636F727265637420706172616D650D
:101480007465722075736167650A004D6573682025
:10149000706F696E74206F7574206F662072616E54
:1014A00067650A004F666673657473204170706CDF
:1014B000696564004572723A20546F6F20666172EC
:1014C0002100546F6F206661722066726F6D20720A
:1014D00065666572656E636520706F696E740A007B
:1014E000454550524F4D204F4B0A002E0A002028F0
:1014F000302D313029002076616C7565206F757450
:10150000206F662072616E676500416476616E636C
:1015100065204B3D004F4646004F4E00506F7765AB
:10152000722D6C6F7373207265636F7665727920AC
:10153000004D383400446F6E65207072696E7469B6
:101540006E672066696C650A004D3737004D333190
:10155000004361703A004D4541545041434B0043B4
:101560004F4F4C45525F54454D5045524154555292
:1015700045004348414D4245525F54454D50455208
:1015800041545552450042414259535445505049E7
:101590004E470041524353004D4F54494F4E5F4D0B
:1015A0004F44455300544845524D414C5F50524FB3
:1015B00054454354494F4E004C4F4E475F46494CAB
:1015C000454E414D45004155544F5245504F5254A0
:1015D0005F53445F5354415455530053445F575233
:1015E00049544500524550454154005344434152EB
:1015F000440050524F4D50545F535550504F525429
:1016000000454D455247454E43595F504152534561
:101610005200434153455F4C494748545F42524949
:101620004748544E45535300544F47474C455F4C31
:10163000494748545300534F4654574152455F5011
:101640004F574552004255494C445F50455243451F
:101650004E54004C4556454C494E475F4441544119
:10166000005A5F50524F42450052554E4F5554005C
:101670004155544F4C4556454C005052494E545FCD
:101680004A4F420050524F47524553530041555420
:101690004F5245504F52545F54454D5000564F4C99
:1016A000554D455452494300454550524F4D004217
:1016B000494E4152595F46494C455F5452414E5341
:1016C0004645520053455249414C5F584F4E5F5872
:1016D0004F4646004649524D574152455F4E414D97
:1016E000453A4D61726C696E20322E302E375F4460
:1016F00057372E3320544D33442032454D44424217
:10170000202841707220323420323032312031377B
:101710003A31353A34322920534F555243455F43CD
:101720004F44455F55524C3A68747470733A2F2F8A
:101730006769746875622E636F6D2F496E73616E91
:101740006974794175746F6D6174696F6E2F4D6145
:10175000726C696E2F747265652F437265616C6976
:1017600074794477696E5F322E302050524F544F57
:10177000434F4C5F56455253494F4E3A312E30201D
:101780004D414348494E455F545950453A53755071
:1017900065522043522D323020455854525544450D
:1017A000525F434F554E543A3120555549443A63A0
:1017B000656465326132662D343161322D343734DF
:1017C000382D396231322D63353563363266333622
:1017D0003766660A0050726F6265204F66667365F1
:1017E00074205A0050726F6265204F66667365748C
:1017F000205A00290A0020746F20003F5A206F757C
:1018000074206F662072616E6765202800290A00C7
:1018100020746F20003F59206F7574206F6620720E
:10182000616E676520282D00290A0020746F200052
:101830003F58206F7574206F662072616E67652057
:10184000282D0050726F6265204F666673657420A4
:10185000580043616E6E6F74206F70656E207375F3
:101860006264697220002569730025696D2025690D
:1018700073002569682025696D2025697300256935
:1018800064202569682025696D2025697300256914
:101890007920256964202569682025696D202569DE
:1018A000730023646566696E652044454641554C66
:1018B000545F00626564004B6420004B6920004B5C
:1018C000702000504944204175746F74756E652016
:1018D00066696E6973686564212050757420746848
:1018E00065206C617374204B702C204B6920616EF5
:1018F00064204B6420636F6E7374616E7473206632
:10190000726F6D2062656C6F7720696E746F204313
:101910006F6E66696775726174696F6E2E680A0012
:10192000504944204175746F74756E652066616915
:101930006C6564212074696D656F75740A00504987
:1019400044204175746F74756E65206661696C65BD
:1019500064212054656D70657261747572652074C0
:101960006F6F20686967680A00204B643A20002086
:101970004B693A2000204B703A200020436C617381
:1019800073696320504944200A00204E6F206F760F
:10199000657273686F6F740A002054753A200020D6
:1019A0004B753A2000206D61783A2000206D696EF9
:1019B0003A200020643A200020626961733A2000D6
:1019C000504944204175746F74756E65207374615D
:1019D00072740A00504944204175746F74756E65C5
:1019E000206661696C6564212054656D7065726163
:1019F0007475726520746F6F20686967680A00509B
:101A00004944204175746F74756E650050494420D7
:101A10004175746F74756E65206661696C656421CB
:101A200020426164206865617465722069640A00FF
:101A30004572723A207574663820666F6E74206E37
:101A40006F7420696E697469616C697A65642E00CF
:101A50004572723A207574663820666F6E74206E17
:101A60006F7420696E697469616C697A65642E00AF
:101A70004572723A207574663820666F6E74206EF7
:101A80006F7420696E697469616C697A65642E008F
:101A9000FFE0FFD140A0C8A6A22FF80023AC00AF02
:101AA00010FFFEFF05FFD0FFE0FFC1FFD1E240A025
:101AB000C8A6A22FF800238127AC00AFFFD0FF6497
:101AC000FFD1A5FFD0FF64FF64FFD1A4FFD0FF16B4
:101AD000FFFE000C0F00FE07022503BB017FFE087E
:101AE000FE08FE05080806000040F0C888889878BF
:101AF00010050808060000C0F88888888888F8055E
:101B000005050600012030F8302005080806000011
:101B10002070F820202020E00509090600FF207031
:101B2000A8A8B888887020070505070001D86C367A
:101B30006CD80509090600FFF8A88888888888A855
:101B4000F8050A0A0600FE205050505088A8A888C0
:101B50007003030306000340A040FFFFFFFFFFFFE9
:101B6000FFFFFFFFFFFFFFFFFFFFFFFFFFFFFFFF85
:101B70000000000605FF0107070602008080808044
:101B8000800080030303060105A0A0A00506060649
:101B9000000050F85050F8500509090600FF207069
:101BA000A8A07028A87020050707060000C8C81064
:101BB0002040989805070706000040A0A040A89084
:101BC000680103030602058080800309090601FFFE
:101BD0002040408080804040200309090601FF80AA
:101BE000404020202040408005070706000020A834
:101BF000702070A8200505050600012020F820208F
:101C00000203030601FFC04080050101060003F83E
:101C1000020202060100C0C0050707060000081006
:101C20001020404080050707060000708898A8C86B
:101C3000887003070706010040C040404040E005AF
:101C40000707060000708808102040F805070706FF
:101C50000000F8081030088870050707060000101B
:101C6000305090F81010050707060000F880F008C3
:101C7000088870050707060000304080F0888870EB
:101C8000050707060000F8081010202020050707A8
:101C900006000070888870888870050707060000B5
:101CA00070888878081060020505060100C0C00031
:101CB000C0C00206060601FFC0C000C04080030588
:101CC000050601012040804020050303060002F8BC
:101CD00000F8030505060101804020408005070744
:101CE000060000708810202000200507070600006D
:101CF0007088B8A8B880700507070600007088884B
:101D0000F8888888050707060000F04848704848AA
:101D1000F00507070600007088808080887005073E
:101D200007060000F04848484848F0050707060045
:101D300000F88080F08080F8050707060000F88032
:101D400080F08080800507070600007088808098FA
:101D50008870050707060000888888F88888880347
:101D60000707060100E04040404040E00507070645
:101D7000000038101010109060050707060000885A
:101D800090A0C0A090880507070600008080808092
:101D90008080F805070706000088D8A8888888880A
:101DA0000507070600008888C8A8988888050707DF
:101DB000060000708888888888700507070600007C
:101DC000F08888F08080800507070600007088880A
:101DD00088A89068050707060000F08888F0A090A2
:101DE000880507070600007088807008887005075E
:101DF00007060000F8202020202020050707060005
:101E00000088888888888870050707060000888809
:101E1000888850502005070706000088888888A811
:101E2000A8500507070600008888502050888805BC
:101E30000707060000888850202020200507070695
:101E40000000F80810204080F80309090601FFE0AF
:101E500080808080808080E0050707060000804049
:101E600040201010080309090601FFE0202020206F
:101E7000202020E00503030600052050880501010D
:101E80000600FEF803030306010580402005050552
:101E90000600007008788878050707060000808033
:101EA000F0888888F005050506000070808088703D
:101EB0000507070600000808788888887805050562
:101EC0000600007088F080700507070600003048A3
:101ED00040E04040400507070600FE70888888788B
:101EE00008700507070600008080F088888888034E
:101EF00007070601004000C0404040E00409090611
:101F000001FE100030101010109060050707060049
:101F10000080808890E09088030707060100C04099
:101F200040404040E0050505060000D0A8A8A8A84C
:101F3000050505060000B0C8888888050505060067
:101F40000070888888700507070600FEF08888887A
:101F5000F080800507070600FE78888888780808E2
:101F6000050505060000B0C880808005050506004F
:101F70000078807008F00507070600002020F82090
:101F80002020180505050600008888889868050542
:101F90000506000088888850200505050600008891
:101FA00088A8A8500505050600008850205088051F
:101FB00007070600FE888888502040800505050632
:101FC0000000F8102040F80309090601FF204040F6
:101FD0004080404040200109090602FF8080808047
:101FE00080808080800309090601FF8040404020F6
:101FF0004040408005030306000248A890FF554E6C
:102000004C4F41442046494C414D454E54004C4FA5
:1020100041442046494C414D454E540046494C41AF
:102020004D454E54204348414E47450042656400AB
:10203000456E636C6F73757265002568753A25305F
:102040003268750025303268753A2530326875007F
:10205000202020202020200020202020001FE02001
:1020600010201020101020102020102010303008D8
:1020700040048003001FE03FF03FF03FF01FE01FEF
:10208000E03FF03FF03FF00FC0078003003FFFF05C
:1020900038007030FC3020FC102078102030102CDC
:1020A00000D02E31D02F7BD02F7BD02E31D02C00E2
:1020B000D020301020781020FC1030FC3038007018
:1020C0003FFFF03FFFF03800703186302387102744
:1020D00087902F87D02F03D02030102078102078C1
:1020E000102030102F03D02F87D027879023871000
:1020F0003186303800703FFFF01FFFF81FFFF804F3
:1021000010400208200208200410400820801041DE
:10211000001041000820800410400000001FFFF85C
:102120001FFFF8FFFFFF8000018E00E19F01F19388
:1021300081399F81F99F81F99FB9F98F28F1803802
:10214000018000019FFFF99174999B06A99B54A9F6
:102150009B56A99B54999FFFF9FFFFFF6E6F74690F
:102160006669636174696F6E200063616E63656C9C
:10217000005072696E742041626F7274656400442D
:1021800069736D6973730055492041626F7274659C
:1021900064004D323520500A4D323400526573755B
:1021A0006D65005549205061757365005061757308
:1021B000696E672E2E2E00726573756D65004D3247
:1021C000340000FE0003FF8007C7C00701E00000E5
:1021D000E00000F00000700400700E00701F00703E
:1021E0003F80F00E00E00F01E007C7C003FF800052
:1021F000FE0000FE0003FF8007C7C00F01E00E00D5
:10220000E03F80F01F00700E00700400700000704E
:102210000000F00000E00701E007C7C003FF8000F6
:10222000FE000E000E000E000E000E000E000E004E
:102230000E007FC03F801F000E00040004000E004F
:102240001F003F807FC00E000E000E000E000E002B
:102250000E000E000E00FFFFFF7F80FFC0FFC0FFDB
:10226000C07F807F80FFC0FFC0FFC03F001E000C0A
:102270000050726F6265205A204F66667365740065
:102280004C6F6164206D6D00556E6C6F6164206DE4
:102290006D0046696C2E204469612E004520696EF0
:1022A000206D6D5E3300416476616E6365204B0086
:1022B0004D333033205531204525692053256900A1
:1022C000504944204175746F74756E65202A005022
:1022D00049442D44202A005049442D49202A0050C9
:1022E00049442D50202A00200820466163740020B4
:1022F00008204D6178002008204D696E004F666609
:10230000004F6E004175746F74656D7000565472A5
:102310006176204D696E00566D696E00566D61786C
:10232000204500566D6178205A00566D617820591D
:1023300000566D6178205800416D6178204500415C
:102340006D6178205A00416D6178205900416D61BE
:1023500078205800412D54726176656C00412D52F1
:1023600065747261637400416363656C0056652D2A
:102370004A65726B00565A2D4A65726B0056592D8C
:102380004A65726B0056582D4A65726B0050726F29
:102390006265205A204F66667365740050726F62E2
:1023A000652059204F66667365740050726F6265D0
:1023B0002058204F666673657400452073746570FD
:1023C000732F6D6D005A2053746570732F6D6D00FF
:1023D000592053746570732F6D6D005820537465C8
:1023E00070732F6D6D00416476616E636564205378
:1023F000657474696E6773003F0043616E63656C5A
:1024000000496E6974004D34323800496E69746950
:10241000616C697A6520454550524F4D0046696CA4
:10242000616D656E740054656D706572617475726E
:10243000650053746570732F6D6D0050726F626527
:10244000204F666673657473004A65726B00416362
:1024500063656C65726174696F6E0056656C6F635D
:102460006974790053657420486F6D65204F666606
:102470007365747300436F6E666967757261746922
:102480006F6E003F004E65787420506F696E740067
:10249000446F6E65004E65787400486F6D696E67B5
:1024A0002058595A003F0043616E63656C204F62AB
:1024B0006A656374004E4F005945530043616E6373
:1024C000656C204F626A656374203D004D61696EE2
:1024D0000053572D4D6F64650053746F770044654A
:1024E000706C6F790053656C662D5465737400527F
:1024F0006573657400426564004E6F7A7A6C65009E
:1025000046616E20537065656400436F6E6669674F
:1025100075726174696F6E00526573746F726520B5
:1025200044656661756C7473004C6F61642053651B
:102530007474696E67730053746F726520536574A9
:1025400074696E6773005072656865617420242039
:10255000436F6E66004F6666004F6E00506F776582
:1025600072204F7574616765004C434420436F6E61
:10257000747261737400424C546F756368005072DA
:102580006F6265205A204F666673657400416476F9
:10259000616E6365642053657474696E6773004D82
:1025A00061696E004D37303220542564004D36305D
:1025B0003020423020542564004D373032203B25F6
:1025C00064004D37303120542564004D37303200DF
:1025D0004D373031004D363030204230004D61698A
:1025E0006E00436F6E74696E756500507572676535
:1025F000206D6F726500524553554D45204F505424
:10260000494F4E533A005052494E54205041555371
:1026100045440020204E6F7A7A6C653A2000506164
:10262000726B696E672E2E2E000000576169742050
:10263000666F720066696C616D656E7420636861B7
:102640006E676500746F20737461727400576169FE
:102650007420666F720066696C616D656E742075BA
:102660006E6C6F616400004E6F7A7A6C65206865ED
:102670006174696E6700506C65617365207761698C
:10268000742E2E2E00005072657373206275747460
:102690006F6E00746F2068656174206E6F7A7A6C5B
:1026A000650000496E736572742066696C616D65C2
:1026B0006E7400616E64207072657373206275744D
:1026C000746F6E00746F20636F6E74696E75650051
:1026D0005761697420666F720066696C616D656E22
:1026E00074206C6F616400005072657373204275D2
:1026F00074746F6E00746F20726573756D652070F1
:1027000072696E7400005761697420666F72207080
:1027100072696E7400746F20726573756D652E2E0C
:102720002E00005761697420666F720066696C61E3
:102730006D656E7420707572676500003E2000251F
:102740006C642E25696D004578747275646564202B
:10275000546F74616C003E20004C6F6E676573743B
:10276000204A6F622054696D65003E2000546F74EA
:10277000616C205072696E742054696D6500436FFE
:102780006D706C65746564003A20005072696E74F7
:1027900020436F756E74003A2000313530003500EB
:1027A0004245443A204154432031303447542D327D
:1027B0000052756E617761792057617463683A20C1
:1027C0004F4E004D61782054656D700034353000F7
:1027D0004D696E2054656D7000350045313A2053C7
:1027E0006C696365456E6720343530C2B043005074
:1027F00053550047656E657269630050726F746F60
:10280000636F6C00312E30004261756400323530E8
:1028100030303000437265616C6974793344205202
:10282000414D50530042696C696E656172204C6580
:1028300076656C696E67004578747275646572734D
:1028400000310074696E796D616368696E65733318
:10285000642E636F6D0053755065522043522D32C4
:102860003000323032312D30342D313800322E30BC
:102870002E375F4457372E33004D61726C696E00FE
:102880005072696E74657220537461747300546879
:1028900065726D6973746F727300426F6172642048
:1028A000496E666F005072696E74657220496E667B
:1028B0006F004D61696E004D313030300053746FE0
:1028C00070205072696E7400526573756D6520508A
:1028D00072696E7400506F776572204F757461670E
:1028E00065004D3139305335350A4732380A4732A1
:1028F000390A4D3430300A4D313034533231350AD3
:102900004732380A4D313039533231350A4D34327D
:102910003053310A47315831303059313030463533
:102920003030300A47315A300A4D3530300A4D3197
:10293000313720536574205A204F666673657400E2
:102940004D313036533132380A4D333033433853FA
:102950003231354530550A4D3530300A4D31313739
:10296000205049442054756E6520446F6E65004DBB
:102970003139305335350A4D313034533231350A1F
:102980004732380A4732394C310A47312058313002
:10299000305931303046353030300A47315A300006
:1029A0004D3530300A4D3131372053657474696EBE
:1029B00067732053746F726564005072657020668F
:1029C0006F72205A2041646A757374005049442024
:1029D00054756E650053746F726520536574746925
:1029E0006E6773005365747570004D61696E003FCA
:1029F000004261636B0053746F70005072696E74B3
:102A00002066726F6D204D65646961004368616E78
:102A10006765204D65646961004D32310041626F28
:102A20007574205072696E746572004368616E67D8
:102A3000652046696C616D656E74004C6576656CE9
:102A4000696E6720546F6F6C7300436F6E666967C1
:102A500075726174696F6E0054656D706572617432
:102A6000757265004D6F74696F6E00486F737420E6
:102A7000537461727400526573756D65205072698C
:102A80006E74004E6F204D656469610043616E6332
:102A9000656C204F626A6563740054756E650053FF
:102AA000746F70205072696E740050617573652088
:102AB0005072696E7400496E666F2053637265656B
:102AC0006E003F005374617274205072696E74001E
:102AD00043616E63656C005072696E740043616E91
:102AE0006E6F7420656E74657220737562646972AE
:102AF0003A2000022E2E004D61696E002100486FC1
:102B000074656E6420746F6F20636F6C6400426143
:102B1000636B0050726F6365656400536F66742069
:102B2000456E6473746F7073004D6F74696F6E00DF
:102B300044697361626C652053746570706572736B
:102B4000004D3834004D34382050726F6265205487
:102B5000657374004732384F0A4D34382050313095
:102B6000004C6576656C20436F726E65727300462B
:102B700061646520486569676874004F6666004F48
:102B80006E00426564204C6576656C696E67004C2A
:102B90006576656C20426564004732394E00486FA7
:102BA0006D65205A004732385A00486F6D652059CC
:102BB000004732385900486F6D6520580047323859
:102BC00058004175746F20486F6D650047323800BA
:102BD0004D61696E005072656865617420242045FE
:102BE0006E640050726568656174202420426564DB
:102BF0000054656D706572617475726500436F6F26
:102C00006C646F776E005072656865617420240093
:102C100046616E205370656564207E0042656400E5
:102C20004E6F7A7A6C65004D61696E0050726F620A
:102C300065205A204F666673657400416476616E44
:102C40006365204B00466C6F770046616E205370C1
:102C5000656564207E00426564004E6F7A7A6C651B
:102C6000005370656564004D61696E00486F6D6961
:102C70006E67204661696C6564006F70656E005414
:102C80005249474745524544003A20007A5F6D69F2
:102C90006E00795F6D696E00785F6D696E005265D8
:102CA000706F7274696E6720656E6473746F7020E4
:102CB0007374617475730A0020746F6F206C6F6E8B
:102CC0006720657874727573696F6E2070726576AF
:102CD000656E7465640A0020636F6C6420657874A7
:102CE000727573696F6E2070726576656E74656457
:102CF0000A00486F6D65202573257325732046698A
:102D0000727374005761726E696E673A20486F6D16
:102D1000696E672042756D702044697669736F72C1
:102D2000203C20310A0002020400000000000000E4
:102D30000000000000000070430000704300007AB3
:102D400043000000410000004100000040FFFFFF81
:102D500000000001000000010000800055555500F2
:102D60000000400033333300AAAA2A00499224000D
:102D700000002000C7711C0099991900D145170067
:102D8000555515003BB113002449120011111100D3
:102D9000000010000F0F0F00E3380E0043790D0004
:102DA000CCCC0C00C3300C00E8A20B0064210B005B
:102DB000AAAA0A00703D0A009DD80900427B0900BA
:102DC00092240900DCD3080088880800104208001B
:102DD00000000800F0C10700878707007550070052
:102DE000711C07003EEB0600A1BC060069900600BE
:102DF00066660600703E06006118060017F40500BE
:102E000074D105005BB00500B29005006272050048
:102E10005555050078390500B81E05000505050063
:102E20004EEC040087D40400A1BD040090A7040068
:102E300049920400C17D0400EE690400C7560400F5
:102E4000444404005C3204000821040041100400E2
:102E5000000004003FF00300F8E0030026D2030066
:102E6000C3C30300CCB503003AA803000A9B0300C8
:102E7000388E0300C08103009F750300D0690300F2
:102E8000505E03001D53030034480300913D0300CE
:102E90003333030016290300381F0300971503007E
:102EA000300C0300030303000BFA020049F1020097
:102EB000BAE802005CE002002DD802002DD002002A
:102EC00059C80200B0C0020031B90200DAB10200F4
:102ED000AAAA0200A0A30200BC9C0200FA9502006C
:102EE0005C8F0200DF88020082820200457C0200C3
:102EF0002776020027700200436A02007C64020009
:102F0000D05E02003F590200C8530200FFFDFCFAE8
:102F1000F8F6F4F2F0EEECEAE9E7E5E3E1E0DEDC16
:102F2000DAD9D7D5D4D2D0CFCDCBCAC8C7C5C3C2C2
:102F3000C0BFBDBCBAB9B7B6B4B3B2B0AFADACAA3E
:102F4000A9A8A6A5A4A2A1A09E9D9C9A9998979590
:102F5000949392908F8E8D8B8A89888786848382C2
:102F600081807F7E7D7B7A797877767574737271D4
:102F7000706F6E6D6C6B6A696867666564636261C9
:102F8000605F5E5D5C5B5A595858575655545352B2
:102F90005150504F4E4D4C4B4A4A49484746464582
:102FA0004443424241403F3E3E3D3C3B3B3A393840
:102FB0003837363535343332323130302F2E2E2DEE
:102FC0002C2B2B2A29292827272625252423232291
:102FD000212120201F1E1E1D1C1C1B1B1A19191825
:102FE00018171616151514131312121111100F0FAE
:102FF0000E0E0D0D0C0C0B0A0A090908080707062E
:1030000006050504040303020201000000007043EA
:103010000000704300007A43000000000000000040
:103020000000000053657474696E67732053746FF9
:1030300072656400454550524F4D20496E69746970
:10304000616C697A65640A003B20003A0A0020201E
:103050004D36303320002055004C0046696C616DC0
:10306000656E74206C6F61642F756E6C6F61642087
:103070006C656E677468733A0020204D39303020DB
:103080004B004C696E65617220416476616E6365C8
:103090003A0020204D3835312058005A2D50726F9B
:1030A0006265204F66667365740020204D343133AD
:1030B000205300506F7765722D4C6F7373205265EB
:1030C000636F766572793A0020204D3235302043A7
:1030D000004C434420436F6E74726173743A002055
:1030E000440020490020204D33303420500020443B
:1030F0000020490020204D333031205000504944F9
:103100002073657474696E67733A00204600204826
:103110000020204D3134352053004D6174657269B3
:10312000616C2068656174757020706172616D6595
:10313000746572733A00204A0020204732392057C4
:1031400020490020204D3432302053004175746FE7
:1031500020426564204C6576656C696E673A002094
:10316000204D323036205800486F6D65206F6666FE
:103170007365743A0020580020530020204D3230EF
:1031800035204200416476616E6365643A20423CBA
:103190006D696E5F7365676D656E745F74696D658B
:1031A0005F75733E20533C6D696E5F666565647242
:1031B0006174653E20543C6D696E5F747261766522
:1031C0006C5F66656564726174653E20583C6D6134
:1031D000785F785F6A65726B3E20593C6D61785FFD
:1031E000795F6A65726B3E205A3C6D61785F7A5FE9
:1031F0006A65726B3E20453C6D61785F655F6A650C
:10320000726B3E0020540020520020204D3230349A
:10321000205000416363656C65726174696F6E2054
:1032200028756E6974732F7332293A20503C70727E
:10323000696E745F616363656C3E20523C726574B5
:10324000726163745F616363656C3E20543C7472A9
:103250006176656C5F616363656C3E0020204D3272
:1032600030312058004D6178696D756D2041636380
:10327000656C65726174696F6E2028756E69747310
:103280002F7332293A0020204D3230332058004D20
:103290006178696D756D20666565647261746573CA
:1032A0002028756E6974732F73293A005374657002
:1032B000732070657220756E69743A002044002096
:1032C000204D3230302053002044697361626C65B8
:1032D000640A0046696C616D656E74207365747470
:1032E000696E67733A0020204D3134392043203B0A
:1032F00020556E69747320696E2043656C7369751F
:10330000730A0020286D6D290020204732312020CB
:1033100020203B20556E69747320696E206D6D000E
:1033200000803B4400803B44000020410000964266
:103330000000A0420000A0420000C8430000BE42BE
:10334000D0070000D0070000640000004B00000020
:1033500024F4D43050C38E20C2A24017828B701147
:10336000127A910D816CD90AA861E108C7586607E5
:10337000615143061E4B5D05C145A7041A41110466
:10338000093D9803713931034036DB026533910200
:10339000D4305402802E1D02632CEE01752AC50123
:1033A000B028A001102781018F2564012B244B0137
:1033B000E0223401AC211F018D200D01801FFC0093
:1033C000841EED00971DDF00B81CD200E61BC6006E
:1033D000201BBC00641AB200B219A8000A19A00090
:1033E0006A189900D117910040178B00B516840018
:1033F00031167E00B31579003A157300C7146F00BB
:1034000058146A00EE1366008813630025135E00EB
:10341000C7125B006C12570015125400C111510005
:1034200070114F0021114B00D61049008D1047003C
:103430004610440002104200C00F4000800F3E00C2
:10344000420F3C00060F3B00CB0E3800930E3700B6
:103450005C0E3500270E3400F30D3200C10D310033
:10346000900D3000600D2E00320D2D00050D2C004A
:10347000D90C2B00AE0C2900850C29005C0C270010
:10348000350C27000E0C2600E80B2400C40B24008A
:10349000A00B23007D0B23005A0B2100390B2100C8
:1034A000180B2000F80A1F00D90A1E00BB0A1E00D4
:1034B0009D0A1D00800A1D00630A1C00470A1B00AC
:1034C0002C0A1B00110A1A00F7091A00DD0919005D
:1034D000C4091900AB091900920917007B091800EB
:1034E000630917004C09160036091600200916005A
:1034F0000A091500F5081500E0081400CC081400AE
:10350000B8081400A4081400900813007D081200E5
:103510006B08130058081200460812003408110006
:10352000230811001208110001081100F007100013
:10353000E0071000D0071000C0071000B0070F0010
:10354000A107100091070E0083070F0074070F00FA
:1035500065070E0057070E0049070E003B070D00D8
:103560002E070E0020070D0013070D0006070D00A3
:10357000F9060C00ED060D00E0060C00D4060C0068
:10358000C8060C00BC060C00B0060C00A4060B001C
:1035900099060C008D060B0082060B0077060B00C7
:1035A0006C060B0061060A0057060B004C060A0069
:1035B00042060A0038060A002E060A0024060A00FF
:1035C0001A060A001006090007060A00FD05090090
:1035D000F4050900EB050900E2050900D905090019
:1035E000D0050900C7050900BE050900B50508009A
:1035F000AD050800A50509009C0508009405080014
:103600008C050800840508007C0508007405080086
:103610006C050700650508005D05070056050800F4
:103620004E0507004705070040050800380507005C
:10363000310507002A050700230507001C050600C1
:10364000160507000F05070008050600020507001C
:10365000FB040600F5040700EE040600E80406007B
:10366000E2040700DB040600D5040600CF040600D0
:10367000C9040600C3040600BD040600B704060022
:10368000B1040500AC040600A6040600A004050071
:103690009B04060095040500900406008A040500BA
:1036A00085040500800406007A0405007504050001
:1036B000700405006B040500660405006104050044
:1036C0005C04050057040500520405004D04050084
:1036D00048040500430405003E0404003A040500C4
:1036E00035040500300404002C0405002704040000
:1036F000230405001E0404001A0404001604050037
:10370000110404000D04040009040500040404006D
:1037100000040400FC030400F8030400F4030400A4
:10372000F0030400EC030400E8030400E4030400D5
:10373000E0030400DC030400D8030400D403040005
:10374000D0030400CC030400C8030300C503030036
:1037500024F404D9201BC40C5C0E9804C4095F0235
:1037600065077101F405F900FB04B3004804870004
:10377000C10369005803550003034500BE023A0027
:103780008402310053022A0029022500040220008D
:10379000E4011C00C8011900AF01170098011400D2
:1037A00084011300710110006101100051010E002D
:1037B00043010D0036010B002B010B0020010B0013
:1037C000150109000C01090003010800FB000800B5
:1037D000F3000800EB000700E4000600DE0006002E
:1037E000D8000600D2000600CC000500C700050086
:1037F000C2000500BD000400B9000400B5000400CB
:10380000B1000400AD000400A9000400A5000300FD
:10381000A20003009F0004009B0003009800030027
:103820009500020093000300900003008D00020049
:103830008B00030088000200860002008400030061
:10384000810002007F0002007D0002007B00020078
:103850007900020077000100760002007400020087
:1038600072000100710002006F0002006D00010093
:103870006C0002006A00010069000200670001009C
:1038800066000100650001006400020062000100A2
:1038900061000100600001005F0002005D000100A6
:1038A0005C0001005B0001005A00010059000100AA
:1038B00058000100570001005600010055000100AA
:1038C00054000100530000005300010052000100A9
:1038D00051000100500001004F0001004E000000A7
:1038E0004E0001004D0001004C0001004B000000A3
:1038F0004B0001004A00010049000100480000009F
:103900004800010047000100460000004600010099
:103910004500000045000100440001004300000094
:10392000430001004200000042000100410000008D
:1039300041000100400001003F0000003F00010085
:103940003E0000003E0001003D0000003D0001007F
:103950003C0000003C0000003C0001003B00000077
:103960003B0001003A0000003A000100390000006D
:103970003900010038000000380000003800010064
:10398000370000003700010036000000360000005C
:103990003600010035000000350000003500010050
:1039A0003400000034000000340001003300000047
:1039B000330000003300010032000000320000003C
:1039C0003200010031000000310000003100010030
:1039D0003000000030000000300001002F00000027
:1039E0002F0000002F0000002F0001002E0000001B
:1039F0002E0000002E0001002D0000002D00000010
:103A00002D0000002D0001002C0000002C00000003
:103A10002C0000002C0001002B0000002B000000F7
:103A20002B0000002B0001002A0000002A000000EB
:103A30002A0000002A0001002900000029000000DF
:103A400029000000290000002900010028000000D2
:103A500028000000280000002800000028000100C5
:103A600027000000270000002700000027000000BA
:103A700027000100260000002600000026000000AC
:103A8000260000002600010025000000250000009F
:103A90002500000025000000250000002500010091
:103AA0002400000024000000240000002400000086
:103AB0002400010023000000230000002300000078
:103AC0002300000023000000230000002300010069
:103AD000220000002200000022000000220000005E
:103AE000220000002200010021000000210000004F
:103AF0002100000021000000210000002100000042
:103B00002100010020000000200000002000000033
:103B10002000000020000000200000002000000025
:103B2000200001001F0000001F0000001F00000017
:103B30001F0000001F0000001F0000001F00010008
:103B40001E0000001E0000001E0000001E000000FD
:103B5000232C0000B8220000561800003A0F000085
:103B6000B8080000B1040000710200003E0100002E
:103B700020436F756E7420583A00426564004531E9
:103B800000626564002C2073797374656D20737412
:103B90006F7070656421204865617465725F494487
:103BA0003A200048656174696E67204661696C65FA
:103BB000640048656174696E67206661696C65645C
:103BC000004D3131322053687574646F776E001088
:103BD00000C90210012C014001220170011801B03E
:103BE000010E01F00104015002FA00B002F00030B1
:103BF00003E600D003DC009004D2007005C800A0EA
:103C000006BE000008B400B009AA00D00BA00060F6
:103C10000E960060118C000015820020197800C0FB
:103C20001D6E00A0226400B0275A00902C500000A6
:103C3000314600E0343C0010383200903A280060F1
:103C40003C1E00A03D1400803E0A00203F000054AE
:103C50004845524D414C2052554E41574159005410
:103C60006865726D616C2052756E6177617900458F
:103C700072723A204D415854454D50004D415854B0
:103C8000454D5020747269676765726564004572BE
:103C9000723A204D494E54454D50004D494E5445C1
:103CA0004D502074726967676572656400202F004B
:103CB0002042403A0020403A0020573A0020573A2C
:103CC00000496E76616C696420657874727564650C
:103CD000720A007C3C3E5E2B3D3F2F5B5D3B2C2AF5
:103CE000225C0043616E6E6F74206F70656E20738E
:103CF00075626469722000534420496E69742046DD
:103D000061696C0053442063617264206F6B0A0028
:103D10006F70656E526F6F74206661696C65640ABE
:103D200000766F6C756D652E696E697420666169C9
:103D30006C65640A004E6F20534420636172640A0C
:103D4000000A4D3234004D3233202573002E0A0014
:103D50006F70656E206661696C65642C2046696CC5
:103D6000653A200046696C652073656C656374650F
:103D7000640A002053697A653A200046696C652020
:103D80006F70656E65643A2000454E44205355427D
:103D9000524F5554494E450A002220706F7300223D
:103DA00020706172656E743A2200535542524F552D
:103DB00054494E452043414C4C20746172676574F0
:103DC0003A220053756263616C6C204F76657266AF
:103DD0006C6F77004578636565646564206D617814
:103DE00020535542524F5554494E452064657074D6
:103DF000683A002E0A0044656C6574696F6E20662F
:103E000061696C65642C2046696C653A20004669DE
:103E10006C652064656C657465643A005344207079
:103E200072696E74696E67206279746520004E6FE6
:103E300074205344207072696E74696E670A004181
:103E4000425300504C41002F6175746F25632E67FB
:103E50000057726974696E6720746F2066696C65BB
:103E60003A2000667265736800646F696E670020AF
:103E700066696C653A20004E6F77200002FD55554B
:103E80005555555FFFFFFFFFFFFFFFFFFFFE0000DF
:103E90000000003FFFFFFFFFFFFFFFFFFFFD0000EF
:103EA00007FFFFFFFFFFFFFFFFFFFFFFFFFE07C052
:103EB0000555555555555FFFFFFFFFFFFFFC0A20D5
:103EC0000600000000003FFFFFFFFFFFFFFE141091
:103ED00005000007FFFFFFFFFFFFFFFFFFFC2808B3
:103EE0000607C00555555555555FFFFFFFFE5404A5
:103EF000040A200600000000003FFFFFFFFC6004F2
:103F000006141005000007FFFFFFFFFFFFFE50042F
:103F10000428080607C00555555555555FFC600433
:103F2000065404040A200600000000003FFE54046A
:103F30001C60040614100500000000001FFC280887
:103F40002E50040428080607C00001F03FFE14109C
:103F5000546004065404040A200002081FFC0A20CE
:103F60006654041C60040614100005043FFE07C0DC
:103F70005428082E5004042808000A021FFC0000E0
:103F80002E14105460040654040015013FFE000076
:103F90001C0A206654041C60040018011FFC000069
:103FA0000607C05428082E50040014013FFE0000EC
:103FB0000400002E14105460040018011FFCFFFFC1
:103FC000FE00001C0A206654041C15013FFED55556
:103FD0005400000607C05428082A0A021FFC841057
:103FE0004600000400002E14105105043FFEC410CA
:103FF00044FFFFFE00001C0A206102881FFC8410A1
:1040000046D5555400000607C05101F03FFE84100C
:104010004484104600000400002A00001FFCC41065
:1040200046C41044FFFFFE00001C00003FFE841049
:1040300044841046D5555400000000001FFCD5559F
:104040005684104484104600000000003FFCFFFF2F
:10405000FCC41046C41044FFFFFFFFFF9FFE00009A
:1040600006841044841046D555555555BFFD555509
:1040700054D5555684104484104104109FFFFFFF0F
:10408000FCFFFFFCC41046C410410411BFFFFFFF3A
:10409000FE00000684104484104104109FFFFFFFBF
:1040A000FD555554D5555684104104109FFFFFFF10
:1040B000FFFFFFFCFFFFFCC410410411BFFFFFFF27
:1040C000FFFFFFFE00000684104104109FFFFFFF6A
:1040D000FFFFFFFD555554D555555555BFFFFFFF03
:1040E000FFFFFFFFFFFFFCFFFFFFFFFF9FFFFFFF43
:1040F000FFFFFFFFFFFFFE00000000003FFFFFFF8C
:10410000FFFFFFFFFFFFFD55555555555FFFFFFFB3
:10411000FFFFFFFFFFFFFFFFFFFFFFFFFFFFFFFFAF
:10412000FFFFFFFFFFFFFFFFFFFFFFFFFFFFFFFF9F
:10413000FFFFFFFFFFFFFFFFFFFFFFFFFFFFFFFF8F
:10414000FFFFFFFFFFFFFFFFFFFFFFFFFFE02EFB73
:104150007DFBFBCFC1DFBB3EC0E1FE3C1FFDEE7B24
:1041600039F9F3CF9EDFBB3EDFDEFCDDE7FDEE3B42
:10417000BBF9EBD7BF5FBB5EDFDEFDEDF7FDEEBB4E
:10418000D3FAEBB73FDFBB4EDFDFFFCDF3FDEEDB56
:10419000C7FAEBBB7FC03B6EC0E3FF1DF3FDEECB68
:1041A000EFFADBBB7FDFBB66DFF8FFCDF3FDEEEBA5
:1041B000EFFB5B033F5FBB76DFFE7FEDF3FDEEF3CE
:1041C000EFFB5B79BEDFBB7ADFDE7DEDF7FDEEF363
:1041D000EFFBBAFD9EDFBB7CDFDEFDCDE7FDEEFB36
:1041E000EFFBBAFDC1DFBB7EC0E0FE1C1F6D61723C
:1041F0006C696E66772E6F726700322E302E375FD5
:104200004457372E33001FFFFFFFFFFFFF60000002
:10421000000001FF400000000000FF8000000000DF
:10422000007F83CF00000C303F87FF80000C301FE1
:10423000867980000C000F8C30C7838C30E78C307F
:10424000CFC7CC31F38C30DCECEC33B98C30D86C8C
:104250006C33198C30D06C0C33198C30D86C0C3317
:10426000198C30DC6C0E3B198C30CF7C079F198C7D
:1042700030C77C038F19400000000000026000007E
:10428000000000061FFFFFFFFFFFF86001F4017050
:1042900001EA019001E001B001D601D001CC01009A
:1042A00002C2013002B8016002AE019002A401D046
:1042B000029A012003900170038601C0037C013043
:1042C000047201A004680120055E01B0055401607C
:1042D000064A0120074001F0073601F0082C0110C2
:1042E0000A2201500B1801C00C0E01500E040130BF
:1042F00010FA002012F0005014E600C016DC007026
:1043000019D200501CC800501FBE007022B400B06B
:1043100025AA00F028A000202C9600302F8C001039
:10432000328200A0347800F0366E00E038640080FD
:104330003A5A00403B5500E03B5000F03C4600C07C
:104340003D3C00603E3200E03E2800303F1E005001
:104350003F1900703F1400A03F0A00C03F0000D08A
:104360003FF6FFE03FECFF2020506C616E6E6572FF
:1043700042756666657242797465733A200020461C
:10438000726565204D656D6F72793A2000436F6DDF
:1043900070696C65643A204170722032342032308A
:1043A00032310A00204C6173742055706461746569
:1043B000643A20323032312D30342D3138207C2097
:1043C000417574686F723A2054696E794D61636803
:1043D000696E657333440A00322E302E375F4457BE
:1043E000372E330A004D61726C696E0020536F6680
:1043F00074776172652052657365740A0020576195
:10440000746368646F672052657365740A002042A4
:10441000726F776E206F75742052657365740A0031
:104420002045787465726E616C2052657365740AFC
:1044300000506F77657255700A0073746172740A68
:10444000004732385859004D3130303100657272B2
:104450006F722077726974696E6720746F20666965
:104460006C650A00446F6E6520736176696E672023
:1044700066696C652E0A004D323900456E647374AE
:104480006F7073002553202563202563202563204A
:10449000256300205A3A0020593A0020583A006516
:1044A0006E6473746F7073206869743A2000000042
:1044B0000A0B02090C0D0E0807030401000000009E
:1044C00000000000000000000000000000000000EC
:1044D00000000000000000000000121110000000A9
:1044E00000000000000000000000000000000000CC
:1044F00000000000004D6F76652025736D6D004D46
:104500006F766520302E316D6D004D6F76652031F0
:104510006D6D004D6F76652031306D6D004D6F769D
:10452000652041786973004578747275646572001E
:104530004D6F7665205A004D6F76652059004D6F9E
:104540007665205800433E3F3E4368616E676520B4
:1045500046696C616D656E7400556E6C6F616420A8
:1045600046696C616D656E74004C6F6164204669CC
:104570006C616D656E74005072656865617420438E
:104580007573746F6D0050726568656174202400E6
:104590004261636B0050726F62696E6720466169A9
:1045A0006C656400205A3A200020593A2000426588
:1045B0006420583A200070726F6D70745F007368E9
:1045C0006F7700627574746F6E00626567696E0064
:1045D00050757267654D6F726500506175736564E3
:1045E00000436F6E74696E7565004C6F61642046A0
:1045F000696C616D656E74205400496E73657274E8
:104600002066696C616D656E7420616E64207365EF
:104610006E64204D3130380A00220A00556E6B6EF0
:104620006F776E20636F6D6D616E643A202200209B
:1046300042002050006F6B0053755065522043526A
:104640002D32302052656164792E005072696E748B
:10465000696E672E2E2E005072696E74205061753F
:1046600073656400204500205A00205900204D3910
:104670003220580020453A00205A3A0020593A008A
:10468000583A0020746F6F206C6F6E6720657874E5
:10469000727573696F6E2070726576656E7465648D
:1046A0000A0020636F6C6420657874727573696F9B
:1046B0006E2070726576656E7465640A005265736B
:1046C000656E643A20006E6F74696669636174692F
:1046D0006F6E200000002200250028002B002E0015
:1046E0003100340002010000050108010B01000047
:1046F0002100240027002A002D0030003300010192
:104700000000040107010A01050505050705080861
:104710000808020202020A0A08080404040401014B
:104720000101010101010303030303030303040760
:1047300007070C0C0C0C0C0C0C0C020202020606F7
:104740000606060606060B0B0B0B0B0B0B0B0102EA
:104750001020200808102040102040800201020193
:10476000080402010102040810204080804020104B
:1047700008040201800402018040201008040201A4
:10478000080402010102040810204080010204080C
:1047900010204080A801B20111241FBECFEFD1E24A
:1047A000DEBFCDBF00E00CBF13E0A0E0B2E0E8E563
:1047B000FFEE02E00BBF02C007900D92AC39B107CB
:1047C000D9F729E1ACE9B3E001C01D92A537B207E2
:1047D000E1F713E2CBECD3E200E006C02197010938
:1047E000802FFE010F940974CA3CD10780E00807AE
:1047F000A9F70F943B620D949A770C940000FC018A
:1048000084910895FC018081089590E080E00895EE
:10481000CF93DF93DB01F9019C919130C1F094308B
:1048200080F094509C938830D1F4808191810097DE
:1048300071F0019791838083480F591FEA01188214
:1048400006C08C3539F49C5F9C93943041F4DF9121
:10485000CF9108958B3339F781E08C93F8CF208185
:104860003181B9016F5F7F4F71836083420F531FA6
:10487000EA018883808191818F3591056CF7E7CFBC
:104880000F931F9381E00091661710916717209195
:1048900068173091691740916217509163176091C2
:1048A000641770916517041715072607370708F472
:1048B00080E01F910F91089590E080E00895282FE7
:1048C0009091DD08833021F495FD0FC094FD0FC059
:1048D000892F90E0B0E0A0E004C0B695A795979529
:1048E00087952A95D2F78170089581E0089580E038
:1048F0000895CF92DF92EF92FF92CF93DF93EC0176
:10490000CC80DD80EE80FF8027E137EB41ED58EB76
:10491000C701B6010F94727687FD23C027E030E00F
:1049200040E753E4C701B6010F94206D1816CCF090
:10493000C880D980EA80FB8027E137EB41ED58EB56
:10494000C701B6010F94727687FD0BC0C1E027E066
:1049500030E040E753E4C701B6010F94206D18160C
:104960000CF4C0E08C2FDF91CF91FF90EF90DF909F
:10497000CF9008952F923F924F925F926F927F92C5
:104980008F929F92AF92BF92CF92DF92EF92FF925F
:104990000F931F93CF93DF93CDB7DEB72E970FB64C
:1049A000F894DEBF0FBECDBFE82ED62E042F122FF7
:1049B000282F30E03C872B87462F50E05A874987C5
:1049C00065E0F62EF29EC001F39E900D11249E87A5
:1049D0008D87FA01E80FF91FEE0FFF1FEE0FFF1F83
:1049E000E35EF94F60817181828193819B01AC010B
:1049F0000F940477882309F434C1E00E612F6D0D04
:104A0000FE9CF0011124A985BA85AE0FBF1FAA0F25
:104A1000BB1FAA0FBB1FA35EB94FAC901196BC90F1
:104A200011971296CC9012971396DC90E00EFE9C94
:104A3000A0011124A985BA85A40FB51FAA0FBB1F19
:104A4000AA0FBB1FA35EB94FEC901196FC90119773
:104A500012960C91129713969C90862F90E0AD853C
:104A6000BE85A80FB91FAA0FBB1FAA0FBB1FA35E4D
:104A7000B94F8C9011967C90119712966C9012976A
:104A800013965C90610F70E0AD85BE85A60FB71FD1
:104A9000AA0FBB1FAA0FBB1FA35EB94F4C90119664
:104AA0003C90119712961C91129713962C90E80F38
:104AB000F91FEE0FFF1FEE0FFF1FE35EF94FB081EE
:104AC000B98321812A8332813B8383818C83FA01DC
:104AD000E60FF71FEE0FFF1FEE0FFF1FE35EF94F0C
:104AE00090819D83A181AE83B281BF83238128877A
:104AF0009701402F592DB701802F992D0F940477DE
:104B0000882321F0E12CF12C00E0912C9501A601E5
:104B1000B501C6010F940477882319F05701C02E00
:104B2000D92C242D332D412F522D642D732D812FFF
:104B3000922D0F940477882321F0412C312C10E022
:104B4000212C282D372D462D552D682D772D862D7E
:104B5000952D0F940477882321F0842C732C612EDB
:104B6000522C2D813E814F8158856D817E818F81B0
:104B700098850F940477882321F01D821E821F825E
:104B8000188629813A814B815C8169817A818B8188
:104B90009C810F940477882341F03D8139834E81B5
:104BA0004A835F815B8388858C8385E0EB85FC8508
:104BB0008E9FD0018F9FB00D112429853A85A20FB9
:104BC000B31FAA0FBB1FAA0FBB1FA35EB94FBA87A3
:104BD000A9879501A601B501C6010F94127497012A
:104BE000402F592D0F9411746B017C01282D372D06
:104BF000462D552D682D772D862D952D0F941274E9
:104C0000242D332D412F522D0F9411749B01AC0193
:104C1000C701B6010F9412746B017C0129813A819E
:104C20004B815C8169817A818B819C810F941274A4
:104C30002D813E814F8158850F9411749B01AC01E9
:104C4000C701B6010F94127420E030E040E450E454
:104C50000F940C75A985BA856D937D938D939C9364
:104C600013972E960FB6F894DEBF0FBECDBFDF911F
:104C7000CF911F910F91FF90EF90DF90CF90BF9059
:104C8000AF909F908F907F906F905F904F903F90EC
:104C90002F900895129A0895269A2E9A0895EF92C9
:104CA000FF920F931F93CF93DF93EC018B017A0157
:104CB0008A859B858617970731F0888199810F94A3
:104CC000645A1B870A87B701888199810F948E4B9C
:104CD0002E813F81820F932F911D9F838E8390E0C1
:104CE00080E0DF91CF911F910F91FF90EF90089599
:104CF0009F92AF92BF92CF92DF92EF92FF920F936B
:104D00001F93CF93DF93EC018B01942EA52E8A8500
:104D10009B858617970731F0888199810F94645A93
:104D20001B870A8788859985019649F5BC800A8189
:104D30008E81080FC880D980D6015596ED91FC91DF
:104D4000C6011995B80EE92CFA2C10E0F701219153
:104D50007F01211127C08E819F81810F911D9F832B
:104D60008E8390E080E0DF91CF911F910F91FF90B3
:104D7000EF90DF90CF90BF90AF909F9008950E81FD
:104D80001F81692D7A2D888199810F948E4B800F18
:104D9000912F911D288539852817390738F681E02C
:104DA00090E0E1CF4B2D602FC6010F94BC5A080F45
:104DB000180FCCCFDF92EF92FF920F931F93CF93F8
:104DC000DF93EC01D62E1CAD0BAD7C0184E0E80E28
:104DD000F11CE98DFA8DC7011995412F480F2D2D32
:104DE000602FC7010F94BC5A9BAD890F8BAF81E038
:104DF00090E0DF91CF911F910F91FF90EF90DF90A6
:104E00000895AF92BF92DF92EF92FF920F931F939C
:104E1000CF93DF938C01EB01D42E79018FE04817FB
:104E200009F486C0A5E14A17B1F1BAE04B130EC0F0
:104E3000EC81FD8130E020E042E061E0C80119959D
:104E400045EA5AE1BE01C8010F94675B0A80DB8125
:104E5000C02DF2E3DF1609F4E2C0FD1508F491C09D
:104E600085E1D81609F4E0C0A7E1DA1609F4EFC02D
:104E7000B4E1DB127BC0EE81FF818D8190E0880F71
:104E8000991F8E0F9F1F11928E179F07E1F7CE017A
:104E90000F9484586BC0AA80BB8040E95AE1C801D6
:104EA0000F94675BF5014481440F406BBE01C8015C
:104EB0000F944F5B41E0BE01C8010F94575BD501D1
:104EC00016962D913C911797EC81FD8115964C918A
:104ED00066E0C801199540E0BE01C8010F945F5B10
:104EE00040E95AE1BE01C8010F94675BF5014481B6
:104EF000440F4F5F406BBE01C8010F944F5B41E010
:104F0000BE01C8010F94575BD50115964C911597BA
:104F100016962D913C91240F311DEC81FD8166E0A8
:104F2000C801199540E0BE01C8010F945F5B8ECFA8
:104F300041E0C8010F945F5B40E0BE01C8010F94DF
:104F4000575B41E8BE01C8010F944F5BF7014081F8
:104F500050E05595479555954795BE01C8010F946A
:104F60004F5B40E0BE01C8010F945F5B81E0DF91C1
:104F7000CF911F910F91FF90EF90DF90BF90AF9076
:104F80000895E6E4DE1609F471C0F7E4DF1609F4CB
:104F900071C08BE3D812EACFD70111969C9111977B
:104FA00013968C9138E0390F813031F0833011F055
:104FB000392F02C0392F985021E04B81491708F44E
:104FC00020E041E0391708F040E091E05A813517C0
:104FD00008F490E0322F342B932311F4242331F280
:104FE000F701128100E0D12C843048F490E0FC01FC
:104FF000E054FD4FD08084549D4FDC010C9117FF8D
:1050000004C0B701CE010F948B58F70180818D0D3C
:1050100080838181800F8183110F89F7A7CFB7012A
:10502000CE010F948B58A2CFCE010F946E588823D7
:1050300009F49DCFEE81FF818D8190E0880F991F4B
:105040008E0F9F1F11928E179F07E1F78FCFD70109
:105050001C928A8111968C9311978D8181501296A2
:105060008C9312978B8113968C9380CF8D81F7014F
:1050700080837CCF8981D7018C9378CFAB01BC0131
:10508000409366175093671760936817709369177A
:105090008FEC98E10C945FE580932F028032B8F595
:1050A00090916305891724F091E0980F9093630520
:1050B00040915F05509160056091610570916205B6
:1050C000082E04C076956795579547950A94D2F7B0
:1050D00041704093DA1087FD1DC0282F082E000C68
:1050E000330B3F938F9382E49AE09F938F9382E5F3
:1050F0009AE09F938F931F920E94F1C98DB79EB73C
:1051000007960FB6F8949EBF0FBE8DBF08951092FC
:10511000DA10E1CF0D9457470F931F93CF93DF938E
:1051200000D01F92CDB7DEB79C0108EA18E090E1ED
:10513000E3EDF9E0D80101900D929A95E1F7F901BC
:105140002081318142815381F8016085718582859A
:1051500093850F941274F801608771878287938713
:1051600080E090E0A0EAB0E489839A83AB83BC83BB
:10517000CE0101960F94DB180F900F900F900F90B7
:10518000DF91CF911F910F9108952F923F924F92EF
:105190005F926F927F928F929F92AF92BF92CF92C7
:1051A000DF92EF92FF921F93CF93DF93CDB7DEB7DD
:1051B0002C970FB6F894DEBF0FBECDBF7A01190150
:1051C000DC012D913D914D915C912D833E834F8368
:1051D0005887FB0140805180628073808090D309A2
:1051E0009090D409A090D509B090D609A50194015A
:1051F0006D817E818F8198850F94206D81110EC005
:1052000011E0A30192016091D7097091D8098091B2
:10521000D9099091DA090F94206D811110E0D10124
:105220002D913D914D915C9129873A874B875C8701
:10523000F701C080D180E280F38020911302309189
:1052400014024091150250911602C701B6010F9445
:10525000206D882309F44EC0C0921302D09214022C
:10526000E0921502F09216028091DF099091E00918
:10527000A091E109B091E2094091D7095091D80974
:105280006091D9097091DA098092A8089092A908D2
:10529000A092AA08B092AB084093AC085093AD0816
:1052A0006093AE087093AF08C092B008D092B10876
:1052B000E092B208F092B3088093B4089093B508D6
:1052C000A093B608B093B70820E030E040E05FE379
:1052D000609108117091091180910A1190910B1140
:1052E0000F94866D69837A838B839C83CE010196AC
:1052F0000F94DB182D813E814F8158852093A8089B
:105300003093A9084093AA085093AB084092AC0888
:105310005092AD086092AE087092AF08D1012D9105
:105320003D914D915C916091B4087091B508809168
:10533000B6089091B7080F9412746093B4087093F4
:10534000B5088093B6089093B70811112FC020E0DC
:1053500030E0A90169857A858B859C850F94206D45
:10536000811133C060E070E088EC92E469837A8355
:105370008B839C83CE0101960F94DB182C960FB67D
:10538000F894DEBF0FBECDBFDF91CF911F91FF908C
:10539000EF90DF90CF90BF90AF909F908F907F90D5
:1053A0006F905F904F903F902F9008952AEF3EE7C7
:1053B0004AE25FE360910C1170910D1180910E1122
:1053C00090910F110F94866DD1CF60E070E080EA6C
:1053D00091E4CCCFCF93DF9300D01F92CDB7DEB74F
:1053E00080E090E0A0EAB0E489839A83AB83BC8339
:1053F00061E0CE0101960F94E5100F900F900F9091
:105400000F90DF91CF91089580912205909123050F
:10541000009731F04AE050E070E060E00D943B6BA3
:1054200060E070E0CB0108958091E70982FF0BC036
:1054300063E686E29BE00E940CCA0F9478520E94B9
:1054400006D181E0089580E0089580912205909131
:105450002305009731F04AE050E070E060E00D94E1
:105460000D6A60E070E0CB0108950E94252A97FD47
:105470000CC00E94252A6F3F71058105910509F036
:1054800034F40E94252A862F089580E008958FEF36
:1054900008958091220590912305892B41F00E9467
:1054A000352A91E0811101C090E0892F089591E0A3
:1054B000FCCFCF92DF92EF92FF920F931F93CF9387
:1054C000DF936B017A01EC01C255DB4F28813CE090
:1054D000389F8001399F100D112427FF24C0FB0144
:1054E0001182108288818F5F888388819801280FBC
:1054F000311D87FD3A95C9012091D316F601281771
:10550000190629F024F088818C300CF43CC080818D
:105510009181049680349C4908F475C0F60180811D
:105520009181049672C088819801280F311D87FDF2
:105530003A95C9012091D3162817190699F294F2C9
:105540008881A801480F511D87FD5A95FA01EE0F79
:10555000FF1FE40FF51FE557F94E808187FFC2CF8B
:105560008881F801E80FF11D87FDFA95CF01EE0F54
:10557000FF1FE80FF91FE557F94E808160E08F7734
:105580000F941D50AFCF808191812881A801420FD7
:10559000511D27FD5A959A01FA01EE0FFF1FE20FE8
:1055A000F31FE557F94E21813281820F931FF701D6
:1055B0009183808388819801280F311D87FD3A955A
:1055C000F901EE0FFF1FE20FF31FE557F94E80813F
:1055D00087FF20C08881080F111D87FD1A95F801EB
:1055E000EE0FFF1FE00FF11FE557F94E808161E0DC
:1055F0008F77DF91CF911F910F91FF90EF90DF9008
:10560000CF900D941D5080E49CE9F7019183808335
:105610008FEF8883DF91CF911F910F91FF90EF90D3
:10562000DF90CF900895AF92BF92CF92DF92EF922A
:10563000FF920F931F93CF93DF93EC015B018A01DD
:10564000FB01199587FD16C0C82ED12CF12CE12C39
:105650002196F801C082D182E282F382CE01DF91ED
:10566000CF911F910F91FF90EF90DF90CF90BF905F
:10567000AF900895982F907E903CA9F48F7190E0A0
:10568000B0E0A0E06C017D0156E0CC0CDD1CEE1C0E
:10569000FF1C5A95D1F7CE010196F50119958F732C
:1056A000C82A2296D6CF982F907F903E11F58F7002
:1056B00090E0B0E0A0E06C017D0136E0CC0CDD1C98
:1056C000EE1CFF1C3A95D1F7CE010196F501199514
:1056D0008F73C82A46E0CC0CDD1CEE1CFF1C4A95DB
:1056E000D1F7CE010296F50119958F73C82A23963A
:1056F000B0CF982F987F903F79F5877090E0B0E019
:10570000A0E06C017D0186E0CC0CDD1CEE1CFF1CD2
:105710008A95D1F7CE010196F50119958F73C82AA4
:1057200096E0CC0CDD1CEE1CFF1C9A95D1F7CE0147
:105730000296F50119958F73C82A26E0CC0CDD1C62
:10574000EE1CFF1C2A95D1F7CE010396F5011995A1
:105750008F73C82A24967DCF982F907C903841F47F
:10576000807C803869F42196CE01F5011995F8CF37
:105770008E7F8D3F28F02196CE01F5011995F8CF47
:10578000C12CD12C760165CF9CE0899F802D1124FE
:1057900091E0980F909364052CE0280F2093A208C5
:1057A00030E02E5F3F4F409158174217130619F013
:1057B00014F080E0089520915A179217D0F76623CD
:1057C00041F08E5F0F947E598091A2088E5F0F94F6
:1057D0007E598091A20890915817891750F3209113
:1057E0005A1790916405291720F310925B17809344
:1057F0005C1781E0089520915605022E000C330BB2
:105800008217130641F08093560562ED7AE184E237
:1058100097E10D94645A08951F93CF93DF931F92DD
:10582000CDB7DEB78F3F910519F014F08FEF90E000
:105830008837910514F488E790E090935A0280939A
:105840005902182F80915D17811105C081E0809366
:105850005D170F94A558609126177091271719832B
:105860009E012F5F3F4F4FE084E297E10F94A158D4
:105870000F90DF91CF911F910895CF93809157059D
:1058800081114FC010925B1710925C1710925D1738
:10589000109229171092281710922B1710922A177E
:1058A00010922D1781E080932C1782E280932E179F
:1058B0001092331710923217E7E4F7E125E537E14C
:1058C0008FEF81932E173F07E1F7C1E0C093441794
:1058D00028E632E030933A1720933917C0933B17EC
:1058E00010923C1710923D1790E490933E1710923F
:1058F0003F1720E331E0309356172093551722E2EB
:1059000032E0309327172093261799E19093491797
:105910009BE190934817809347170F94A558C09325
:1059200057058091590290915A020E940C2C81E0F7
:105930008093580580E99AE190933D1680933C1638
:1059400010923F1610923E16CF910895CF92DF929B
:10595000EF92FF920F931F93CF93DF93CDB7DEB7F4
:105960002C970FB6F894DEBF0FBECDBF6F3F710509
:105970008105910509F0D0F480E297E10E94DA26D2
:10598000E0912817F09129173196849190E02C9698
:105990000FB6F894DEBF0FBECDBFDF91CF911F9140
:1059A0000F91FF90EF90DF90CF900895F0905B17EC
:1059B000E0905C172091580521110FC040E75AE193
:1059C0006E2D8F2D0F94285B90E080E0F80EF09202
:1059D0005B17E0925C179927DACFC0902817D09018
:1059E000291724E237E13A8329832F2D30E03C83C5
:1059F0002B832E2D30E03E832D8318861F822FEFC0
:105A00003FEF3A8729871C861B8608E716E29E012E
:105A10002F5F3F4FAB01BC01C6010F946930B60147
:105A200084E297E10F94645A8F819885CFCFCF930A
:105A3000DF93FC0125AD211104C021E025AF0F94B7
:105A4000A558C0912617D0912717E0915517F091CE
:105A5000561782E01995E0915517F091561781E09D
:105A6000199530E020E044E1BE0184E297E10F9413
:105A7000A15827E537E147E1BE0184E297E10F94A1
:105A8000A158E0915517F091561780E0DF91CF9122
:105A90001994CF92DF92EF92FF920F931F93CF93BF
:105AA000DF93CDB7DEB72C970FB6F894DEBF0FBEED
:105AB000CDBFF0905B17E0905C1720915805211145
:105AC0001DC040E55AE16E2D8F2D0F94285B90E0AC
:105AD00080E0F80EF0925B17E0925C1799272C9605
:105AE0000FB6F894DEBF0FBECDBFDF91CF911F91EF
:105AF0000F91FF90EF90DF90CF900895C0902817FE
:105B0000D090291724E237E13A8329832F2D30E002
:105B10003C832B832E2D30E03E832D8318861F82FD
:105B20007A8769871C861B8608E716E29E012F5F2D
:105B30003F4F4FEF53E2BC01C6010F942D31B60128
:105B400084E297E10F94645A8F819885C2CF6FEFFA
:105B50007FEF0C94492DCF92DF92EF92FF920F933B
:105B60001F93CF93DF93CDB7DEB72C970FB6F89482
:105B7000DEBF0FBECDBFF0905B17E0905C172091A9
:105B8000580521111DC040E35AE16E2D8F2D0F9451
:105B9000285B90E080E0F80EF0925B17E0925C17D3
:105BA00099272C960FB6F894DEBF0FBECDBFDF91BC
:105BB000CF911F910F91FF90EF90DF90CF900895BC
:105BC000C0902817D090291724E237E13A8329831F
:105BD0002F2D30E03C832B832E2D30E03E832D8310
:105BE00018861F827A8769871C861B8608E716E25B
:105BF0009E012F5F3F4F42E054E2BC01C6010F946B
:105C00002D31B60184E297E10F94645A8F81988513
:105C1000C2CFBF92CF92DF92EF92FF920F931F936A
:105C2000CF93DF938B01F42EE90141FB662760F9E6
:105C30000E94C42B882309F45AC0B12C0115110508
:105C400021F0C8010E94D7D1B82EE12C209721F075
:105C5000CE010E94C2D3E82E80E8C82ED12CF0FEDF
:105C60001EC085E190E08B199109B7FC93958E19C0
:105C70009109E7FC939597FD019695958795F82EE8
:105C800030E8C32ED12CFA94F7FC09C060E270E032
:105C900080E090E00E94A62CC81AD90AF4CFBB205D
:105CA00099F0C60166E070E00F94E173262F4091F1
:105CB000A4085091A5086091A308C8010E9417D1BB
:105CC00096E0899F60011124EE2031F0B601CE01EB
:105CD0000E94AB2DC81AD90A87E0C816D10438F043
:105CE00060E270E080E090E00E94A62CF3CFDF91AC
:105CF000CF911F910F91FF90EF90DF90CF90BF90C9
:105D000008956FEF7FEF0C94AB2DAF92BF92CF92BF
:105D1000DF92EF92FF920F931F93CF93DF935C017B
:105D20006B010E94D7D1E82EC6010E94C2D3F12C8C
:105D300003E110E0081B1109C5E20E151F050CF464
:105D4000CFE18C2F90E09C012E5F3F4F4091581780
:105D50004217130609F0CCF5099720915A17281716
:105D600019069CF14091A4085091A5086091A308E0
:105D700010925B17C0935C1725E1C5010E9417D1F3
:105D8000D1E0C114D104B1F06AE370E080E090E0AA
:105D90000E94A62C0E151F05D4F4C45F80915817DD
:105DA000C81740F020915A174C2F4950550B241713
:105DB00015067CF4DF91CF911F910F91FF90EF902A
:105DC000DF90CF90BF90AF900895D0E0DACFDD2381
:105DD00089F3802F880F080F000F00935B17C09383
:105DE0005C1760E270E080E090E00E94A62CC601A3
:105DF000DF91CF911F910F91FF90EF90DF90CF90A7
:105E0000BF90AF900C94812E8F929F92AF92BF92D1
:105E1000CF92DF92EF92FF920F931F93CF93DF9376
:105E2000CDB7DEB72C970FB6F894DEBF0FBECDBF4F
:105E3000982F862F5A017901D02E692F0E94C42BEA
:105E4000882309F489C0C701002391F10E94D7D1AA
:105E5000C82E80902817909029178091580581119D
:105E600045C01FEF23E12C194091A4085091A508CB
:105E70006091A308C5010E9417D1CC2009F46CC021
:105E8000B6E08B9F500111246AE370E080E090E05F
:105E90000E94A62C57E0A516B10408F444C060E2A5
:105EA00070E080E090E00E94A62CA81AB90AF2CF18
:105EB0000E94C2D3C82E80902817909029178091F5
:105EC0005805882371F2FE0133968AE0DF011D92A6
:105ED0008A95E9F784E297E19A8389830FE416E2D1
:105EE0009E012F5F3F4F42E054E212C0FE01339605
:105EF0008AE0DF011D928A95E9F784E297E19A83AF
:105F000089830FE416E29E012F5F3F4F4FEF53E26C
:105F1000B701C4010F942D31B40184E297E10F94CD
:105F2000645A1F819FCF4091A208212F30E0A6E044
:105F3000CA9EC00111242E5F3F4F281739070CF469
:105F40009C0180E8821B80935B1740935C17C7011C
:105F5000DD20A9F00E94A72D2C960FB6F894DEBF85
:105F60000FBECDBFDF91CF911F910F91FF90EF90AA
:105F7000DF90CF90BF90AF909F908F9008950E9438
:105F8000812EEACFE0E2F7E183AF64AFCA010C945F
:105F9000812E2F923F924F925F926F927F928F92BB
:105FA0009F92AF92BF92CF92DF92EF92FF920F93A8
:105FB0001F93CF93DF93D62FC72FFC018080918052
:105FC000A280B380C501B40120E831E541E050E092
:105FD0000F946473C9016DE671E00F94E1736B0176
:105FE0007C01C501B40120E13EE040E050E00F94A7
:105FF0006473CA01B90128E130E040E050E00F9439
:106000006473362E272E062F172F8CE3482E512C23
:10601000612C712CC501B401A30192010F9464732A
:10602000B62EA72ECA01B901A30192010F94647381
:10603000CB01C114D10479F1AF92BF927F936F93DA
:106040002F923F92FF92EF92DF92CF928EE898E1EB
:106050009F938F93CF93DF930F94B76C8DB79EB7B9
:106060000E960FB6F8949EBF0FBE8DBF8D2F9C2F3E
:10607000DF91CF911F910F91FF90EF90DF90CF9024
:10608000BF90AF909F908F907F906F905F904F9058
:106090003F902F900895E114F104C9F0AF92BF92A0
:1060A0007F936F932F923F92FF92EF928EE798E14A
:1060B0009F938F93CF93DF930F94B76CEDB7FEB799
:1060C0003C960FB6F894FEBF0FBEEDBFCFCF012BAD
:1060D000B9F0AF92BF927F936F932F923F9282E776
:1060E00098E19F938F93CF93DF930F94B76C8DB705
:1060F0009EB70A960FB6F8949EBF0FBE8DBFB6CF5F
:10610000892BA9F0AF92BF927F936F938AE698E1B3
:106110009F938F93CF93DF930F94B76CEDB7FEB738
:1061200038960FB6F894FEBF0FBEEDBF9FCFAF926B
:10613000BF9286E698E19F938F93CF93DF930F945E
:10614000B76C0F900F900F900F900F900F908ECF15
:106150008F929F92AF92BF92CF92DF92EF92FF9277
:106160000F931F93CF93DF93109255051092540510
:106170002FE320934F0510924E0510924D0510927B
:106180004C05109250051092510510925205109234
:1061900053059C01F90190812F5F3F4F9032D1F35D
:1061A0009E34C9F4818190ED980F9A3020F08D32A1
:1061B00011F08B3281F432969F012F5F3F4F808127
:1061C00080538A3008F47BC09F012F5F3F4F80814E
:1061D000803209F476C0F093C608E093C5088F01B9
:1061E0000F5F1F4FC0816AE270E0C8010F946077B3
:1061F000009731F0FC01319780818032E1F3118208
:10620000CD3429F0C43519F0C73409F04BC0F8017A
:1062100080810F5F1F4F8032D1F380538A3008F0A6
:1062200041C0C0934F0530E020E04AE0DF01119605
:10623000429FC001439F900D11249C0120533109BE
:106240008081280F311D87FD3A95818190ED980F4F
:106250009A30C8F130934E0520934D058E3261F48B
:10626000329690E04AE0DF0131968C9150ED580F64
:106270005A3058F190934C05CD01DC0101964C91B8
:106280004032D9F3CD3489F52E31310539F018F586
:106290002731310519F02C31310539F5B093550509
:1062A000A0935405DF91CF911F910F91FF90EF9034
:1062B000DF90CF90BF90AF909F908F900895F9019D
:1062C0007BCFF90181CFFD01B1CF949F800D1124C7
:1062D00090ED980FC8CF2537310538F027373105B5
:1062E000E8F2203A83E03807C9F2D091C50840E0CF
:1062F00050E0BA0110E000E0C12CD12C7601C3942B
:10630000FD0131968C91882309F47FC08132E1F43C
:10631000CD34D1F420323105B9F440935005509377
:1063200051056093520570935305F0935505E09322
:10633000540563E270E0CF010F946077009709F491
:10634000B1CFFC011082AECF81548A3108F058C021
:10635000DF019D91903291F0A0EDA90FAA30E8F0F5
:106360009E3271F4918190539A30B8F00115110565
:1063700019F48F010150110990E013C0FD01E8CF1D
:106380009D3211F09B3291F79181A0EDA90FAA30B7
:1063900020F09E3259F79281E6CF9E2F9D1B3097B9
:1063A00059F3A82FB0E04601570104C0880C991C8E
:1063B000AA1CBB1C8A95D2F7482959296A297B292E
:1063C000AE5CBA4F9C9380818154DF018A3108F41E
:1063D00097CFDF018191882309F492CF90ED980F38
:1063E0009A30B8F393ED980F923098F38B3289F38B
:1063F000CD010196EC91E03209F082CFDC01F8CFBB
:106400000115110501F78D01DECF1093550500939D
:106410005405409350055093510560935205709375
:10642000530540CFFC016591759185919491089534
:106430008091B908882319F080E00F943E1C80E019
:1064400008954F925F926F927F928F929F92AF9238
:10645000BF92CF92DF92EF92FF92CF93DF9300D063
:1064600000D01F921F92CDB7DEB75C01DB01CD904B
:10647000DD90ED90FC90E091E316F091E416FE8340
:10648000ED8384819581A681B78189839A83AB83CB
:10649000BC839C01AD01C701B6010F9411742B019F
:1064A0003C01F50180809180A280B380AD81BE81E6
:1064B0008D919D910D90BC91A02D8D839E83AF8376
:1064C000B88727E137EB41ED58EBC301B2010F94D8
:1064D000727687FDD0C027E030E040E753E4C30187
:1064E000B2010F94206D18160CF4C5C02D813E81A9
:1064F0004F815885C501B4010F9411742B013C01E3
:1065000027E137EB41ED58EB0F94727687FDB3C06E
:1065100027E030E040E753E4C301B2010F94206D5F
:1065200018160CF4A8C020E030E0A9016D817E812E
:106530008F8198850F9412742B013C0120E030E08C
:1065400040E450E40F94206D87FF05C0412C512C8E
:1065500030E4632E762C27E137EB41ED58E3C3019D
:10656000B2010F9411749B01AC01C501B4010F94E9
:10657000727687FD80C020E030E040E753E46D8113
:106580007E818F8198850F9412742B013C0120E04D
:1065900030E043E653E40F947276181634F4412C3D
:1065A000512C23E6622E23E4722E27E137EB41EDD6
:1065B00058E3C301B2010F9412749B01AC01C501F1
:1065C000B4010F94206D18160CF455C020E030E093
:1065D000A90169817A818B819C810F9412744B018E
:1065E0005C0120E030E040E951E40F94206D87FF2A
:1065F00006C0812C912C90E9A92E91E4B92E27E1B7
:1066000037EB41ED58E3C501B4010F9411749B01C0
:10661000AC01C701B6010F94727687FD2CC020E053
:1066200030E040E753E469817A818B819C810F944B
:1066300012744B015C0120E030E044E553E40F9418
:106640007276181634F4812C912C84E5A82E83E4FC
:10665000B82E27E137EB41ED58E3C501B4010F94A3
:1066600012749B01AC01B1E0B983C701B6010F946C
:10667000206D18160CF41982898128960FB6F894AB
:10668000DEBF0FBECDBFDF91CF91FF90EF90DF90C7
:10669000CF90BF90AF909F908F907F906F905F90C2
:1066A0004F9008958F929F92AF92BF92CF92DF92B8
:1066B000EF92FF92CF93DF93EC018090DE089090F1
:1066C000DF08A090E008B090E10820E030E0A901E8
:1066D000C501B4010F94206D882309F452C0C8800D
:1066E000D980EA80FB80A7019601C501B4010F940F
:1066F000206D18160CF04AC020911E0530911F0520
:106700004091200550912105C701B6010F94206DDD
:10671000882321F1C0921E05D0921F05E09220052A
:10672000F092210520911A0530911B0540911C051E
:1067300050911D05C701B6010F94866D9B01AC01F8
:1067400060E070E080E89FE30F941174609317029B
:10675000709318028093190290931A0260911702A5
:10676000709118028091190290911A02DF91CF91D5
:10677000FF90EF90DF90CF90BF90AF909F908F9061
:10678000089560E070E080E89FE3F0CF60E070E0A3
:10679000CB01ECCF9B01AC01485F5F4FBC016C5F4C
:1067A0007F4F0C94C5280F931F93CF93DF9300D096
:1067B00000D01F921F92CDB7DEB7FC018B0183A5DD
:1067C000811112C081E083A784819581A681B78160
:1067D000B05889839A83AB83BC83BE016F5F7F4FC0
:1067E00088EA98E00E94CA331D821E821F821886A2
:1067F00020E030E040E05FE36091DB097091DC096C
:106800008091DD099091DE090F94127469837A8377
:106810008B839C839E012B5F3F4FAE014F5F5F4F89
:1068200067ED79E083ED99E00E94C5281D821E8204
:106830001F82188620E030E040E05FE3F8016085C9
:106840007185828593850F94127469837A838B8313
:106850009C83B8016C5F7F4F9E012B5F3F4FAE0161
:106860004F5F5F4FC8010E94C52828960FB6F89465
:10687000DEBF0FBECDBFDF91CF911F910F91089565
:106880002F923F924F925F926F927F928F929F9240
:10689000AF92BF92CF92DF92EF92FF920F931F932E
:1068A000CF93DF93CDB7DEB7A2970FB6F894DEBFD4
:1068B0000FBECDBF8C011B015E834D834090D30979
:1068C0005090D4096090D5097090D6098090D7096E
:1068D0009090D809A090D909B090DA09DB018D9188
:1068E0009D910D90BC91A02D8F87988BA98BBA8B11
:1068F0009C01AD01C301B2010F9411746B017C01C5
:10690000D10114968D919D910D90BC91A02D8B8BF2
:106910009C8BAD8BBE8B9C01AD01C501B4010F9466
:1069200011746F8B788F898F9A8FAD81BE818D9115
:106930009D910D90BC91A02D8F839887A987BA87D0
:106940009C01AD01C301B2010F9411746B8F7C8F58
:106950008D8F9E8FAD81BE8114968D919D910D90EE
:10696000BC91A02D8B879C87AD87BE879C01AD0114
:10697000C501B4010F9411746F8F78A389A39AA3F2
:10698000A7019601C701B6010F94866D6B017C01CA
:106990002F89388D498D5A8DCA01B9010F94866DA2
:1069A0009B01AC01C701B6010F9412744B015C014D
:1069B0002F85388949895A896F81788589859A8593
:1069C0000F9411742B013C012B893C894D895E8900
:1069D0006B857C858D859E850F9411746B017C0180
:1069E000A3019201C301B2010F94866D2B013C01FA
:1069F000A7019601C701B6010F94866D9B01AC01FA
:106A0000C301B2010F9412740F94C0766B017C0124
:106A10002B8D3C8D4D8D5E8DCA01B9010F94866D15
:106A20002B013C012F8D38A149A15AA1CA01B901FE
:106A30000F94866D9B01AC01C301B2010F941274D7
:106A40009B01AC01C501B4010F9472761816B4F520
:106A500020E030E0A901C701B6010F94727687FFEC
:106A60002AC0C701B601905820E030E040EA50E467
:106A70000F947276181614F5A1016D817E81C801FC
:106A80000E944034A2960FB6F894DEBF0FBECDBF71
:106A9000DF91CF911F910F91FF90EF90DF90CF90FA
:106AA000BF90AF909F908F907F906F905F904F902E
:106AB0003F902F900895C701B601D6CF20E030E077
:106AC00040E050E4C501B4010F947276181624F426
:106AD000B101C8010E94D33319821A821B821C8221
:106AE000BE016F5F7F4FC1010E94CA332DEC3CECA9
:106AF0004CEC5CE3C701B6010F94866D9B01AC01C1
:106B0000F80160817181828193810F94866D698320
:106B10007A838B839C83C8010F94C04ABE016F5F48
:106B20007F4F8D819E810E94CA33ACCF3F924F929E
:106B30005F926F927F928F929F92AF92BF92CF920D
:106B4000DF92EF92FF920F931F93CF93DF93CDB716
:106B5000DEB76C970FB6F894DEBF0FBECDBFDB017A
:106B60000C91142F100F153008F067C11196DC90AE
:106B7000C22ECD0CB4E0BC1508F45FC1ED2DF0E0E1
:106B8000EF5EFA4F8080912CB12CA12C002E04C016
:106B9000B694A794979487940A94D2F780FE4DC137
:106BA000EC2DF0E0EF5EFA4F8080912CB12CA12CFF
:106BB000012E04C0B694A794979487940A94D2F7B0
:106BC00080FE3BC1322E642F7C01409081065090A4
:106BD0008206609083067090840680918906909169
:106BE0008A06A0918B06B0918C06898F9A8FAB8F05
:106BF000BC8F660F770B072E000C880B990B0F9438
:106C0000276D4B015C01602F000F770B880B990BF0
:106C10000F94276D298D3A8D4B8D5C8D0F94866D69
:106C2000A30192010F941274A50194010F941274A0
:106C30006D877E878F87988B612F110F770B880B5D
:106C4000990B0F94276D298D3A8D4B8D5C8D0F9488
:106C5000866DA30192010F941274A50194010F9403
:106C6000117469837A838B839C834090850650904E
:106C70008606609087067090880680918D069091B8
:106C80008E06A0918F06B0919006898F9A8FAB8F58
:106C9000BC8F632D660F770B072E000C880B990BAA
:106CA0000F94276D4B015C016D2DDD0C770B880B6C
:106CB000990B0F94276D298D3A8D4B8D5C8D0F9418
:106CC000866DA30192010F941274A50194010F9493
:106CD0001274698B7A8B8B8B9C8B6C2DCC0C770B05
:106CE000880B990B0F94276D298D3A8D4B8D5C8DF8
:106CF0000F94866DA30192010F941274A501940163
:106D00000F9411746D837E838F839887F70180853C
:106D10009185A285B38589879A87AB87BC878D8B40
:106D20009E8BAF8BB88F4FEE50E061E070E0CE01EC
:106D300041960E9447F44FEE50E061E070E0CE01D2
:106D400005960E9447F44FEE50E061E070E0CE01FE
:106D50000D960E9447F44FEE50E061E070E0CE01E6
:106D600001960E9447F489889A88AB88BC8827E1FD
:106D700037EB41ED58EBC501B4010F94727687FDF6
:106D80005CC027E030E040E753E4C501B4010F9454
:106D9000206D18160CF451C08D849E84AF84B88881
:106DA00027E137EB41ED58EBC501B4010F94727642
:106DB00087FD43C027E030E040E753E4C501B4015C
:106DC0000F94206D1816CCF18D809E80AF80B88412
:106DD00027E137EB41ED58EBC501B4010F94727612
:106DE00087FD2BC027E030E040E753E4C501B40144
:106DF0000F94206D18160CF189809A80AB80BC80AE
:106E000027E137EB41ED58EBC501B4010F947276E1
:106E100087FD13C027E030E040E753E4C501B4012B
:106E20000F94206D18164CF0AE014F5F5F4FBE01FE
:106E3000635F7F4FC7010E9440346C960FB6F89491
:106E4000DEBF0FBECDBFDF91CF911F910F91FF909D
:106E5000EF90DF90CF90BF90AF909F908F907F90FA
:106E60006F905F904F903F9008958C38910514F08B
:106E70008CE890E09093EA088093E9080C94AEDCEB
:106E80000E94252ACB0108950F931F93CF938091E1
:106E90002205909123050097E9F0FC018F01C19133
:106EA0002C2F2F7D81F0C53411F0C536B9F7F801CC
:106EB000108270E060E00F94AF68F801C083CF915A
:106EC0001F910F91089570E060E0CF911F910F9195
:106ED0000D94AF6860E070E0CB01F1CF2FEB280F8D
:106EE0002A3108F047C0E22FF0E0809150059091E0
:106EF0005105A0915205B091530504C0B695A795D0
:106F0000979587952A95D2F780FD02C081700895E4
:106F1000EE5CFA4FE081EE2341F18091C50890913B
:106F2000C608E80FF92FF11D808190ED980F9A3077
:106F300030F08E3251F4818180538A3098F4F0938E
:106F40002305E093220581E008958D3211F08B3204
:106F500049F4818190ED980F9A3088F38E3211F4C4
:106F60008281EACFF0E0E0E0EACF109223051092B0
:106F70002205E9CF80E008950E946E37882341F012
:106F800081E02091220530912305232B09F480E034
:106F90000895CF93DF93EB010E94BC37882319F04B
:106FA0000E94252AEB01CE01DF91CF91089583E560
:106FB0000E94BC378823E9F00F943F526093BA08CF
:106FC0007093BB088093BC089093BD080E9444371F
:106FD00020E030E04AE754E40F94866D0F94857505
:106FE00060931B0270931C0280931D0290931E02FB
:106FF00008958091500584FD0AC08091520587FD57
:1070000006C080915305837011F40C941DFB0E94FF
:107010000CFB88E50E946E37882331F05F9A8091DF
:10702000B8088E7F8093B80889E50E946E37882360
:1070300031F08A9A8091B8088D7F8093B8088AE5EC
:107040000E946E37882359F08091080180958170E5
:10705000809306018091B8088B7F8093B80885E4FF
:107060000E946E3781110C944A260895CF93C62F43
:107070000E94BC37882319F0CF910C94352A8C2FAD
:10708000CF910895CF92DF92EF92FF926A017B0138
:107090000E94BC37882331F0FF90EF90DF90CF90B3
:1070A0000C944437C701B601FF90EF90DF90CF906A
:1070B00008954F925F926F927F928F929F92AF92BC
:1070C000BF92CF92DF92EF92FF921F93CF93DF9305
:1070D00000D01F92CDB7DEB719821A821B821C82A4
:1070E000CE0101964C0183EDC82E89E0D82E98EA96
:1070F000E92E98E0F92E27ECA22E29E0B22E10E01E
:1071000088E5810F0E94BC37F40181934F018823E9
:1071100041F00E9444372B013C018091DA10882312
:1071200059F0F60180819181A281B381F7018083BA
:107130009183A283B38314C0812F0E945F2488238C
:1071400009F4D0C0F6012081318142815381C3010D
:10715000B2010F941274F701608371838283938369
:107160001F5FF4E0CF0ED11C84E0E80EF11C94E028
:10717000A90EB11C133021F685E40E94BC378C8324
:10718000882309F4B9C00E9444376B017C0183E075
:107190000E945F24882371F02091DF093091E0097B
:1071A0004091E1095091E209C701B6010F941274B0
:1071B0006B017C01C092B408D092B508E092B60889
:1071C000F092B70880911C06882359F180916A17C4
:1071D00082FF27C08C81882321F18981811103C01E
:1071E0008A818823F1F02DEC3CEC4CE45DE3609166
:1071F0001E0970911F0980912009909121090F9417
:1072000012749B01AC016091DB097091DC098091E3
:10721000DD099091DE090F947276181614F40F941C
:10722000135D40E050E0BA0186E40E94423820E05D
:1072300030E0A9010F947276181684F40E94443746
:1072400020E030E040E752E40F940C756093850233
:107250007093860280938702909388028091DB105E
:1072600083FD2CC08091DA10811128C080911B0809
:10727000882321F12091DF093091E0094091E10953
:107280005091E2096091B4087091B5088091B608F8
:107290009091B7080F941174209128083091290813
:1072A00040912A0850912B080F941274609328087B
:1072B0007093290880932A0890932B080F900F90C1
:1072C0000F900F90DF91CF911F91FF90EF90DF9083
:1072D000CF90BF90AF909F908F907F906F905F9076
:1072E0004F900895F5012081318142815381C3017E
:1072F000B2010F9411742FCF8091DF099091E009B2
:10730000A091E109B091E2098093B4089093B50887
:10731000A093B608B093B70855CFCF93DF93EB0196
:107320000E94BC37882321F0DF91CF910C94403725
:10733000CE01DF91CF910895CF93DF93C82FD62F41
:107340000E94BC37882321F0DF91CF910C94492A09
:107350008C2F0E946E37811101C08D2FDF91CF914C
:107360000895E5E1F9E082EBDF011D928A95E9F7E6
:10737000089580911C06811104C00E94B1390D94BA
:10738000E15D80916A1782FD0D94135D08958091EF
:107390001509882361F09091C609891308C080916E
:1073A0006A1783FF04C083E599E00D94205C80E0B8
:1073B0000895FC01238121110C9420E90895CF92B6
:1073C000DF92EF92FF920F931F93CF939091300231
:1073D000913009F461C0662351F0109200051092BB
:1073E000FC041092FD041092FE041092FF04C82FBA
:1073F0000F943F52C090FC04D090FD04E090FE0436
:10740000F090FF049B01AC012C193D094E095F0966
:1074100069017A01F7FC40C020910005C7FD15C045
:107420004C2F0C2E000C550B4C5F5F4FE22F022EA1
:10743000000CFF0B4E175F077CF144EFC42EDD24D8
:10744000D394E12CF12C2C1734F438EEC32E33E016
:10745000D32EE12CF12CC60ED71EE81EF91EC092C9
:10746000FC04D092FD04E092FE04F092FF04022F8F
:10747000017010E084E2809FB001819F700D701B4D
:10748000112460597C4F82E390E00E9433958091F3
:1074900000058F5F80930005CF911F910F91FF90A2
:1074A000EF90DF90CF9008950F931F9301E010E0CD
:1074B00020E030E0082E04C0000F111F221F331FF0
:1074C0000A94D2F740915F05509160056091610583
:1074D00070916205402B512B622B732B40935F05FB
:1074E00050936005609361057093620590912F023F
:1074F000891303C081E08093DA101F910F910895E2
:107500004F925F926F927F928F929F92AF92BF92B3
:10751000CF92DF92EF92FF920F931F93CF93DF935F
:10752000EC012091810630918206409183065091B2
:107530008406688179818A819B810F9411746B0123
:107540007C012091850630918606409187065091F6
:1075500088066C817D818E819F810F9411744B010F
:107560005C01A701960160910B0270910C02809161
:107570000D0290910E020F94206D882309F450C0E3
:10758000C0920B02D0920C02E0920D02F0920E0219
:107590002091F4043091F5044091F6045091F704E1
:1075A000C701B6010F94866D2B013C010F94B47591
:1075B0006B017C0120E030E0A9010F94206D87FD74
:1075C00070C020E030E040E450E4C701B6010F9401
:1075D000727618162CF4C12CD12CC0E4EC2EFE2CA3
:1075E000A7019601C301B2010F9411746093EC04DA
:1075F0007093ED048093EE049093EF04C701B601FD
:107600000F947E756093EA04062E000C770B6F5F73
:107610007F4F6430710514F064E070E06093E8041B
:10762000D09109021091EA04A501940160910F0222
:107630007091100280911102909112020F94206DAE
:10764000811133C0D11381C02091D0043091D10475
:107650004091D2045091D3046091EC047091ED04F8
:107660008091EE049091EF040F94866D2091D404E4
:107670003091D5044091D6045091D7040F941274E0
:10768000DF91CF911F910F91FF90EF90DF90CF90FE
:10769000BF90AF909F908F907F906F905F904F9032
:1076A0000895C12CD12C76019BCF80920F0290922D
:1076B0001002A0921102B09212022091F8043091AF
:1076C000F9044091FA045091FB04C501B4010F94F0
:1076D000866D4B015C010F94B4756B017C0120E059
:1076E00030E0A9010F94206D87FDF3C020E030E069
:1076F00040E450E4C701B6010F94727618162CF4DA
:10770000C12CD12CB0E4EB2EFE2CA7019601C501B3
:10771000B4010F9411746093F0047093F10480939A
:10772000F2049093F304C701B6010F947E75609341
:10773000EB04062E000C770B6F5F7F4F64307105F2
:1077400014F064E070E06093E904C091EB04D1139D
:1077500005C080910A028C1709F470C08091EA0478
:107760009091EB0490930A02809309020C2E000C76
:10777000DD0B25E01203C0011124FC01EC0FFD1FFD
:10778000EE0FFF1FEE0FFF1FE35EF94F20813181E7
:10779000428153812093E4043093E5044093E6044E
:1077A0005093E7040091E904002E000C110BFC013A
:1077B000E00FF11FEE0FFF1FEE0FFF1FE35EF94F0B
:1077C00060817181828193810F9411746093E004D0
:1077D0007093E1048093E2049093E3042091E80421
:1077E00035E02303F0011124CE0FDF1FCC0FDD1F86
:1077F000CC0FDD1FC35ED94F288139814A815B815F
:107800002093DC043093DD044093DE045093DF04C6
:10781000E00FF11FEE0FFF1FEE0FFF1FE35EF94FAA
:1078200060817181828193810F9411746093D80477
:107830007093D9048093DA049093DB048090F00471
:107840009090F104A090F204B090F3042091E00431
:107850003091E1044091E2045091E304C501B40188
:107860000F94866D2091E4043091E5044091E60484
:107870005091E7040F9412746B017C01C092D40400
:10788000D092D504E092D604F092D7042091D80487
:107890003091D9044091DA045091DB04C501B40160
:1078A0000F94866D2091DC043091DD044091DE045C
:1078B0005091DF040F941274A70196010F94117474
:1078C0006093D0047093D1048093D2049093D30436
:1078D000BBCEC12CD12C760118CF1F93CF93DF9351
:1078E000CDB7DEB72C970FB6F894DEBF0FBECDBF75
:1078F000182F882379F020E030E0A90160918906F3
:1079000070918A0680918B0690918C060F94206D61
:107910008823F9F08091E2088117D9F00E940CFBCE
:107920008CE0E4E9F2E0DE01119601900D928A9577
:10793000E1F7CE0101960E94803A8091E208882307
:1079400091F083ED99E00E942FFB1092E2080F94D2
:10795000EA112C960FB6F894DEBF0FBECDBFDF91B3
:10796000CF911F91089581E08093E20883ED99E023
:107970000E945CFAECCF80E00E946D3C109285067C
:107980001092860610928706109288061092810641
:1079900010928206109283061092840610928D0631
:1079A00010928E0610928F06109290061092890601
:1079B00010928A0610928B0610928C06EDE1F6E08A
:1079C00021E836E080E090E0A0ECBFE7808391837F
:1079D000A283B38384839583A683B78380879187AB
:1079E000A287B38784879587A687B787808B918B7B
:1079F000A28BB38B74962E173F0741F708954F92D1
:107A00005F926F927F928F929F92AF92BF92CF922E
:107A1000DF92EF92FF921F93CF93DF93EC01162F2B
:107A20002091DE083091DF084091E0085091E10894
:107A3000688179818A819B810F94206D882309F464
:107A4000AEC0B090E20880E00E946D3CC880D98052
:107A5000EA80FB8020E030E0A901C701B6010F9465
:107A6000727618161CF0C12CD12C7601C092DE085B
:107A7000D092DF08E092E008F092E1082DEB37E3C6
:107A800046E855EBC701B6010F94727687FD0BC02F
:107A90002DEB37E346E855E3C701B6010F94206D9F
:107AA00018160CF078C0A701960160E070E080E83D
:107AB0009FE30F940C7560931A0570931B058093D8
:107AC0001C0590931D0580EF9FEFA9E7B4EC809310
:107AD0001E0590931F05A0932005B0932105BB20A0
:107AE00009F45DC04090D3095090D4096090D50945
:107AF0007090D6098090D7099090D809A090D909A4
:107B0000B090DA09C090DB09D090DC09E090DD0983
:107B1000F090DE0981E00E946D3C112309F43FC022
:107B20002091D3093091D4094091D5095091D609BB
:107B3000C301B2010F94206D81111CC02091D7099F
:107B40003091D8094091D9095091DA09C501B401A1
:107B50000F94206D81110EC02091DB093091DC095A
:107B60004091DD095091DE09C701B6010F94206DE7
:107B70008823A9F0DF91CF911F91FF90EF90DF90C4
:107B8000CF90BF90AF909F908F907F906F905F90BD
:107B90004F900D946B1960E070E0CB018CCFDF91BA
:107BA000CF911F91FF90EF90DF90CF90BF90AF905B
:107BB0009F908F907F906F905F904F9008958F92DD
:107BC0009F92AF92BF92CF92DF92EF92FF92C090BE
:107BD0008906D0908A06E0908B06F0908C0620E013
:107BE00030E0A901C701B6010F94206D8823E1F1AF
:107BF000A701960160E070E080E89FE30F940C75A8
:107C00006B017C0180908D0690908E06A0908F066F
:107C1000B090900620E030E0A901C501B4010F94B6
:107C2000206D882329F1A501940160E070E080E8CF
:107C30009FE30F940C75C092F404D092F504E09287
:107C4000F604F092F7046093F8047093F9048093BB
:107C5000FA049093FB04FF90EF90DF90CF90BF90D9
:107C6000AF909F908F900895C12CD12C7601CACFF0
:107C700060E070E0CB01DFCFEFE6F0E08081826072
:107C8000808308958091BE089091BF08892B79F474
:107C90008091BE089091BF08892B49F42091BE08BD
:107CA0003091BF0881E0232B19F480E0089581E032
:107CB0000895CF92DF92EF92FF926B017C0183E3F4
:107CC000C816D104E104F10470F082E3C81AD108A7
:107CD000E108F10862E370E080E090E00F940C525C
:107CE0000F94EC11ECCFC701B6010F940C52FF902A
:107CF000EF90DF90CF900D94EC118091A806811148
:107D00000AC08091DC08813041F080916A1782FBC3
:107D1000882780F9089580E0089581E008955F9AAA
:107D20008091B8088E7F8093B8088A9A8091B808AD
:107D30008D7F8093B8088091080180958170809331
:107D400006018091B8088B7F8093B8080C944A266E
:107D500090916A1793FB882780F993FF06C081E012
:107D60009091D218911101C080E008958091A806E9
:107D7000811110C08091DC08823061F00E94A83E21
:107D8000882349F080916A1782FB882780F991E067
:107D90008927089581E008950E94B63E81110DC0A3
:107DA00010925F05109260051092610510926205B5
:107DB000109263058FEF0E944C280D945C2081E0A7
:107DC0000D94CC1FE5E1FAE010821182089581E064
:107DD0000895DC01EC918E2F90E0FC01EE0FFF1F67
:107DE000E80FF91FE557F94E80818F77808308955A
:107DF0008F929F92AF92BF92CF92DF92EF92FF92BB
:107E00000F93CF93DF931F92CDB7DEB75C017B0159
:107E100049016B01C40ED51EF501808191810F943B
:107E20003E738983002311F0F7018083BE016F5FE9
:107E30007F4FC4010F945330F501808191810196E9
:107E400091838083FFEFEF1AFF0AEC14FD0421F702
:107E500080E00F90DF91CF910F91FF90EF90DF9036
:107E6000CF90BF90AF909F908F900895009781F42E
:107E70001092900082E080939100109295001092F1
:107E80009400C19A8091710082608093710008957E
:107E9000019761F41092A00082E08093A1001092FB
:107EA000A5001092A40089BB8093720008957F9270
:107EB0008F929F92AF92BF92CF92DF92EF92FF92FA
:107EC0000F931F93CF93DF93EC017B01888188315F
:107ED00008F0C3C090E0FC01EE0FFF1FE80FF91F90
:107EE000E557F94E80818F770F94113219821A82EB
:107EF00088812CE0622F0F94C773829FB0011124F8
:107F000030E020E0AB01420F531FFA01EE0FFF1FDC
:107F1000E40FF51FE557F94E908197FD08C02F5FDC
:107F20003F4F2C30310571F790E00E94363F78804A
:107F3000072D10E06801CC0CDD1CF601E00FF11FED
:107F4000E557F94E80818068808377FC86C080E2A7
:107F5000E81682E0F8060CF03FC08A8128E532E09E
:107F6000281B310987FD3395220F331F220F331F42
:107F7000032E000C440B550B898178E8872E912C39
:107F8000881A910887FD9394880C991C880C991C79
:107F9000092C000CAA08BB0860E070E0CB01F7FCDC
:107FA0000AC0B701653B710514F064EB70E0072E61
:107FB000000C880B990B281939094A095B090F94A1
:107FC000547324EB30E040E050E00F948673820E4F
:107FD000931EA41EB51E740187E18715D8F0298170
:107FE00088E890E0821B910927FD9395880F991FDF
:107FF000880F991FE816F90604F502972FB7F89431
:10800000E601C00FD11FC557D94E880F991F9A831B
:1080100089832FBF62E370E080E090E0DF91CF9131
:108020001F910F91FF90EF90DF90CF90BF90AF9096
:108030009F908F907F900C94593E2A8188E592E022
:10804000821B910927FD9395880F991F880F991F0F
:10805000E816F90694F6C701D0CFDF91CF911F91B2
:108060000F91FF90EF90DF90CF90BF90AF909F90D7
:108070008F907F900895CF93DF93EB01682F70E08E
:1080800084ED96E10E94573F688179818A819B81C6
:10809000643F21E072078105910520F464EF71E0EF
:1080A00080E090E00E94593E89B183FB882780F9E7
:1080B000DF91CF910895CF93DF9300D01F92CDB77A
:1080C000DEB78EEE92E0A0E0B0E089839A83AB83C6
:1080D000BC83BE016F5F7F4F8AE50E943B400F90DB
:1080E0000F900F900F90DF91CF910895CF93DF9372
:1080F00000D01F92CDB7DEB78EEE92E0A0E0B0E0E8
:1081000089839A83AB83BC83BE016F5F7F4F8AE014
:108110000E943B400F900F900F900F90DF91CF91F6
:108120000895CF93DF9300D01F92CDB7DEB784EFD1
:1081300091E0A0E0B0E089839A83AB83BC83BE0169
:108140006F5F7F4F8CE30E943B400F900F900F902A
:108150000F90DF91CF910895CF93DF9300D01F92BE
:10816000CDB7DEB784EF91E0A0E0B0E089839A83D9
:10817000AB83BC83BE016F5F7F4F80EA0E943B40B0
:108180000F900F900F900F90DF91CF9108951F9255
:108190000F920FB60F9211240BB60F922F933F93AD
:1081A0004F935F936F937F938F939F93AF93BF93FF
:1081B000EF93FF9348EA50E064EA70E081E090E0DA
:1081C0000E94592AFF91EF91BF91AF919F918F919A
:1081D0007F916F915F914F913F912F910F900BBEC7
:1081E0000F900FBE0F901F9018951F920F920FB611
:1081F0000F9211240BB60F922F933F934F935F93DF
:108200006F937F938F939F93AF93BF93EF93FF935E
:1082100048E950E064E970E090E080E00E94592A6B
:10822000FF91EF91BF91AF919F918F917F916F914E
:108230005F914F913F912F910F900BBE0F900FBE0A
:108240000F901F9018959091C00095FFFCCF8093E0
:10825000C6000895CF93DF93EC018991882319F02C
:108260000E942341FACF8DE00E9423418AE0DF91F2
:10827000CF910C942341CF92DF92EF92FF92CF9354
:108280006B017C01C42F4A3069F4F7FE0BC0F094F7
:10829000E094D094C094C11CD11CE11CF11C8DE26F
:1082A0000E9423414C2FC701B601CF91FF90EF9060
:1082B000DF90CF900D94575CCF93DF93EC01FE01DC
:1082C00084912196882319F00E942341F8CFDF91F1
:1082D000CF9108950F931F93CF938C01C62F81E503
:1082E00095E10E945C41C8010E945C418AE30E94C2
:1082F000234180E38C0F0E9423418AE0CF911F919C
:108300000F910C94234184ED96E10E945C4160E062
:1083100084EC96E10E946A4160E08FEA96E10E9457
:108320006A4161E088EA96E10E946A4161E08DE974
:1083300096E10E946A4161E08DE896E10E946A41FF
:1083400060E084E896E10E946A4161E08AE796E194
:108350000E946A4161E080E796E10E946A4160E024
:1083600089E696E10E946A4161E081E696E10E9419
:108370006A4161E083E596E10E946A4161E085E43B
:1083800096E10E946A4160E086E396E10E946A41BC
:1083900060E088E296E10E946A4160E082E196E155
:1083A0000E946A4161E081E096E10E946A4161E0D9
:1083B00082EF95E10E946A4161E08BEE95E10E94B7
:1083C0006A4160E084EE95E10E946A4161E08BEDD4
:1083D00095E10E946A4161E086EC95E10E946A4164
:1083E00061E088EB95E10E946A4161E085EA95E1F0
:1083F0000E946A4160E088E995E10E946A4161E07B
:1084000083E995E10E946A4161E086E895E10E9476
:108410006A4160E082E795E10E946A4160E08FE591
:1084200095E10E946A4160E08EE697E10E945C243B
:10843000682F617086E595E10C946A418091500542
:10844000827149F4809152058C7829F4809153050A
:10845000837009F475C082E40E946E37882351F05E
:108460000E94042A6093EC107093ED108093EE103C
:108470009093EF1083E50E946E37882351F00E949D
:10848000443760931C1170931D1180931E119093BB
:108490001F1184E50E946E37882351F00E944437F3
:1084A00060932011709321118093221190932311D6
:1084B00088E50E946E37882351F00E94443760930C
:1084C000FD097093FE098093FF099093000A89E5E6
:1084D0000E946E37882351F00E9444376093010A4E
:1084E0007093020A8093030A9093040A8AE50E941B
:1084F0006E378823B1F00E9444376093050A709369
:10850000060A8093070A9093080A2DEC3CEC4CEC89
:108510005DE30F94206D181624F08FEF9FE00E940A
:108520005C4185E40E946E37882351F00E944437F5
:108530006093090A70930A0A80930B0A90930C0ABD
:108540000895AF92BF92CF92DF92EF920F931F9355
:10855000CF93DF935B01EA016901882309F463C0CB
:1085600085EE9FE00E945C41F5016081718182810E
:10857000938146E00E941AEFE1100BC08CED9FE062
:108580000E945C41688179818A819B8146E00E94DA
:108590001AEF85ED9FE00E945C41F60160817181D8
:1085A0008281938143E00E941AEF8EEC9FE00E944B
:1085B0005C41F801608171818281938143E00E9476
:1085C0001AEF85EC9FE00E945C41F6012081318129
:1085D00042815381F80160817181828193810F947E
:1085E000117443E00E941AEFEE20F9F08AE00E9435
:1085F000234180EB9FE00E945C41688179818A8100
:108600009B8146E00E941AEF8AE00E9423418AE0A3
:10861000DF91CF911F910F91EF90DF90CF90BF909E
:10862000AF900C942341E110E4CFDF91CF911F91E3
:108630000F91EF90DF90CF90BF90AF9008950F9380
:108640001F93CF938C01C62F88E59AE00E945C416E
:10865000C8010E945C41CC2331F08AE0CF911F9188
:108660000F910C942341CF911F910F91089560E0D9
:1086700086EB95E40E941F4388E69AE00E945C41E5
:108680008AE00C942341EF92FF920F931F93CF93B4
:108690007C018B01C42F60E086EB95E40E941F43B0
:1086A000C7010E945C4180E20E942341C8010E94F0
:1086B0005C41CC2319F08C2F0E9423418AE0CF919A
:1086C0001F910F91FF90EF900C942341DF92EF9256
:1086D000FF920F931F93CF93DF93D82E7B018A01D4
:1086E000E9010E943743D092C00840E0B7018AEC0C
:1086F00095E40E9443430115110531F040E0B801B3
:1087000083EC95E40E944343209731F040E0BE01A2
:1087100083EC95E40E94434360E086EB95E40E947D
:108720001F438EEB95E40E945C418AE0DF91CF917C
:108730001F910F91FF90EF90DF900C94234161E027
:1087400082E69AE00C941F43AF92BF92CF92DF92E1
:10875000EF92FF920F931F93CF93DF938FEA99E0ED
:108760000E945C41C0E0D7E0D15021F080E20E943D
:108770002341FACF8C2F0F94BE5CCF5FC53099F7A1
:108780008AE00E9423410DE116E0C0E080E20E94F1
:1087900023418C2F0F94BE5C5801D5E080E20E94EB
:1087A0002341F501C080D180E280F380A7019601CA
:1087B000C701B6010F940477882369F180E20E9413
:1087C00023418DE30E9423418DE30E9423418DE3E9
:1087D0000E9423418DE30E9423418DE30E942341A7
:1087E000D150F4E1AF0EB11CD111D8CF8AE00E9474
:1087F0002341CF5F0C5F1F4FC53041F68AE0DF9108
:10880000CF911F910F91FF90EF90DF90CF90BF908D
:10881000AF900C94234120E030E0A901C701B601DC
:108820000F94727687FD03C08BE20E94234143E0E0
:10883000C701B6010E941AEFD3CFCF93DF93EB01AC
:108840000E945C41CE01DF91CF910D94C55CCF9326
:10885000C62F0E945C418C2FCF910D94BE5CCF92AD
:10886000DF92EF92FF926A017B010E945C4142E03D
:10887000C701B601FF90EF90DF90CF900C941AEFF4
:108880008091510587FD2BC0809152058E7039F57E
:1088900040911011509111116091121170911311AA
:1088A0008FEE9FE00E942F444091141150911511BA
:1088B00060911611709117118CEE9FE00E942F4469
:1088C000409118115091191160911A1170911B115A
:1088D00084E092E30E942F448AE00C94234183E5D4
:1088E0000E94BC37882391F00E9444376093101196
:1088F00070931111809312119093131160931811BA
:108900007093191180931A1190931B1180E50E94A6
:10891000BC37882351F00E94443760931011709344
:108920001111809312119093131182E50E94BC37AC
:10893000882351F00E9444376093141170931511ED
:10894000809316119093171184E50E94BC378823F9
:1089500051F00E944437609318117093191180935D
:108960001A1190931B110895CF92DF92EF92FF920C
:108970006A017B010E945C414AE0C701B601FF9099
:10898000EF90DF90CF900C943B412F923F924F920B
:108990005F926F927F928F929F92AF92BF92CF928F
:1089A000DF92EF92FF920F931F93CF93DF93CDB798
:1089B000DEB7C654D1090FB6F894DEBF0FBECDBFE7
:1089C00070E060E085E40E948D39182F8F3F09F434
:1089D00083C08823E9F08CE09AE1CA5BDF4F0FB6D1
:1089E000F894DEBF0FBECDBFDF91CF911F910F91E5
:1089F000FF90EF90DF90CF90BF90AF909F908F90BF
:108A00007F906F905F904F903F902F900C945C41BF
:108A100024EB30E03A83298383E50E94BC37882326
:108A200021F00E9440379A83898365E070E083E4F7
:108A30000E948D398AA760E085E50E949C392596C1
:108A40008FAF259760E08FEF99E10E940CCAA98152
:108A5000BA81BD01BB0F880B990B0F94276D6D83F5
:108A60007E838F8327969FAF27970F943F52688B03
:108A7000798B8A8B9B8B1F3F09F045C420E030E047
:108A80004CE053E46D817E818F8127969FAD2797BF
:108A90000F94727618160CF0AAC184ED99E10E9429
:108AA0005C41CA5BDF4F0FB6F894DEBF0FBECDBF8F
:108AB000DF91CF911F910F91FF90EF90DF90CF90BA
:108AC000BF90AF909F908F907F906F905F904F90EE
:108AD0003F902F900D94574746E450E05A834983C6
:108AE0009BCF1FAEAFC12496EEADFFAD2497808320
:108AF00083C2FBEE4F2E512C612C712C04C384E1F8
:108B000090E0A0E0B0E08C8B9D8BAE8BBF8BE4E15E
:108B10004E2E512C612C712C04C34C8A5D8A6E8AB6
:108B20007F8AFFC22496EEADFFAD24978083D4C325
:108B300089819A81AB81BC8129A93AA94BA95CA9F9
:108B4000821B930BA40BB50BB7FD59C08FAD0E94D0
:108B5000BEEF8AE00E94234189819A81AB81BC816A
:108B60008053984FAF4FBF4F89AB9AABABABBCAB09
:108B70009DA9911177C02EA93FA948AD59ADB1016A
:108B8000802F26969FAD26970F94727618160CF0BC
:108B900053C020E030E040E050E4B101802F269641
:108BA0009FAD26970F9412746EAB7FAB88AF99AFD1
:108BB0002CA53DA54EA55FA589819A81AB81BC817D
:108BC000280F391F4A1F5B1F2AAF3BAF4CAF5DAF69
:108BD00020E030E040EC50E46D817E818F8127966B
:108BE0009FAD27970F9411749101402F26965FAD8A
:108BF00026970F94206D881F8827881F8DAB888942
:108C00009989AA89BB89C816D906EA06FB0610F419
:108C1000D701C60129813A814B815C81281B390B20
:108C20004A0B5B0BDA01C90181389F44A241B105AF
:108C3000A8F180E299E10EC289819A81AB81BC8161
:108C40002AAD3BAD4CAD5DAD821B930BA40BB50BB8
:108C500043EA5BE362EB7BE3B7FDD1CF812F0E9458
:108C600089F4CDCF20E030E040EF51E46D817E818A
:108C70008F8127969FAD27970F9411749B01AC01AC
:108C8000B101802F26969FAD26970F94206D87FF08
:108C9000B6CF4FE45CE36FE57CE3E0CF4AA55BA58C
:108CA000888D998D481759070CF09EC003970CF4D6
:108CB0009BC083EC98E10E945C411F3F09F076C0A5
:108CC000A3EBB8E1BA83A98382EA98E10E945C41F0
:108CD00089819A810E945C41488559856A857B8596
:108CE0008FEB98E10E942F448AE00E94234182EAA0
:108CF00098E10E945C4189819A810E945C4149A16E
:108D00005AA16BA17CA18BEB98E10E942F448AE0D1
:108D10000E94234182EA98E10E945C4189819A8104
:108D20000E945C41B501A40187EB98E10E942F44A9
:108D30008AE00E9423412596FFAD2597FF2391F1FC
:108D40002CEA35EC47E25EE369A17AA18BA19CA1F4
:108D50000F94866D6B017C012CEA35EC47E25EE3F3
:108D6000C501B4010F940C75288539854A855B854A
:108D70001F3F09F52093EC083093ED084093EE086F
:108D80005093EF08C092F008D092F108E092F208F8
:108D9000F092F3086093F4087093F5088093F60856
:108DA0009093F70881E080936A027BCEE4EFF4E4CD
:108DB000FA83E98389CF20934F163093501640935E
:108DC000511650935216C0925316D0925416E092F8
:108DD0005516F09256166093571670935816809356
:108DE000591690935A16DECF0E9447CE80C080EC71
:108DF00099E10E945C410E947CF38FE78093EB082D
:108E000024EB30E0A8EEB3E00F94B8736CA77DA715
:108E10008EA79FA7288939894A895B89260F371F22
:108E2000481F591F2AAF3BAF4CAF5DAF10926A028B
:108E300081E08093790232E0310F3EAF323008F4A6
:108E400050CE1FAFC888D988EA88FB88C9AADAAA99
:108E5000EBAAFCAA812C912C540189A29AA2ABA264
:108E6000BCA288869986AA86BB868FE790E0A0E0A0
:108E7000B0E08C8B9D8BAE8BBF8B1C8690E49A8F61
:108E8000ACE1AB8FB6E4BC8F1D8E1E8E1F8E18A278
:108E90003FE7432E512C612C712C1DAA8EAA9FAA4C
:108EA000A8AEB9AE1EA21FA218A619A6E1E0EDA3B6
:108EB000198E188E212C312C00E026961FAE269795
:108EC000F5E11F02C00111249C012A5B394E229654
:108ED0003FAF2EAF2297285F3F4F24963FAF2EAF74
:108EE00024974AA5042E000C550B5BA74AA7809136
:108EF0007902882309F4B0C00F943F5269837A83C2
:108F00008B839C835091A60658AB552309F48BC0E4
:108F10000E942FF46091E7087091E8081F3F39F034
:108F20002296AEADBFAD229714966D917C91072E1F
:108F3000000C880B990B0F94276D1B01082F2696A8
:108F40009FAF26972D8D3E8D4F8D58A126969FADB4
:108F500026970F94727618163CF42D8E3E8E0F8F46
:108F60002696BFAD2697B8A32C853A8D4B8D5C8D88
:108F7000B101802F26969FAD26970F94206D87FF15
:108F800007C02C863A8E0B8F2696EFAD2697EC8F76
:108F9000FDA19101402F26965FAD26976D817E81C0
:108FA0008F8127969FAD2797FF2309F45AC00F940E
:108FB000206D87FF38C049815A816B817C814C19B3
:108FC0005D096E097F09DB01CA0188589341A10937
:108FD000B109B7FD28C08C899D89AE89BF898419E4
:108FE0009509A609B709B595A795979587951F3F48
:108FF00009F079CD8093EB084EA35FA368A779A70A
:10900000FD81FD8F2E812E8F3F813F8F27964FADA3
:10901000279748A389819A81AB81BC81888B998BE2
:10902000AA8BBB8B1DA220E030E040EF51E46D81A4
:109030007E818F8127969FAD27970F94127491019F
:10904000402F26965FAD26970F94206D87FF70CD39
:109050008EE399E10E945C41109279020E947CF3B8
:10906000A1CE0F9472761816F4F689819A81AB819D
:10907000BC81288939894A895B89821B930BA40B9F
:10908000B50BAC01BD01485853416109710977FD29
:10909000CACF488D598D452B09F40DC1CEA0DFA054
:1090A000E8A4F9A4C80ED91EEA1EFB1E2EA13FA1FA
:1090B00048A559A5281B390B4A0B5B0BC301B2010C
:1090C0000F945473A70196010F9486734C885D88A2
:1090D0006E887F88420E531E641E751E54E145162D
:1090E0005104610471040CF40ACD8CEE481651044D
:1090F000610471040CF0FDCC90E849165104610440
:1091000071040CF40ACD4C8A5D8A6E8A7F8A2EEF38
:1091100030E040E050E0241935094609570929019B
:109120003A014C895D896E897F8988EB99E10E94BB
:10913000B444B301A20183EB99E10E94B4444C858D
:109140005A8D6B8D7C8D8CEA99E10E942F444D8D58
:109150005E8D6F8D78A185EA99E10E942F44A88DDC
:10916000B98D13970CF4A7C0C301B2010F94276DFA
:1091700020E030E040E850E40F94866D4B015C0144
:109180002C853A8D4B8D5C8D6D8D7E8D8F8D98A14C
:109190000F9411742BED3FE049E450E40F94866D79
:1091A00020E030E040E05FE30F94866D9B01AC016E
:1091B000C501B4010F940C756C877D878E879F87DE
:1091C000C701B6010F94276D2FE632E143E85AE359
:1091D0000F94866D6B017C011E3F59F02AE939E935
:1091E00049E15FE3812C912CA12C6EE3B62E1F3F49
:1091F00059F42DEC3CEC4CE45EE37BEA872E7AEAF2
:10920000972EA92C7EE3B72E6C857D858E859F8554
:109210000F94866D688779878A879B879B01AC014D
:109220000F941274A70196010F940C7569A37AA389
:109230008BA39CA3288539854A855B85C701B60128
:109240000F94866DA50194010F94866D4B015C010E
:109250004C855D856E857F858FE999E10E942F445D
:10926000B701A60189E999E10E942F448AE00E9492
:109270002341BEAD8AE899E1B23010F08BE799E165
:109280000E945C41488559856A857B8585E799E11F
:109290000E942F4449A15AA16BA17CA18FE699E1BC
:1092A0000E942F44B501A40189E699E10E942F4450
:1092B0008AE00E9423418C899D89AE89BF89840DF3
:1092C000951DA61DB71DB595A795979587951F3F29
:1092D00009F028CC8093EB08288D398D2F5F3F4F04
:1092E000398F288F3D813C874E814A8F5F815B8F0C
:1092F00027968FAD27978C8FC980DA80EB80FC8012
:1093000098A99DA390CEE12E012E000CFF08F70135
:1093100083E0EE0FFF1F8A95E1F7EF58FD4F66815E
:1093200077816F507109072E000C880B990B0F94F1
:10933000276D9B01AC016D817E818F8127969FAD4A
:1093400027970F94727618160CF4A7CB80EC99E14E
:109350000E945C410E947CF385E18E9DF0018F9D0F
:10936000F00D1124EA5BF94E8FE7808722E330E0AD
:1093700049CDCF93DF93EB010E945C41CE01DF9199
:10938000CF910D940A323F924F925F926F927F92EB
:109390008F929F92AF92BF92CF92DF92EF92FF9205
:1093A0000F931F93CF93DF938091520587FD38C0B1
:1093B000809153058370A1F5C091E316D091E41616
:1093C000488159816A817B8183E498E10E942F441E
:1093D0004C815D816E817F818AE696E40E942F44F4
:1093E0004091DF165091E0166091E1167091E216FF
:1093F00087E696E40E942F448AE0DF91CF911F9187
:109400000F91FF90EF90DF90CF90BF90AF909F9023
:109410008F907F906F905F904F903F900C9423417E
:109420006090D7167090D8168090D9169090DA1662
:10943000A090DB16B090DC160091DD161091DE16C0
:10944000C090DF16D090E016E090E116F090E216A2
:1094500088E50E94BC37C82F882309F49AC00E946F
:109460004437362E472E582ED92F20E030E046E6DE
:1094700053EC0F94727687FD0DC020E030E046E695
:1094800053E4632D742D852D9D2F0F94206D181698
:109490000CF081C066EE70E080E398E10E94B9496B
:1094A00066EE70E08BE298E10E94B94988E298E1AB
:1094B0000E945C41C0E089E50E94BC37882361F1CD
:1094C0000E944437362E472E582ED92F20E030E008
:1094D00046E653EC0F94727687FD0DC020E030E035
:1094E00046E653E4632D742D852D9D2F0F94206D3A
:1094F00018160CF055C066EE70E085E198E10E9408
:10950000B94966EE70E080E198E10E94B9498DE0CA
:1095100098E10E945C41C0E08AE50E94BC37882344
:1095200009F443C00E9444376B017C0120E030E025
:1095300040E151EC0F94727687FD0AC020E030E0E4
:1095400040E151E4C701B6010F94206D18166CF587
:1095500067EF7FEF8BEF97E10E94B94969E070E018
:1095600086EF97E10E94B94983EF97E1DF91CF91B0
:109570001F910F91FF90EF90DF90CF90BF90AF9031
:109580009F908F907F906F905F904F903F900C9442
:109590005C41C1E090CF632C742C852C9D2E8BCF29
:1095A000A32CB42C052D1D2FB7CFCC23E1F0C30184
:1095B000D4018093D7169093D816A093D916B09360
:1095C000DA16C501D8018093DB169093DC16A093C0
:1095D000DD16B093DE16C092DF16D092E016E09250
:1095E000E116F092E216DF91CF911F910F91FF905B
:1095F000EF90DF90CF90BF90AF909F908F907F9033
:109600006F905F904F903F9008952F923F924F92AE
:109610005F926F927F928F929F92AF92BF92CF9202
:10962000DF92EF92FF920F931F93CF93DF93CDB70B
:10963000DEB7CB54D1090FB6F894DEBF0FBECDBF55
:109640002DB73EB739AF28AF87E00F945F2E811159
:109650000BC061E086E50E9436388DA3853060F04E
:109660008BE89FE00E945C41A8ADB9AD0FB6F894BD
:10967000BEBF0FBEADBF40C33DA1332321F08BE67B
:109680009FE00E945C416AE080E50E943638182F16
:109690008CEF810F8F3218F087E49FE0E3CF60E01A
:1096A00085E40E949C39882309F448C081E08FAB8F
:1096B000E090E316F090E416D7012D913D914D9185
:1096C0005C916091D3097091D4098091D5099091F2
:1096D000D6090F941274AB01BC0188E50E94423890
:1096E00069877A878B879C87F7012481358146813A
:1096F00057816091D7097091D8098091D9099091CB
:10970000DA090F941274AB01BC0189E50E9442385A
:109710006D877E878F87988BBE01635F7F4FCE01F9
:1097200009960E942132382E81110BC063E683E333
:109730009FE00E940CCA8BE19FE094CF92E09FAB28
:10974000B7CF8CE40E946E37082F882309F431C10B
:109750000E94352A8EA3803118F084EF9EE082CFDC
:10976000FEA1F13009F427C160E083E50E949C3935
:109770008AAF882321F0011102C037E03EA38DA1FA
:10978000833020F08AED9EE00E945C419091E208D7
:109790009DAF80E00E946D3C0F94AE0F1D8A1E8A23
:1097A0001F8A188E198E1A8E1B8E1C8E83EF9FE4D3
:1097B000A3ECB7E48D8F9E8FAF8FB8A383EF9FE4A8
:1097C000A3ECB7EC89A39AA3ABA3BCA3A12FB0E0F1
:1097D000BCA7ABA7EDB7FEB724E0129FE019F109D3
:1097E00011240FB6F894FEBF0FBEEDBF8DB79EB724
:1097F00001969CAF8BAF2DA14FA9BE01635F7F4F38
:10980000CE0109960F94D3489B01AC010F940477C5
:10981000811162C20F943F52611571058105910556
:1098200011F00F94A668212C1BAA1CAA1DAA1EAA1F
:10983000AEA1A150BB0B2C96BFAFAEAF2C97E22DC3
:10984000F0E0F8A7EFA32BA53CA5E217F3070CF077
:1098500074C23196FEA7EDA73F932F93FF93EF932A
:1098600086EC9EE09F938F9380ED9EE09F938F9375
:109870001F920E94F1C98DB79EB709960FB6F89452
:109880009EBF0FBE8DBF9EA1992309F458C10F94AE
:1098900057682AE030E040E050E00F9486730F9460
:1098A000276D20E030E040EA50E40F9472760FEF2D
:1098B0001FEF181614F001E010E00F94576828E627
:1098C00031E040E050E00F9486730F94276D2B0138
:1098D0003C010F94576827E130E040E050E00F94DE
:1098E00086736B5F7F4F8F4F9F4F0F94276D4B0198
:1098F0005C01ADA1A430D1F4BC01A40188EB9EE0D1
:109900000E942F44B301A20180EB9EE00E942F44ED
:109910008AEA9EE00E945C410130110519F483E45B
:109920000E94234186EA9EE00E945C41312CC801DE
:10993000110FAA0BBB0B2A968CAF9DAFAEAFBFAF7A
:109940002A972C96AEADBFAD2C973A161B060CF09D
:10995000F6C02A966CAD7DAD8EAD9FAD2A970F9463
:10996000276D6B017C01BAADBB2341F1AC019B01BA
:109970000F94127420E030E040E952E40F94866DB9
:109980009B01AC01C301B2010F9412742B013C0185
:1099900020E030E044EB53E40F9472761816FCF4A8
:1099A00020E030E044EB53E4C301B2010F941174A2
:1099B000EDCF1EA2D9CE22E02EA3D6CE0F945768AB
:1099C00024E130E040E050E00F948673675E7F4F03
:1099D0008F4F9F4F0F94276DA7019601CFCF20E0A7
:1099E00030E0A901C301B2010F94206D87FF0BC0C5
:1099F00020E030E044EB53E4C301B2010F94127451
:109A00002B013C01ECCF0091E3161091E416F80114
:109A100024813581468157816D857E858F85988922
:109A20000F94117422966CAF7DAF8EAF9FAF2297CB
:109A30002BED3FE049E450E4C301B2010F94866D81
:109A400020E030E044E353E40F940C756B017C019B
:109A50000F9407756FA778AB89AB9AABD8012D919E
:109A60003D914D915C9169857A858B859C850F949C
:109A7000117426966CAF7DAF8EAF9FAF2697A50170
:109A800094016FA578A989A99AA90F94866D9B0165
:109A9000AC0126966CAD7DAD8EAD9FAD26970F9433
:109AA000127469837A838B839C83C701B6010F94F8
:109AB000B276A50194010F94866D22962CAD3DAD32
:109AC0004EAD5FAD22970F9412746D837E838F83AA
:109AD000988740EF50E070E060E0CE0101960E9470
:109AE00047F440EF50E070E060E0CE0105960E9440
:109AF00047F4BDA1B43099F449815A816B817C81CE
:109B00008AE99EE00E942F444D815E816F817885B5
:109B10008AE696E40E942F448AE00E942341198A33
:109B20001A8A1B8A1C8AAE014F5E5F4FBE016B5FB3
:109B30007F4FCE0101960F94A410339402CF20E002
:109B40004FA9BE01635F7F4FCE0109960F94D348A2
:109B50004B015C01312CAC019B010F940477811106
:109B600002C033243394A5019401C501B4010F94BC
:109B700004778111E2C0EFA1F8A5EE0FFF1FEE0FF1
:109B8000FF1F2BAD3CADE20FF31F80829182A282BA
:109B9000B382A50194016D8D7E8D8F8D98A10F9458
:109BA0007276181624F48D8E9E8EAF8EB8A2A50103
:109BB000940169A17AA18BA19CA10F94206D87FFCC
:109BC00004C089A29AA2ABA2BCA2A50194016BA970
:109BD0007CA98DA99EA90F9412746BAB7CAB8DAB45
:109BE0009EABADA5BEA5BD01BB0F880B990B0F9415
:109BF000276D6FA378A789A79AA79B01AC016BA9D2
:109C00007CA98DA99EA90F940C752B013C014D8A4E
:109C10005E8A6F8A788EEBADFCADF8ABEFA710E0F3
:109C2000C12CD12C7601AFA5B8A96D917D918D91F4
:109C30009D91B8ABAFA7A30192010F9411749B0142
:109C4000AC010F94866D9B01AC01C701B6010F9466
:109C500012746B017C011F5F211628F72FA138A514
:109C600049A55AA50F940C750F94C076698F7A8F09
:109C70008B8F9C8FBDA1B23068F18DA59EA50F94EE
:109C80000A326BA57CA585E99EE00E94B9498FE860
:109C90009EE00E945C4143E0C501B4010E941AEFBE
:109CA00080E20E94234181E0EDA1E3300CF480E0EA
:109CB000E12C8E010F5D1F4F9E01235E3F4FAE01D1
:109CC000475E5F4FBE016B5E7F4F0E94A1428AE0FC
:109CD0000E9423412394B3CD0E9418320F94950F14
:109CE0008DAD0E946D3C0F946B1988AD99AD0FB688
:109CF000F8949EBF0FBE8DBFE8ADF9AD0FB6F894D6
:109D0000FEBF0FBEEDBFC55BDF4F0FB6F894DEBFE1
:109D10000FBECDBFDF91CF911F910F91FF90EF90BC
:109D2000DF90CF90BF90AF909F908F907F906F907B
:109D30005F904F903F902F9008950E9418323320EB
:109D400069F284E89EE00E945C4181E0FDA11F165B
:109D50000CF080E0EE24E3948E010F5D1F4F9E0116
:109D6000235E3F4FAE01475E5F4FBE016B5E7F4F8C
:109D70000E94A142698D7A8D8B8D9C8D00521109B4
:109D800026E042E00F94ED679F938F9383E79EE078
:109D90009F938F938DE79EE09F938F931F920E94D6
:109DA000F1C92DB73EB7295F3F4F0FB6F8943EBFBC
:109DB0000FBE2DBF93CF2F923F924F925F926F9223
:109DC0007F928F929F92AF92BF92CF92DF92EF924B
:109DD000FF920F931F93CF93DF93CDB7DEB7CC588D
:109DE000D1090FB6F894DEBF0FBECDBF84E69DE06B
:109DF0000E945C4187E00F945F2E81118FC084E543
:109E00000E94BC37882329F00E94403781110E94AC
:109E100008EF80E090E0A0E8BFE389839A83AB83FA
:109E2000BC838D839E83AF83B8878DEC9CECACE4C0
:109E3000BEE389879A87AB87BC8780E090E0A0E289
:109E4000B1E48D879E87AF87B88B8CE390E09A8BC7
:109E5000898B8DEC90E09C8B8B8B8DEC9CECACEC2F
:109E6000BEE38D8B9E8BAF8BB88F80E090E0A0EE31
:109E7000BFE3898F9A8FAB8FBC8F1BA61CA64AE9C4
:109E800059E969E97EE38FE40E9442386D8F7E8F45
:109E90008F8F98A360E083E40E949C3989A360E0DF
:109EA0008BE40E949C398AA389E40E94BC3710E0AD
:109EB000F12CE12C8823C1F00E94352A90E018167D
:109EC000190614F481E090E011E0180F212F2150C1
:109ED000330BC90126E0289FF001299FF00D1124C2
:109EE000EC58F74FE280F38082E40E94BC3788236D
:109EF00019F00E9440377C01E114F10459F1C701C7
:109F000088978536910520F16CE870E086E39DE046
:109F10000E94B94981E39DE00E945C41C457DF4F34
:109F20000FB6F894DEBF0FBECDBFDF91CF911F916A
:109F30000F91FF90EF90DF90CF90BF90AF909F90E8
:109F40008F907F906F905F904F903F902F900895EB
:109F5000FA8AE98A8CE40E94BC378823E1F00E94E7
:109F600044376B017C01C986DA86EB86FC8620E0EB
:109F700030E0A9010F94727687FD0AC020E030E03E
:109F800040E050E4C701B6010F94206D18161CF490
:109F900089E09DE0C1CF81E50E946E37882331F1D1
:109FA0008091220590912305892BE9F00E94443786
:109FB0006B017C01CD82DE82EF82F8862DEC3CECD9
:109FC0004CE45DE30F94727687FD0AC020E030E038
:109FD00040E751E4C701B6010F94206D181634F420
:109FE00088ED9CE099CF8DEA9CE096CF83E50E94B6
:109FF000BC378823E9F00E9444376B017C01CD8A8D
:10A00000DE8AEF8AF88E2DEC3CEC4CEC5DE30F948D
:10A01000727687FD0AC020E030E040E050E4C701DE
:10A02000B6010F94206D18161CF486E89CE074CFDE
:10A0300080E50E946E37882341F08091220590913F
:10A040002305892B29F58FEF8BA786E40E94BC3767
:10A05000882309F43DC00E9444376B017C01C98EFE
:10A06000DA8EEB8EFC8E20E030E040E85FE30F9468
:10A07000727687FD0AC020E030E040E850E4C70176
:10A08000B6010F94206D18161CF585E39CE044CFB3
:10A090008BA58F5F8BA70E9444376B017C01CD8617
:10A0A000DE86EF86F88A20E030E0A9010F94727610
:10A0B00087FD0BC020E030E048EC51E4C701B60159
:10A0C0000F94206D18160CF0C0CF8EE59CE024CFC5
:10A0D000C98CDA8CEB8CFC8C8D889E88AF88B88C10
:10A0E000A7019601C701B6010F94866D9B01AC01D3
:10A0F00060E070E084E490E40F940C7529813A816B
:10A100004B815C810F94866D2B013C01A50194016C
:10A11000C501B4010F94866DA70196010F94866D59
:10A120002CEE31E548EB5DE30F940C759B01AC011F
:10A13000C301B2010F94866D69837A838B839C83FC
:10A14000112309F1412F4150550B26E0249FF001C6
:10A15000259FF00D1124EC58F74F0081118188E400
:10A160000E94BC37882319F00E9440378C010115EA
:10A17000110571F0C801855A91098F30914030F076
:10A1800087E09CE0C9CE10E000E0E9CF1C8B0B8B90
:10A1900085E50E946E378823C9F00F943F52611500
:10A1A00071058105910511F00F94A6688091220533
:10A1B00090912305892BC9F00E94443760931605BE
:10A1C0007093170580931805909319056AE170E064
:10A1D00082E50E948D39AD969FAF8EAFAD97181670
:10A1E000190644F083ED9BE097CE60E070E088E4D0
:10A1F00092E4E4CF89E50E94BC37882381F10E9474
:10A2000044372091CB093091CC094091CD09509130
:10A21000CE090F9411746B017C0188E50E94BC3754
:10A22000882331F10E9444372091C7093091C80931
:10A230004091C9095091CA090F9411746BA37CA372
:10A240008DA39EA3CFA2D8A6E9A6FAA6CE01839697
:10A250000E947924811115C089EA9BE05DCEC090EF
:10A26000D709D090D809E090D909F090DA09D5CF74
:10A270006091D3097091D4098091D5099091D60944
:10A28000DDCF84E40E946E3711E081270E946D3C8F
:10A2900080E090E0A0EAB0E48DA79EA7AFA7B8AB9E
:10A2A00060E0CE018D960F94E5108091FC08CD57AB
:10A2B000DF4F8883C358D0401092FC080E9416DC00
:10A2C00086E59BE00E945C4189899A894A970CF057
:10A2D00091C063E683E39BE00E940CCA0F9478521E
:10A2E0008B899C890E948EFA41E061E080E00E94A7
:10A2F000B6F1882309F491C00F9457470F94785210
:10A300001092DF091092E0091092E1091092E2091F
:10A310008FED99E00F94AF0C1BA5112309F4E2C057
:10A3200020E030E040E751E460910C1170910D1194
:10A3300080910E1190910F110F940C7521966CAFB6
:10A340007DAF8EAF9FAF21971F3F09F00DC581E014
:10A3500080935D0563E68BE89BE00E940CCA68E889
:10A3600073E182E090E00E94339580E1E3EDF9E053
:10A37000A8EAB8E001900D928A95E1F7CE01019626
:10A380000F94C04AC12CD12C76018091E70982FD3F
:10A390009EC068E873E182E090E00E94339520E07F
:10A3A00030E040E85EE36091B4087091B5088091B8
:10A3B000B6089091B7080F9412746093B408709324
:10A3C000B5088093B6089093B70820E030E040E8E5
:10A3D0005EE3C701B6010F9412746B017C0120E0AB
:10A3E00030E84BE354E40F94727687FD60C010921E
:10A3F0005D0513C063E686E49BE00E940CCA0F94DF
:10A40000785210935D0589899A890E94353761E0F9
:10A4100081E00E9431F081115CCF6FEF8DE99BE00C
:10A420000E940CCA8CA5811112C081E08CA78D817D
:10A430009E81AF81B885B0588DA79EA7AFA7B8AB56
:10A44000BE01635D7F4F88EA98E00E94CA3380E0D6
:10A4500090E0A0EAB0E48093B0089093B108A09394
:10A46000B208B093B3081DA61EA61FA618AABE0167
:10A47000635D7F4F88EA98E00E94CA33CD57DF4F73
:10A480005881C358D0405093FC080E9416DC1092AB
:10A490005D058AA1811142CD1092EA081092E90867
:10A4A0000E94AEDC90E080E00E948EFA37CDCE01B3
:10A4B000CD960F94DB1880E1E3EDF9E0A8EAB8E06F
:10A4C00001900D928A95E1F70E940CFB5ECF0E94ED
:10A4D00006D163E68EE79BE00E940CCA0F94785287
:10A4E00010925D05E1E1F5E085E0DF011D928A95BE
:10A4F000E9F780E1E3EDF9E0A8EAB8E001900D9218
:10A500008A95E1F789859A85AB85BC858093B008EB
:10A510009093B108A093B208B093B3081DA61EA6ED
:10A520001FA618AABE01635D7F4F88EA98E00E94CB
:10A53000CA33BE01635E7F4F88EA98E00E94CA3347
:10A5400081E080935D0589A1882309F463C420918B
:10A55000D3093091D4094091D5095091D609E59697
:10A560002CAF3DAF4EAF5FAFE5978091D70990918B
:10A57000D809A091D909B091DA09E1968CAF9DAFC5
:10A58000AEAFBFAFE197312C212C9FEFA4969FAFC8
:10A59000A497AFEFA896AFAFA897BFEFC158DF4F12
:10A5A000B883CF57D040EFE4C058DF4FE883C0589E
:10A5B000D040F3ECCF57DF4FF883C158D04027E4A9
:10A5C000CE57DF4F2883C258D04081E090E0A0E012
:10A5D000B0E0022C04C0880F991FAA1FBB1F0A9469
:10A5E000D2F7CC57DF4F88839983AA83BB83C458A3
:10A5F000D040A1E1B5E0E796BFAFAEAFE79710E07E
:10A6000000E09101032C000C440B550BC857DF4FA1
:10A61000288339834A835B83C858D040C457DF4FAF
:10A620002882CC58D040E796AEADBFADE7978D916C
:10A63000E796BFAFAEAFE79790E0B0E0A0E0CC57B1
:10A64000DF4F288139814A815B81C458D040822301
:10A650009323A423B523892B8A2B8B2B09F024C1A8
:10A66000C857DF4F688179818A819B81C858D04063
:10A670000F94276D2091890630918A0640918B06B0
:10A6800050918C060F94866D209181063091820640
:10A6900040918306509184060F941274EB966CAF30
:10A6A0007DAF8EAF9FAFEB97B801012E000C880BEA
:10A6B000990B0F94276D20918D0630918E06409155
:10A6C0008F06509190060F94866D209185063091EB
:10A6D000860640918706509188060F9412746B018C
:10A6E0007C01EB962CAD3DAD4EAD5FADEB97E596A5
:10A6F0006CAD7DAD8EAD9FADE5970F9411742B01C0
:10A700003C01A7019601E1966CAD7DAD8EAD9FAD8C
:10A71000E1970F9411744B015C01A3019201C301F5
:10A72000B2010F94866D2B013C01A5019401C50176
:10A73000B4010F94866D9B01AC01C301B2010F946B
:10A7400012740F94C0764B015C01EB962CAD3DADBD
:10A750004EAD5FADEB976BA17CA18DA19EA10F9437
:10A7600011742B013C01A70196016FA178A589A561
:10A770009AA50F9411746B017C01A3019201C3018E
:10A78000B2010F94866D2B013C01A7019601C70110
:10A79000B6010F94866D9B01AC01C301B2010F9409
:10A7A00012740F94C07620E030E040E751E40F943B
:10A7B0000C75A50194010F9412746B017C018090BB
:10A7C000160590901705A0901805B090190520E087
:10A7D00030E040E85FE3C501B4010F9472761816CB
:10A7E000F4F4C501B4010F947E754B015C0160E087
:10A7F00070E0CB01181419041A041B0434F40F94EC
:10A800005768A50194010F9486730F94276D9B01DF
:10A81000AC01B601C7010F9412746B017C01C158E1
:10A82000DF4F2881CF57D040C058DF4F3881C05804
:10A83000D040CF57DF4F4881C158D040CE57DF4F6F
:10A840005881C258D040B601C7010F94206D87FFD0
:10A850002BC0A4960FAFA497C457DF4F3881CC58B4
:10A86000D040A8963FAFA897EC96CFAEEC97ED9668
:10A87000DFAEED97EE96EFAEEE97EF96FFAEEF9769
:10A88000C158DF4FC882CF57D040C058DF4FD88261
:10A89000C058D040CF57DF4FE882C158D040CE5784
:10A8A000DF4FF882C258D0400F5F1F4F05301105AF
:10A8B00009F0B9CE4FEF241A340A55E025163104B9
:10A8C00009F083CEA4968FADA497E82FF0E0EF5E59
:10A8D000FA4F208181E090E0A0E0B0E0A8960FACB4
:10A8E000A89704C0880F991FAA1FBB1F0A94D2F70C
:10A8F000822B8083A8969FADA8976A969FAF6A9790
:10A90000A496AFADA4976B96AFAF6B97EC968FAD57
:10A91000EC97ED969FADED97EE96AFADEE97EF9677
:10A92000BFADEF976F968CAF9DAFAEAFBFAF6F97D8
:10A93000A896BFADA897BF3F09F4FAC1A496EFADA2
:10A94000A497EF3F09F4F4C16B2FBB0F770B880B73
:10A95000990B0F94276D2091890630918A064091BA
:10A960008B0650918C060F94866D20918106309154
:10A97000820640918306509184060F941274162F1C
:10A98000072F382E292E862F902FA32DB22D6596B6
:10A990008CAF9DAFAEAFBFAF6597A496FFADA49748
:10A9A0006F2FFF0F770B880B990B0F94276D20915A
:10A9B0008D0630918E0640918F06509190060F942F
:10A9C000866D2091850630918606409187065091CC
:10A9D00088060F9412746B017C016996CCAEDDAED3
:10A9E000EEAEFFAE6997CE018F5A9F4F0E94792439
:10A9F000882309F4A1C120E030E040EA50E4612F4F
:10AA0000702F832D922D0F9412744B015C01CB019A
:10AA1000D50121968CAF9DAFAEAFBFAF21972596E4
:10AA2000CCAEDDAEEEAEFFAE2597A8962FADA897C3
:10AA300021112AC2A4963FADA4973111FAC120E09A
:10AA400030E040EA50E4C701B6010F9412746B0184
:10AA50007C01A4964FADA497442309F40CC2A4969C
:10AA60008FADA49784300CF006C222ED422E23E570
:10AA7000522E2BE7622E21E4722E21968CAC9DACD7
:10AA8000AEACBFAC219725968CAD9DADAEADBFAD44
:10AA90002597A7968CAF9DAFAEAFBFAFA7979C0190
:10AAA000AD0169966CAD7DAD8EAD9FAD69970F948C
:10AAB0001174AB966CAF7DAF8EAF9FAFAB97A50116
:10AAC000940165966CAD7DAD8EAD9FAD65970F948D
:10AAD00011742D966CAF7DAF8EAF9FAF2D97AB9657
:10AAE0002CAD3DAD4EAD5FADAB9761962CAF3DAF9C
:10AAF0004EAF5FAF6197A50194016091D30970914A
:10AB0000D4098091D5099091D6090F9411744B0105
:10AB10005C01A7962CAD3DAD4EAD5FADA7976091A2
:10AB2000D7097091D8098091D9099091DA090F94C9
:10AB30001174A7966CAF7DAF8EAF9FAFA797812F93
:10AB4000902FA32DB22D8DA79EA7AFA7B8ABC9AAF2
:10AB5000DAAAEBAAFCAAC984DA84EB84FC84CDAA25
:10AB6000DEAAEFAAF8AE2DEC3CEC4CEC5CE3C301A2
:10AB7000B2010F94866D29813A814B815C810F94DB
:10AB8000866D2091DF093091E0094091E1095091F3
:10AB9000E2090F94127469AF7AAF8BAF9CAFA50135
:10ABA0009401C501B4010F94866D4B015C01A79619
:10ABB0002CAD3DAD4EAD5FADA797CA01B9010F9465
:10ABC000866D9B01AC01C501B4010F94127420E0A5
:10ABD00030E040E050E40F9472761816ACF420E0B8
:10ABE00030E040E05FE3C701B6010F94127429968C
:10ABF0006CAF7DAF8EAF9FAF2997BE01635C7F4F77
:10AC0000CE0101960E94D33389859A85AB85BC8598
:10AC100029968CAF9DAFAEAFBFAF2997A3961CAE60
:10AC20001DAE1EAE1FAEA397BE01615A7F4FCE016F
:10AC3000CD960E94CA33CE0101960F94C04AE0908F
:10AC40000411F09005110091061110910711A090C8
:10AC50000011B0900111C0900211D0900311950124
:10AC6000A601B701C8010F947276181614F4750185
:10AC700086018090850290908602A0908702B09015
:10AC800088022DEC3CEC4CEC5DE3B701C8010F945D
:10AC9000866D6093850270938602809387029093FD
:10ACA000880240E0BE01675B7F4FCE018D960F9416
:10ACB000395380E1E3EDF9E0A8EAB8E001900D92A4
:10ACC0008A95E1F78092850290928602A09287028F
:10ACD000B09288020E94142A81119FCB20E04FEF8E
:10ACE000BE01675A7F4FCE0101960E94963520E043
:10ACF00041E0BE01675A7F4FCE0101960E94963512
:10AD00002FEF40E0BE01675A7F4FCE0101960E94AF
:10AD1000963521E040E0BE01675A7F4FCE01019693
:10AD20000E9496350E940CFB0E94142A811175CB5B
:10AD30008091241180932511AD964EAD5FADAD97F6
:10AD400041505109AD965FAF4EAFAD97452B09F419
:10AD500064CB6A968FAD6A9787FD5FCB6B968FAD9C
:10AD60006B9787FFF0CB59CB63E68BE69BE00E94A5
:10AD70000CCA0F94785280E1E3EDF9E0A8EAB8E05C
:10AD800001900D928A95E1F72D853E854F85588972
:10AD90006091B4087091B5088091B6089091B70899
:10ADA0000F9412746093B4087093B5088093B6083A
:10ADB0009093B708CE01CD960F94DB182D853E8574
:10ADC0004F8558896091B4087091B5088091B60894
:10ADD0009091B7080F9411746093B4087093B508FC
:10ADE0008093B6089093B7088CA581117BCB81E046
:10ADF0008CA78D819E81AF81B885B0588DA79EA705
:10AE0000AFA7B8ABBE01635D7F4F88EA98E00E94B0
:10AE1000CA3368CB2BA13CA14DA15EA1E5962CAF16
:10AE20003DAF4EAF5FAFE5978FA198A5A9A5BAA595
:10AE3000A4CB812F902FA32DB22D21968CAF9DAF47
:10AE4000AEAFBFAF219720E030E040EA50E4C70149
:10AE5000B6010F94117425966CAF7DAF8EAF9FAF86
:10AE60002597A4965FADA49754300CF4E8CD182D27
:10AE7000092D3A2C2B2C92ED492E93E5592E9BEF60
:10AE8000692E90E4792EF9CDA8969FADA8979430BD
:10AE90000CF452C0A496AFADA497A4300CF120E0FE
:10AEA00030E040EA50E4612F702F832D922D0F94F3
:10AEB000117421966CAF7DAF8EAF9FAF219720E0CC
:10AEC00030E040EA50E4C701B6010F9411746B0101
:10AED0007C01A496EFADA497E4300CF4C6CDCBCFA3
:10AEE000812F902FA32DB22D21968CAF9DAFAEAFA9
:10AEF000BFAF219720E030E040EA50E4C701B6013F
:10AF00000F94127425966CAF7DAF8EAF9FAF2597CF
:10AF1000A496BFADA497B111D2CF20E030E040EAB3
:10AF200050E4612F702F832D922D0F941174162FE2
:10AF3000072F382E292E9FCFA496FFADA497F1118D
:10AF40000DC020E030E040E251E4B401C5010F94AF
:10AF50001174162F072F382E292E87CDA4962FADCA
:10AF6000A49724309CF020E030E040E251E4B401AA
:10AF7000C5010F94117421966CAF7DAF8EAF9FAF5A
:10AF80002197182D092D3A2C2B2C6FCD182D092D1A
:10AF90003A2C2B2C82ED482E83E5582E8BEF682E11
:10AFA00081E4782E6ACD88EA99E00C945C4182EACB
:10AFB00099E00C945C41CF92DF92EF92FF928AE588
:10AFC0000E94BC37882309F45AC00E94443720E00D
:10AFD00030E040E050EC0F94206DC12CD12CE12CDE
:10AFE00090ECF92E87FD0FC00E94443720E030E03E
:10AFF00040E050E40F94727618160CF462C00E9480
:10B0000044376B017C012091F8103091F910409188
:10B01000FA105091FB10C701B6010F94866D0F9482
:10B020007E75CB010F94F35280E50E946E3781113B
:10B030004EC0A70196016091DF167091E0168091D5
:10B04000E1169091E2160F9412746093DF167093DC
:10B05000E0168093E1169093E2160E94D757409134
:10B06000DF165091E0166091E1167091E21684EEC1
:10B0700097E10E942F448AE00E94234105C083E5A6
:10B080000E94BC378111A1CF8091520587FD24C059
:10B0900080915305837001F50E94D7574091DF16C8
:10B0A0005091E0166091E1167091E21685ED97E1FE
:10B0B0000E942F448AE0FF90EF90DF90CF900C9495
:10B0C0002341C12CD12CE12C80E4F82E9CCF0E948E
:10B0D000492A8111AECFD8CF82E50E946E37811107
:10B0E000DBCFFF90EF90DF90CF900895CF9384E572
:10B0F0000E94BC37C0E08823D9F00E94352AC82FAF
:10B100001816B4F40E94D7578DE40E942341809111
:10B110004D0590914E050F94C55C6C2FCC0F770BAD
:10B1200082EF90E10E94B9498AE00E942341CFEF6B
:10B130008C2FCF9108954F925F926F927F928F9252
:10B140009F92AF92BF92CF92DF92EF92FF92CF93F6
:10B15000DF93CDB7DEB72C970FB6F894DEBF0FBEE6
:10B16000CDBF4090C7095090C8096090C909709040
:10B17000CA0920914102309142024091430250910C
:10B180004402C301B2010F94127469837A838B83E2
:10B190009C838090CB099090CC09A090CD09B09071
:10B1A000CE092091450230914602409147025091CC
:10B1B0004802C501B4010F9412746D837E838F839E
:10B1C0009887C090CF09D090D009E090D109F09035
:10B1D000D2092091490230914A0240914B0250918C
:10B1E0004C02C701B6010F94127469877A878B8766
:10B1F0009C8720914D0230914E0240914F02509118
:10B200005002C301B2010F9412742B013C01209132
:10B210005102309152024091530250915402C501A3
:10B22000B4010F9412744B015C01209155023091CE
:10B2300056024091570250915802C701B6010F942F
:10B2400012746B017C010E94D75783E490E10E9445
:10B250005C4183E50E946E37882321F00E94492AD1
:10B2600080933F0280913F02811151C085E195E1B9
:10B270000E945C418BE390E10E945C4149815A81CC
:10B280006B817C8185E791E30E942F444D815E8133
:10B290006F8178858AE696E40E942F4449855A8515
:10B2A0006B857C8587E696E40E942F4489E390E1D4
:10B2B0000E945C4181E390E10E945C41B301A201E4
:10B2C00085E791E30E942F44B501A4018AE696E444
:10B2D0000E942F44B701A60187E696E40E942F44FE
:10B2E0008AE02C960FB6F894DEBF0FBECDBFDF917B
:10B2F000CF91FF90EF90DF90CF90BF90AF909F9055
:10B300008F907F906F905F904F900C94234189E1D4
:10B3100095E1AECF2F923F924F925F926F927F92C4
:10B320008F929F92AF92BF92CF92DF92EF92FF9255
:10B330000F931F93CF93DF93CDB7DEB76A970FB606
:10B34000F894DEBF0FBECDBF83E50E946E37182F85
:10B350003090E208882319F00E94492A382E409044
:10B36000D3095090D4096090D5097090D609809186
:10B37000D7099091D809A091D909B091DA098B8B9E
:10B380009C8BAD8BBE8B8091DB099091DC09A091E9
:10B39000DD09B091DE098F8B988FA98FBA8F1123A9
:10B3A00029F0311003C080E00E946D3C86E50E94C8
:10B3B0006E37888B20E030E0A9016091890670919A
:10B3C0008A0680918B0690918C060F94206D8823BD
:10B3D00009F4C5C083E40E946E37882309F498C03D
:10B3E0000E9444376B017C01ADE1B6E0B987A887C4
:10B3F000BF83AE83F5E0FD831D861E8628EC2F8774
:10B4000002EC1A86212C88EC8B8792E49C87AE8113
:10B41000BF81BA8BA98B15E0E989FA898190919057
:10B42000A190B190FA8BE98B2A85322D4B855C85F2
:10B43000C501B4010F94206D87FF04C08A86292CB2
:10B44000AB86BC862D853E854F85502FC501B40146
:10B450000F947276181624F48D869E86AF860B2D77
:10B460001150D1F6FD81F150FD838E819F8144966C
:10B470009F838E83F111CBCF2D853E854F85502F35
:10B480006A85722D8B859C850F94127420E030E0C4
:10B4900040E05FE30F94866DA70196010F9412744C
:10B4A0006B017C012DEB37E346E855EB0F94727688
:10B4B00087FD0AC02DEB37E346E855E3C701B60127
:10B4C0000F94206D181624F580E00E946D3C15E065
:10B4D000A884B98405E0D5016D917D918D919D91F0
:10B4E0005D014D01B4E08B1A9108A70196010F94FC
:10B4F0001174F4016083718382839383015059F73F
:10B500001150888599854496998788871111E0CFD5
:10B51000A889AA2381F020E030E0A9016091890682
:10B5200070918A0680918B0690918C060F94206D05
:10B5300081110E94A4438AE50E946E37882359F046
:10B540000E94443769837A838B839C8360E0CE01B9
:10B5500001960E94FF3C832D0E946D3C0BC0311070
:10B5600003C09889992339F30E94D75784EB9DE053
:10B570000E945C41332051F08091E208811106C0A5
:10B580000E94D35785E99DE00E945C410E94D757F5
:10B5900087E89DE00E945C418091E208811172C0C1
:10B5A00085E195E10E945C418AE00E9423410E946E
:10B5B000D7578AE79DE00E945C41C090DE08D0909A
:10B5C000DF08E090E008F090E10820E030E0A90119
:10B5D000C701B6010F94727618160CF056C042E0FF
:10B5E000C701B6010E941AEF8DE00E9423418AE054
:10B5F0000E942341A30192016091D3097091D40963
:10B600008091D5099091D6090F94206D81111FC0AA
:10B610002B893C894D895E896091D7097091D80941
:10B620008091D9099091DA090F94206D81110FC092
:10B630002F89388D498D5A8D6091DB097091DC0915
:10B640008091DD099091DE090F94206D81110F9496
:10B650006B196A960FB6F894DEBF0FBECDBFDF91AF
:10B66000CF911F910F91FF90EF90DF90CF90BF90FF
:10B67000AF909F908F907F906F905F904F903F9092
:10B680002F90089589E195E18DCF85E79DE00E9497
:10B690005C41B0CFCF93C82F82E0C11184E040E07D
:10B6A00060E00E94619B0E94D7578DE79AE0CC230F
:10B6B00011F082E99AE0CF910C945C410E947CF3F6
:10B6C0000E94DF3E80E00F947947809173088130BB
:10B6D000A1F40E94D3578BE299E00E945C4160E0A4
:10B6E00081E299E00E940CCA6EE571E080E090E092
:10B6F0000E94593E88E0809373080895CF92DF92AC
:10B70000EF92FF921F93CF93DF9300D01F92CDB79C
:10B71000DEB78EEEC82E82E0D82EE12CF12CC98245
:10B72000DA82EB82FC82BE016F5F7F4F8AE50E9466
:10B730003B4081110EC010E0812F0F900F900F90B1
:10B740000F90DF91CF911F91FF90EF90DF90CF90FE
:10B7500008950E94AC40C982DA82EB82FC82BE016D
:10B760006F5F7F4F8AE50E943B40182F882319F3B3
:10B770000E94D35785E09AE00E945C410E945E5B84
:10B78000DBCFCF92DF92EF92FF921F93CF93DF93A5
:10B7900000D01F92CDB7DEB78EEEC82E82E0D82E35
:10B7A000E12CF12CC982DA82EB82FC82BE016F5F50
:10B7B0007F4F8AE00E943B4081110EC010E0812F34
:10B7C0000F900F900F900F90DF91CF911F91FF90EE
:10B7D000EF90DF90CF9008950E94AC400E945B40B4
:10B7E0000E9476400E945B40C982DA82EB82FC8232
:10B7F000BE016F5F7F4F8AE00E943B40182F882375
:10B80000E9F20E94D35788EC99E00E945C410E94C3
:10B810005E5BD5CFFF920F931F93CF93DF93EC0125
:10B820008B01F42E0E947CF30E94D35781E099E0B3
:10B830000E945C410115110511F404EF14E42097F6
:10B8400011F4C8EFD8E00E94F9D01F930F93DF9353
:10B85000CF9388EE98E09F938F9381E08F930E941F
:10B86000F1C90E94789AC0912517C695C69580E2C5
:10B8700097E10E94172DDC2FDD0F1D2F1C0FEDB758
:10B88000FEB737960FB6F894FEBF0FBEEDBF83E04C
:10B890000E94FB2B4BED53E16C2F80E00E94C22FE6
:10B8A00010925B17D0935C1789ED98E00E94A72D4A
:10B8B00010925B1710935C178CEC98E00E94A72DF8
:10B8C00084E297E10F94325A8111E1CF61E08FEE6B
:10B8D00098E00E941F4389EE93E030E6019729F03B
:10B8E000232F2A950000E9F7F9CFF89489EE93E029
:10B8F00038EE019729F0232F2A950000E9F7F9CFB8
:10B900000E947CF3FF2041F00E948F3E0E944C2653
:10B91000909905C0A895FCCF0E944A26F7CF909B2E
:10B9200002C0A895FCCFF0E0E0E0DF91CF911F913D
:10B930000F91FF9019945F926F927F928F929F92D6
:10B94000AF92BF92CF92DF92EF92FF920F931F932D
:10B95000CF93DF931F92CDB7DEB77C0139018B0106
:10B960005B01A40EB51ED12CC12CA016B10609F4A2
:10B9700050C0F70180809180F80151908F01598269
:10B98000C4010F943E735816B9F1652DC4010F948C
:10B990004673FFEFCF1ADF0AC6018F779927892BED
:10B9A00021F162E070E080E090E00F940C52C4015D
:10B9B0000F943E7399818917F9F00E94D7578BE64F
:10B9C00096E00E945C4181E00F90DF91CF911F9142
:10B9D0000F91FF90EF90DF90CF90BF90AF909F902E
:10B9E0008F907F906F905F90089562E070E080E0AC
:10B9F00090E00E94593EDBCFBE016F5F7F4FC301D5
:10BA00000F945330F7018081918101969183808357
:10BA1000ACCF80E0D9CF80912411909125112FEFE8
:10BA20003FEF981751F0E92FF0E0EC5DFE4E2281D8
:10BA300030E09F5F9F7790932511C90108951F9271
:10BA40000F920FB60F9211240F900FBE0F901F9000
:10BA500018951F920F920FB60F9211240BB60F92EA
:10BA60002F933F934F935F936F937F938F939F9306
:10BA7000EF93FF939091C6005091251130912411BE
:10BA800041E0430F4F772091AD04213108F099C078
:10BA9000E22FF0E08827E05BF24A8F4F0D940974A3
:10BAA000615D8A5D995DA85DAF5DE15DB35DE15D5E
:10BAB000B75DBB5DE15DBF5DC35DC75DCE5DE15D53
:10BAC000D95D903229F0F8F49A3011F09D3001F5EB
:10BAD000541731F0E32FF0E0EC5DFE4E9283342FEB
:10BAE00030932411FF91EF919F918F917F916F91EE
:10BAF0005F914F913F912F910F900BBE0F900FBE12
:10BB00000F901F9018959D3481F081E09E3471F064
:10BB100080E10CC09A3338F49033D0F69032C1F201
:10BB20009D32B1F7D5CF9D3499F782E08093AD0473
:10BB3000CFCF913359F018F4903251F2E9CF88E029
:10BB40009433A1F38BE0983389F3E2CF83E0EECF17
:10BB500084E0903359F386E0913341F3D9CF85E007
:10BB60009833B1F6E3CF87E0923391F6DFCF89E0E7
:10BB7000913371F6DBCF8AE0903351F6D7CF8CE06A
:10BB8000973331F6D3CF8DE0963311F6CFCF903285
:10BB900009F49ECF8EE0933549F2BACF80ED890F3C
:10BBA0008A3008F095CF2FE02093AD048093AC0449
:10BBB0008FCF9A3019F09D3009F08ACF1092AD04E2
:10BBC00087CF9A3019F09D3009F082CF80915E17AF
:10BBD0008823A1F3273001F138F4253079F710924A
:10BBE00079021092C208EACF2A30D1F02F3031F713
:10BBF0002091AC048091C0081092C008823089F373
:10BC0000843091F08130D1F6222319F02130B1F641
:10BC100082E08093C108D2CF81E080939B06CECF93
:10BC200081E080939A06CACF6EEB71E2709331087F
:10BC300060933008C3CF8EBD0DB407FEFDCF0895CD
:10BC40008FEF8EBD0DB407FEFDCF8EB50895909198
:10BC500064009B7F90936400982F906A96959CBD9A
:10BC600080FD03C091E0863009F490E09DBD089509
:10BC7000CF93DF93EB010E945C41CE01DF91CF9126
:10BC80000C941EE5AF92BF92CF92DF92EF92FF929B
:10BC90000F931F93CF93DF93CDB7DEB7E6970FB621
:10BCA000F894DEBF0FBECDBF00915405109155052D
:10BCB000F80101900020E9F731976F01C01AD10A0D
:10BCC000F801CF01801B910B8C159D053CF48191EF
:10BCD0008F32B9F7DF0111971C92F3CF8BE1EBE8BC
:10BCE000F7E1DE015C9601900D928A95E1F7F12C67
:10BCF000E12CEC14FD040CF05DC0F801EE0DFF1D0D
:10BD00008081811103C08FEFE81AF80A5801AE0C48
:10BD1000BF1CF5018081882309F44CC0FFEFEF1AA6
:10BD2000FF0AF801EE0DFF1D7F01E01AF10A819173
:10BD30008111FACFCE014C960E94B1E98BE1FE0150
:10BD40007C96DE01119601900D928A95E1F7B5017E
:10BD5000CE0101960E94BFE1CE0101960E94D93921
:10BD60008FE20E9423418091981381113BC08CE89F
:10BD700093E00E941EE580916A1784FF1BC0198220
:10BD80001C8221E0A501BE01645E7F4FCE010196B9
:10BD90000E9484EB811129C08AE00E9423410E9405
:10BDA000D757B50182E598E10E94385ECE01019631
:10BDB0000E94D9398AE00E942341CE014C960E940C
:10BDC000D939E6960FB6F894DEBF0FBECDBFDF912E
:10BDD000CF911F910F91FF90EF90DF90CF90BF9088
:10BDE000AF90089588E993E1C4CFCE014C960E94AC
:10BDF00020E98BE1FE013196DE015C9601900D9207
:10BE00008A95E1F7CE0101960E94D93972CF2F921F
:10BE10003F924F925F926F927F928F929F92AF92DA
:10BE2000BF92CF92DF92EF92FF920F931F93CF9327
:10BE3000DF9300D000D000D01F921F92CDB7DEB7A5
:10BE4000B82E80911112843008F0D1C10F943F5266
:10BE50006B017C0180911112811108C08091241125
:10BE600090912511891B8F7709F463C681E6A82E6E
:10BE700013C08A3019F08D3009F0F6C010920C1200
:10BE80008091AA119091AB11FC01EA55FE4E1682E9
:10BE9000892BF1F40F94EC1180911112843008F089
:10BEA000ECC08091241190912511891B8F7709F4A2
:10BEB000E4C00E940B5D97FFDCCF0E94D35781EB5B
:10BEC00097E00E945C418091241180932511E4CF7A
:10BED0001092AB111092AA110CEA11E1F8018191B4
:10BEE000803209F446C08E3409F0A9C06CEA77E0CC
:10BEF000C8010F949D6C4C01892B41F06EE470E0F9
:10BF0000C80104960F946077009709F4C8014AE0CD
:10BF100050E070E060E001960F940D6A2B013C0147
:10BF20008091A6119091A711A091A811B091A9118B
:10BF30000196A11DB11D481659066A067B0629F017
:10BF400060E089E797E0892851F16AE270E0C80172
:10BF50000F948F779C01009729F1982F901B912CBB
:10BF6000992349F09150F801E90FF11D808198263D
:10BF7000F7CF8F01B3CF4AE050E070E060E0C90135
:10BF800001960F940D6A292D30E050E040E06217D1
:10BF900073078407950751F060E08AE597E00F94F6
:10BFA00055367ACF60E080E397E0F9CF4092A61152
:10BFB0005092A7116092A8117092A91180917308F4
:10BFC0008130E1F067E470E0C8010F94607700977A
:10BFD000A9F04AE050E070E060E001960F940D6A2D
:10BFE000643071058105910548F48FE896E00E9460
:10BFF0005C4160E085E896E00E940CCAC092C708E8
:10C00000D092C808E092C908F092CA088091AC1199
:10C010008B3309F441CF80911112843008F03CCF6A
:10C02000809113128A9DC00111246CEA71E18C5E2B
:10C030009D4E0F946B7780E00F940F362DCF80913B
:10C040006A1780FFBBCF67E774E4C8010F949D6C4B
:10C05000009731F0FC01838180538A3008F0AECF25
:10C0600060E086E097E09BCF2AEA31E14CEA51E1BB
:10C070006CE072E10E9408240FCF80916A1782FF62
:10C08000B6C01A82198271E6F72EE0E1EE2EF9E6CB
:10C09000DF2E80911112843008F0A9C00E94402444
:10C0A0008111A5C041E050E0BE016B5F7F4F8FEC76
:10C0B00098E10E9473E70D8110E0019711F00FEFF6
:10C0C0001FEF8091D7189091D818A091D918B091EE
:10C0D000DA188093661790936717A0936817B09348
:10C0E00069170E9440240F3F100749F4811107C0CF
:10C0F0000E94D3578FEC97E00E945C41CACF4091D9
:10C100001312242F30E00A3061F00D3051F08823F3
:10C1100009F45FC089819A81009719F001969A838A
:10C1200089831092B00489819A81F29EF001F39E76
:10C13000F00D1124EF5EFD4EE80FF91F1382892BDD
:10C1400069F50F94EC110E944024882309F4A1CFD3
:10C150000E940CFB8FEC98E10E9420E9809161170E
:10C16000882391F18150809361178D9DC001112426
:10C1700062E08355994F0E942DEDE091611724E014
:10C18000E29FF0011124E755F94F608171818281AE
:10C1900093810E943E280E9428E17BCF1A82198257
:10C1A00081E00F940F368091661790916717A091E8
:10C1B0006817B091691780930D1290930E12A09397
:10C1C0000F12B0931012BFCF0E9429E9E0927308BA
:10C1D00060CF4F9DA00111244C5E5D4E9E012F5FEC
:10C1E0003F4F60EB74E0802F0E94082452CF0F94E1
:10C1F0003F526B017C01B11004C08091A8068823D6
:10C2000051F0C092BA08D092BB08E092BC08F092FC
:10C21000BD08BB24B39480912E0590912F05A09169
:10C220003005B09131050097A105B10551F140915C
:10C23000BA085091BB086091BC087091BD08840F8A
:10C24000951FA61FB71FA7019601281B390B4A0B84
:10C250005B0BDA01C901B7FD14C00E94D35760918E
:10C26000C5087091C6088AE298E00E94385E8AE0AC
:10C270000E94234140E070E060E090E080E00E9496
:10C280000A5C80911B0290911C02A0911D02B0914A
:10C290001E02892B8A2B8B2B79F09091E8168091C6
:10C2A000E916981709F4ACC1C092BA08D092BB083D
:10C2B000E092BC08F092BD088091C1049091C20444
:10C2C0009099E0C101969093C2048093C10480913B
:10C2D000C1049091C2048E3E92406CF00E94D357EC
:10C2E00087E098E00E945C4140E070E060E090E010
:10C2F00080E00E940A5C0F943F524B015C018091E8
:10C30000C208811108C02091E8169091E91681E0D9
:10C31000291301C080E020914A1630914B1691E01C
:10C3200089272A3A31050CF480E091E04091B50468
:10C330005091B6046091B7047091B804452B462B18
:10C34000472B09F490E0981789F0882309F4A0C1DD
:10C35000D501C40180569444A24FBF4F8093B504C9
:10C360009093B604A093B704B093B8044090DF094B
:10C370005090E0096090E1097090E2092091B104C9
:10C380003091B2044091B3045091B404C301B2019E
:10C390000F94206D882319F18091B5049091B60413
:10C3A000A091B704B091B8044092B1045092B20485
:10C3B0006092B3047092B404892B8A2B8B2B09F4FE
:10C3C00049C0D501C40180569444A24FBF4F809309
:10C3D000B5049093B604A093B704B093B8048091C9
:10C3E000B5049091B604A091B704B091B804009739
:10C3F000A105B10579F1881A990AAA0ABB0AB7FC06
:10C4000029C01092B5041092B6041092B70410928D
:10C41000B80482EF97E00E945C4160E08EED97E007
:10C420000E940CCA80914C1690914D161816190650
:10C4300024F490E080E00E948EFA8091E9089091C7
:10C44000EA081816190634F41092EA081092E9085E
:10C450000E94AEDC8091BD049091BE04A091BF0407
:10C46000B091C00446015701881A990AAA0ABB0A6A
:10C47000D501C401B7FD9CC12091E8169091E91641
:10C480008091680240916902291306C19091150AB2
:10C49000899FC0011124880F892F881F990B9195BE
:10C4A0008D838091160A489FC0011124880F892F1F
:10C4B000881F990B91958E830F943F5269837A83DD
:10C4C0008B839C8340E0BE016F5F7F4FCE0105965A
:10C4D0000E9465FB6D8170E089E00F94365141E068
:10C4E000BE016F5F7F4FCE0105960E9465FB6E8196
:10C4F00070E087E00F9436518091A706882309F4F5
:10C500004AC100913B0210913C02C8010297209160
:10C510004C1630914D16281739070CF43CC1809009
:10C52000E9168F82188619861A861B868091E8166E
:10C530009F80891509F4CAC0892D90E03BE6A32E9F
:10C54000A89EF001A99EF00D1124E65DF54F4589E6
:10C5500056896789708D452B462B472B81F4418D79
:10C56000528D638D748D452B462B472B41F4458DA1
:10C57000568D678D70A1452B462B472BE1F12BE69D
:10C58000B22EB89E9001B99E300D1124A901465DCE
:10C59000554F1A01FA0161817281838194810F9450
:10C5A000C0764B015C01F10161A172A183A194A14C
:10C5B0000F94256D2B013C01F10165A176A187A1A6
:10C5C00090A50F94256D9B01AC01C301B2010F949E
:10C5D0000C75A50194010F94866D4B015C012885B3
:10C5E00039854A855B850F947276181624F48886FF
:10C5F0009986AA86BB868F818F5F8F708F8396CF37
:10C60000BB2019F01092C30457CE0F943F520091F3
:10C61000BA081091BB082091BC083091BD088090E9
:10C620001B0290901C02A0901D02B0901E02080DEB
:10C63000191D2A1D3B1D601B710B820B930B97FD6F
:10C64000E1CF8091C304811137CE81E08093C30490
:10C650005F9A8091B8088E7F8093B8088A9A8091FB
:10C66000B8088D7F8093B80880910801809581700B
:10C67000809306018091B8088B7F8093B8080E9450
:10C680004A261ACE181619060CF021CE01971BCE99
:10C6900080E090E0DC0162CE2091E9165BE6259F08
:10C6A00090011124265D354FF901EF59FF4F90811C
:10C6B000899FC0011124880F892F881F990B91959C
:10C6C0008D832E593F4FF9018081EDCE20913502A7
:10C6D0003091360240913702509138026885798551
:10C6E0008A859B850F94866D4B015C01B801012EF4
:10C6F000000C880B990B0F94276D9B01AC01C501B1
:10C70000B4010F94127469837A838B839C83409164
:10C71000390250913A02B801CE0101960E9447F4C5
:10C7200089809A80AB80BC804090B9045090BA0454
:10C730006090BB047090BC04A3019201C501B401D8
:10C740000F94206D87FF16C028E431EE4AE75FE3BF
:10C75000C301B2010F94866D20E037ED43EA5CE33C
:10C760000F941274A50194010F94866D69837A83E6
:10C770008B839C8369817A818B819C816093B904CE
:10C780007093BA048093BB049093BC040F947E759D
:10C79000CB010E948EFAF4E6CF0ED11CE11CF11CF5
:10C7A000C092BD04D092BE04E092BF04F092C004D7
:10C7B0000F94EC1180917308882309F47AC1909149
:10C7C0000901892F8095817010910802181709F4CA
:10C7D0005AC020916A17206220936A17809308023A
:10C7E00090FD10C064EF71E080E090E00E94593E3F
:10C7F0000E944BE980916A1783FDBEC1112309F4A1
:10C8000042C002C00E943AE9123008F46BC100E055
:10C810000E943D2C83E0809389020F943F526C5913
:10C820007F4F8F4F9F4F6093590570935A058093A8
:10C830005B0590935C05002331F1123021F5809166
:10C840006A1783FF20C00F94CD5D882379F081E0C3
:10C850000F94E95C42EB50E065E179E080E797E115
:10C860000E9473E780E797E10E9420E90E94C739A0
:10C87000811144C10E94B1390F94E15D81E0809340
:10C8800060170F94295E0F943F526B017C01109149
:10C890001F021123F1F08091C3088823D1F0409149
:10C8A000C4045091C5046091C6047091C704460148
:10C8B0005701841A950AA60AB70AB501A40177FDA3
:10C8C0001AC0833009F430C10CF01FC181300CF064
:10C8D00024C1212F30E0A8EEB3E00F94B873C60E48
:10C8E000D71EE81EF91EC092C404D092C504E0927F
:10C8F000C604F092C7048091DC08813009F073C04F
:10C900000F943F526B017C018091CC049091CD0437
:10C91000A091CE04B091CF04A7019601281B390B3A
:10C920004A0B5B0BDA01C901B7FD3AC0D701C6015A
:10C93000805F984DAF4FBF4F8093CC049093CD0450
:10C94000A093CE04B093CF0480901006909011066F
:10C95000A0901206B09013060F949A1FAB01BC0171
:10C9600040931006509311066093120670931306BD
:10C970008091200890912108A0912208B09123086D
:10C9800088199909AA09BB09840F951FA61FB71F0B
:10C990008093200890932108A0932208B093230845
:10C9A0008091C8049091C904A091CA04B091CB04AD
:10C9B00046015701881A990AAA0ABB0AD501C4017F
:10C9C000B7FD11C020E8C20E2EEED21E26E3E21EF5
:10C9D000F11CC092C804D092C904E092CA04F0923B
:10C9E000CB040E940BFA0F945E230E9447CE8091E5
:10C9F0002D05882379F10F943F526B017C018091C2
:10CA0000290590912A05A0912B05B0912C0546018E
:10CA10005701881A990AAA0ABB0AD501C401B7FDB1
:10CA200019C020912D0530E0A8EEB3E00F94B87343
:10CA3000C60ED71EE81EF91EC0922905D0922A05FF
:10CA4000E0922B05F0922C0580E00E94BEEF8AE078
:10CA50000E94234180912805882359F10F943F5269
:10CA60006B017C018091240590912505A0912605FC
:10CA7000B0912705A7019601281B390B4A0B5B0BC8
:10CA8000DA01C901B7FD15C02091280530E0A8EEF4
:10CA9000B3E00F94B873C60ED71EE81EF91EC092FD
:10CAA0002405D0922505E0922605F09227050E94E4
:10CAB000E6E02B960FB6F894DEBF0FBECDBFDF9138
:10CAC000CF911F910F91FF90EF90DF90CF90BF908B
:10CAD000AF909F908F907F906F905F904F903F901E
:10CAE0002F90089560E087E698E00E940CCA80913C
:10CAF000660581118CCE0E94789A89CE84E898E0F0
:10CB00009093310880933008BECE843009F0E1CE96
:10CB10000E94D7578BE898E004C00E94D7578AEB51
:10CB200098E00E945C41D5CE0E94D75783EA98E0F6
:10CB3000F8CF8091C7089091C808A091C908B0911A
:10CB4000CA08A7019601281B390B4A0B5B0BDA01B7
:10CB5000C901885E9340A109B109B7FD87C989EC75
:10CB600097E00E945C41C092C708D092C808E0924A
:10CB7000C908F092CA087AC9123028F460E085E743
:10CB800098E00E940CCA01E043CE2F923F924F9250
:10CB90005F926F927F928F929F92AF92BF92CF924D
:10CBA000DF92EF92FF920F931F93CF93DF93CDB756
:10CBB000DEB7EE970FB6F894DEBF0FBECDBF809103
:10CBC000E208888B87E50E946E37882309F41FC12D
:10CBD00020E030E0A9016091890670918A06809179
:10CBE0008B0690918C060F94206D811108C00E94D5
:10CBF000D35781E69EE00E945C4110E01BC18AE5AC
:10CC00000E94BC37882339F10E9444372091CF0914
:10CC10003091D0094091D1095091D2090F941174EB
:10CC20006B017C0120E030E040E251ECC701B6012D
:10CC30000F94727687FD0AC020E030E040E251E4B4
:10CC4000C701B6010F94206D181674F40E94D357D3
:10CC500084E59EE0D0CFC090DB09D090DC09E09065
:10CC6000DD09F090DE09DECF40E050E060EC7FE7C8
:10CC700088E50E9442382091C7093091C809409147
:10CC8000C9095091CA090F9411742B013C0140E06D
:10CC900050E060EC7FE789E50E9442382091CB09A3
:10CCA0003091CC094091CD095091CE090F94117467
:10CCB0004B015C016FEF89E40E943638182F6FEF4B
:10CCC0008AE40E943638082FA3019201C301B20101
:10CCD0000F94047781116EC0A5019401C501B401C0
:10CCE0000F940477811166C08BA19CA1ADA1BEA158
:10CCF0008BAB9CABADABBEAB209181063091820675
:10CD00004091830650918406C301B2010F941174BF
:10CD10002B013C0120E030E040E05FE36BA97CA9FF
:10CD20008DA99EA90F94866D9B01AC01C301B20130
:10CD30000F9412742BA93CA94DA95EA90F940C75F0
:10CD40000F947E75162F4FA058A469A47AA4209141
:10CD50008506309186064091870650918806C50168
:10CD6000B4010F9411744B015C0120E030E040E00D
:10CD70005FE3C301B2010F94866D9B01AC01C50155
:10CD8000B4010F941274A30192010F940C750F94C7
:10CD90007E75062F812F012E000C990B97FD2FC059
:10CDA00005977CF5802F002E000C990B97FD2BC06A
:10CDB00005975CF5153008F020CF053008F01DCF41
:10CDC00080E00E946D3C95E01902F0011124E00F13
:10CDD000F11D07FDFA95EE0FFF1FEE0FFF1FE35E3B
:10CDE000F94FC082D182E282F38288890E946D3C31
:10CDF0008889882309F401CF0F946B19FECE10E0C7
:10CE0000D1CF14E0CFCF00E0D5CF04E0D3CF8AE478
:10CE10000E946E37182F811127C070E060E086E510
:10CE20000E948D399A838983059708F18FE29EE0ED
:10CE30000E945C41812FEE960FB6F894DEBF0FBEC4
:10CE4000CDBFDF91CF911F910F91FF90EF90DF90B9
:10CE5000CF90BF90AF909F908F907F906F905F909A
:10CE60004F903F902F9008950E94BB3CC6CE60E04B
:10CE700084E40E949C398F8740E050E0BA018AE543
:10CE80000E9442386BA77CA78DA79EA740E050E880
:10CE90006BE376E483E50E94423820E030E040E72F
:10CEA00052E40F940C7560937D0270937E02809320
:10CEB0007F0290938002E090E316F090E416D70191
:10CEC0008D909D90AD90BC9020E030E0A901C5010F
:10CED000B4010F9412746BAF7CAF8DAF9EAF20E0A6
:10CEE00030E040E450E40F94206D87FF06C01BAE95
:10CEF0001CAEB0E4BDAFE0E4EEAF20E030E040E7D0
:10CF000053E4C501B4010F9412746BAB672E8FAB61
:10CF100098AF20E030E043E653E40F9472761816A1
:10CF200034F41BAA612CF3E6FFAB23E428AFD7014E
:10CF300014968D909D90AD90BC90179720E030E0B6
:10CF4000A901C501B4010F941274D62EE72EF82E54
:10CF5000092F20E030E040E951E40F94206D87FF75
:10CF600005C0D12CE12CF0E9FF2E01E420E030E0F7
:10CF700040E753E4C501B4010F941274B62EC72ED6
:10CF800089AF9AAF20E030E044E553E40F94727625
:10CF9000181634F4B12CC12CB4E5B9AFE3E4EAAF10
:10CFA00088E40E946E37882309F415C20E94443732
:10CFB0000F947E751B0177FF02C06F5F7F4F7595E1
:10CFC00067957195619571096D587F4F072E000C1B
:10CFD000880B990B0F94276D762E872E982EA92EED
:10CFE0002D2D3E2D4F2D502F0F94727618161CF4B8
:10CFF000D72C74010A2D2BAD3CAD4DAD5EAD672D28
:10D00000782D892D9A2D0F947276181624F07BAC0A
:10D010008CAC9DACAEAC872D982DA92DBA2D8B8BE9
:10D020009C8BAD8BBE8B8D2D9E2DAF2DB02F8F8BFE
:10D03000988FA98FBA8FB101330C880B990B0F947D
:10D04000276D1B012C01AC019B016D2D7E2D8F2DB9
:10D05000902F0F941274D62EE72EF82E092F2B2D19
:10D060003C2D49AD5AAD0F94206D87FF04C0BD2CF7
:10D07000CE2CF9AE0AAFA2019101672D782D892D32
:10D080009A2D0F941274D62EE72EF82E092F2BA965
:10D09000362D4FA958AD0F94206D87FF04C0DBAA31
:10D0A0006E2CFFAA08AF8BA9962DAFA9B8AD8B8FB8
:10D0B0009C8FAD8FBE8F8B2D9C2DA9ADBAAD8F8F60
:10D0C00098A3A9A3BAA3BE01695E7F4FCE01439680
:10D0D0000E942132882309F4AFC1BE01615E7F4FF7
:10D0E000CE014B960E942132E82E882309F4A4C178
:10D0F0002F89388D498D5A8D6F8D78A189A19AA17C
:10D100000F94117420E030E040E85EE30F94866DE8
:10D110004B015C012B893C894D895E896B8D7C8D2F
:10D120008D8D9E8D0F94117420E030E040E85EE319
:10D130000F94866D6BA37CA38DA39EA38FA298A64C
:10D14000A9A6BAA689819A811816190674F48DEFDA
:10D150009DE00E945C418F85882321F083EF9DE054
:10D160000E945C418AE00E9423410E940CFB0F94C4
:10D17000AE0F80E00E946D3C80E090E0A0E2B1E460
:10D180008FA798ABA9ABBAAB60E0CE018F960F9496
:10D19000E5102091890630918A0640918B065091C6
:10D1A0008C066BA17CA18DA19EA10F94206D811195
:10D1B00030C020918D0630918E0640918F0650919F
:10D1C00090066FA178A589A59AA50F94206D81116D
:10D1D00020C02091810630918206409183065091B3
:10D1E00084066B897C898D899E890F94206D8111BD
:10D1F00010C0209185063091860640918706509197
:10D2000088066F89788D898D9A8D0F94206D88237B
:10D21000A9F00E94BB3C88E0FE01B396A9E8B6E005
:10D2200001900D928A95E1F788E0FE017396A1E8DE
:10D23000B6E001900D928A95E1F7188A60E085E4E6
:10D240000E949C3988248394811102C062E0862E5A
:10D250001B861C861D861E861A8A9E2C43ECC42EB5
:10D260004DE0D42E51EDA52E5DE0B52E1A89153076
:10D270000CF0ECC06B857C858D859E859B01AC0197
:10D280000F9404778111E2C03324339435E0232EC8
:10D29000911005C033243A9422242A9484E091E02A
:10D2A0009926F12EFF0CFF0CF10EF394898B19894E
:10D2B0006A89121509F4C6C0062E000C770B880B7C
:10D2C000990B0F94276D2FA138A549A55AA50F9446
:10D2D000866D2F89388D498D5A8D0F9412742B01CC
:10D2E0003C01612F110F770B880B990B0F94276D61
:10D2F0002BA13CA14DA15EA10F94866D2B893C8989
:10D300004D895E890F9412746B837C838D839E8319
:10D310004F82588669867A8689819A81892B79F02D
:10D320006F2D8FED9DE00E94274469E170E08DED47
:10D330009DE00E94B9498AED9DE00E945C411F92E8
:10D34000F9E1FF931F92FF92DF92CF92BF92AF92CB
:10D350001F920E94F1C92981482DBE01695F7F4F4C
:10D36000CE0103960F94D3482B013C014B865C867B
:10D370006D867E860FB6F894DEBF0FBECDBFAC01C2
:10D380009B010F94047781115AC009898A8925E08D
:10D39000020380011124080F111D87FD1A95000F4B
:10D3A000111F000F111F035E194FA30192016BA5FE
:10D3B0007CA58DA59EA50F941274D8016D937D93C5
:10D3C0008D939C931397188A81E00E94075FF394D2
:10D3D0008989830D6BCF4D2D5E2D6F2D702F86E4C7
:10D3E0000E9442381B012C014BAD5CAD6DAD7EAD92
:10D3F0008CE40E9442386B8B7C8B8D8B9E8B2F8AAA
:10D40000388E498E5A8E4B2D5C2D69AD7AAD82E4F3
:10D410000E9442386B017C014BA9562D6FA978AD53
:10D4200082E50E9442386B8F7C8F8D8F9E8FCF8ECE
:10D43000D8A2E9A2FAA247CE83E19EE0F9CC88897E
:10D440000E946D3C8A898F5F8A8B10CF0F9457475B
:10D450000E941832882359F088890E946D3C80E030
:10D4600090E0A0ECBFE78B879C87AD87BE876B857C
:10D470007C858D859E859B01AC010F94047781117D
:10D4800059C08F85811126C082E0F82E02E094E019
:10D49000C92E12E0DC2CD11A21E041E0612F802F4F
:10D4A0000E94BA2421E04FEF612F8F2D0E94BA24F1
:10D4B0002FEF41E06D2D802F0E94BA242FEF4FEF08
:10D4C0006D2D8F2D0E94BA24115020F70150F39436
:10D4D0000F3FF9F60E94A4430E94DF3D8F85811122
:10D4E00024C08BED99E00E9452334B015C0183ED27
:10D4F00099E00E94803A9B01AC01C501B4010F94F0
:10D50000866D9B01AC016091DB097091DC09809113
:10D51000DD099091DE090F9411746093DB0970931B
:10D52000DC098093DD099093DE098F858111E888FD
:10D53000E092E2080F94950F8091E20881110F9418
:10D54000EA110E94EA290F946B196B857C858D8501
:10D550009E8511E09B01AC010F94047781116ACC88
:10D560004CCBCF93DF93C82FD62F8091DB1083FD58
:10D5700014C08091270A811110C080918E02909171
:10D580008F02AC014150510920914C1630914D163B
:10D590002417350714F40E948EFA40E06D2F8BE0BB
:10D5A0000E94619BCC2339F040E061E080E0DF9194
:10D5B000CF910C94B6F18091270A91E0892780934E
:10D5C000790280917902882389F080914A1690919E
:10D5D0004B1620914C1630914D16821B930B97FFE2
:10D5E00003C0919581959109029744F410927902B4
:10D5F0008091DB1083FF06C0C1E01AC080E00E946A
:10D60000075FDFCFC091270AC11112C080918E023F
:10D6100090918F02019720914C1630914D1628174A
:10D62000390754F70E94D7578CE69AE00E945C4174
:10D630008C2FDF91CF910895AF92BF92CF92DF925E
:10D64000EF92FF920F931F93CF93DF93CDB7DEB787
:10D6500064970FB6F894DEBF0FBECDBF0E94765818
:10D66000D82E87FDB5C08AE50E94BC37882309F40F
:10D67000C0C040E050E0BA018AE50E9442387B0118
:10D680008C014D2D63E085E00E94619B2091DB09B8
:10D690003091DC094091DD095091DE0960E070E0D5
:10D6A0008AE793E40F9411745B016C019701A80160
:10D6B0000F947276181614F07501860120E030E0A0
:10D6C000A901B701C8010F947276181624F4E12C51
:10D6D000F12C00E010E0B701C8010F947E75072E11
:10D6E000000C880B990B0F94276D6D837E838F83BD
:10D6F000988720E030E0A9010F94206D882321F065
:10D70000CE0105960E948C2880E090E0A0EAB1E46A
:10D7100089879A87AB87BC871D861E861F86188AD5
:10D720008CE40E946E37882309F468C00E94443755
:10D730006B017C0120E030E0A901C701B6010F9424
:10D74000727687FF04C0F7FAF094F7F8F094C98A6C
:10D75000DA8AEB8AFC8A20914C1630914D162430DF
:10D76000310574F080914A1690914B16821B930BF1
:10D7700097FF03C091958195910901E004970CF4FE
:10D7800000E063E080E00E94B16A811140C083E064
:10D7900080933002109265050E94789A6D817E8197
:10D7A0008F8198858B019C01305809831A832B83C4
:10D7B0003C8320E030E0A9010F94206D882321F004
:10D7C000CE0101960E948C28109265050E94789ADD
:10D7D00064960FB6F894DEBF0FBECDBFDF91CF9138
:10D7E0001F910F91FF90EF90DF90CF90BF90AF907F
:10D7F0000895E12CF12C00E211E443CFC09018060B
:10D80000D0901906E0901A06F0901B0693CF83E0A3
:10D81000E82E22E0AE01475F5F4FBE016F5E7F4F93
:10D82000CE010D960F94BF47B9CF6F927F928F9222
:10D830009F92AF92BF92CF92DF92EF92FF920F939F
:10D840001F93CF93DF9300D000D01F921F92CDB7CC
:10D85000DEB75C014B013A01F22E68010091A0068F
:10D8600010929C0610929D0610929E0610929F06A2
:10D870001092A0060F944B5280914C1690914D1629
:10D880008C159D051CF4C6010E948EFA60E080E0B4
:10D890000E94B16A811122C1109265050E94789A96
:10D8A0001C141D0444F4C6010E948EFA40E060E09E
:10D8B00080E00E94B6F140E060E088E00E94619B59
:10D8C00060E081E00E94B16A80E090E0A0E7B2E40D
:10D8D00089839A83AB83BC8380E090E0A0E8B0ECBE
:10D8E0008D839E83AF83B887BE016F5F7F4FCE016C
:10D8F00005960F94351187E00F94C70E811158C01B
:10D900008091DB099091DC09A091DD09B091DE09DD
:10D910004091050550910605609107057091080535
:10D92000C0900105D0900205E0900305F090040539
:10D93000C092A808D092A908E092AA08F092AB0879
:10D940004093AC085093AD086093AE087093AF0855
:10D950008093B0089093B108A093B208B093B30835
:10D9600080E090E0A8E4B2E489839A83AB83BC832F
:10D97000CE0101960F94DB188091090590910A055C
:10D98000A0910B05B0910C058093B0089093B1085D
:10D99000A093B208B093B30880E090E0A0EAB0E4AE
:10D9A00089839A83AB83BC83CE0101960F94DB18E5
:10D9B000C12CD12C80E7E82E82E4F82EC982DA82CD
:10D9C000EB82FC8280E090E0A0E8B0E48D839E834F
:10D9D000AF83B887BE016F5F7F4FCE0105960F946E
:10D9E000351120E030E0A90160910D0570910E0520
:10D9F00080910F05909110050F94206D87FF0BC04B
:10DA0000C982DA82EB82FC82BE016F5F7F4F8DE0BC
:10DA100095E00F94351180910D0590910E05A09120
:10DA20000F05B09110058093DF099093E009A09352
:10DA3000E109B093E2098093B4089093B508A093EC
:10DA4000B608B093B70884EB98E00F94AF0C8091C0
:10DA50001C0681110F94135D109265050E94789A3F
:10DA600061E085E19BE00E941F438091A806815000
:10DA70008093A8064FE751E26DE17BE085E00F94CB
:10DA8000CA488091A806882339F00E9428E1809135
:10DA9000A80681508093A80680E00F947947809172
:10DAA000DC08823011F40F945C200F9457470E94D9
:10DAB000789A28960FB6F894DEBF0FBECDBFDF91DF
:10DAC000CF911F910F91FF90EF90DF90CF90BF907B
:10DAD000AF909F908F907F906F900895E12C2F2DA5
:10DAE000A301B401C5010F94BF47DACE4F925F92F4
:10DAF0006F927F92AF92BF92CF92DF92EF92FF929E
:10DB00001F93CF93DF9300D000D01F921F92CDB709
:10DB1000DEB75C01E62EF42E642F80E00E94B16A2D
:10DB2000182F81111BC0EE2021F0109265050E9474
:10DB3000789A812F28960FB6F894DEBF0FBECDBF1E
:10DB4000DF91CF911F91FF90EF90DF90CF90BF902A
:10DB5000AF907F906F905F904F900895EE2029F0E6
:10DB600040E06F2D83E00E94619B80E090E0A0E7A1
:10DB7000B2E48D839E83AF83B88780E090E0A0E815
:10DB8000B0EC89839A83AB83BC83BE016B5F7F4F0C
:10DB9000CE0101960F94351168E873E180E090E0C2
:10DBA0000E94593EC12CD12C88ECE82E81E4F82E3D
:10DBB000CD82DE82EF82F88680E090E0A0E8B0E4DB
:10DBC00089839A83AB83BC83BE016B5F7F4FCE0199
:10DBD00001960F94351140901411509015116090DA
:10DBE000161170901711C0921411D0921511E09275
:10DBF0001611F092171180E090E0A0E2B2E48D835C
:10DC00009E83AF83B887F50180819181A281B38122
:10DC100089839A83AB83BC83BE016B5F7F4FCE0148
:10DC200001960F9435114092141150921511609283
:10DC3000161170921711129A64E670E080E090E07D
:10DC40000E94593E76CF8F929F92AF92BF92CF9211
:10DC5000DF92EF92FF921F93CF93DF9300D000D01B
:10DC60001F921F92CDB7DEB70E947658182F87FDFE
:10DC7000ADC08AE50E94BC37812C912C90E2A92E80
:10DC800091E4B92E882341F040E050E0BA018AE5E2
:10DC90000E9442384B015C01412F64E083E00E9406
:10DCA000619B20E030E0A901C501B4010F947276B8
:10DCB00018167CF580E090E0A0EAB0E48D839E83A6
:10DCC000AF83B8872091DB093091DC094091DD09F1
:10DCD0005091DE09C501B4010F9412746B017C01EF
:10DCE00020E030E04AE753E40F94206D87FD06C042
:10DCF000C12CD12C8AE7E82E83E4F82EC982DA827F
:10DD0000EB82FC82BE016B5F7F4FCE0101960F94C8
:10DD1000C61085E50E946E37882309F469C00E9409
:10DD200044376B017C0120E030E0A901C701B60156
:10DD30000F94727687FF04C0F7FAF094F7F8F09426
:10DD4000F7FAF094F7F8F094C982DA82EB82FC8259
:10DD500044E061E0CE0101960E94766D20E030E063
:10DD6000A901C501B4010F94727618165CF580E024
:10DD700090E0A0EAB0E48D839E83AF83B887A501CD
:10DD800094016091DB097091DC098091DD0990912B
:10DD9000DE090F9411746B017C0120E030E0A901D1
:10DDA0000F94727618161CF0C12CD12C7601C98202
:10DDB000DA82EB82FC82BE016B5F7F4FCE0101965F
:10DDC0000F94C610109265050E94789A28960FB697
:10DDD000F894DEBF0FBECDBFDF91CF911F91FF90B2
:10DDE000EF90DF90CF90BF90AF909F908F9008956D
:10DDF00088E01802F0011124EC5EF94FC080D18058
:10DE0000E280F38090CFBF92CF92DF92EF92FF92A9
:10DE10000F931F93CF93DF9300D01F92CDB7DEB740
:10DE20007C016B018A01B22E61E088E09BE00E94D8
:10DE30001F434FE751E26FE07BE085E00F94CA4853
:10DE40009091A80681E0890F8093A80680916A17B7
:10DE500082FF06C08B7F80936A179E5F9093A8060F
:10DE60000F94942080E1E3EDF9E0A1E0B5E00190AA
:10DE70000D928A95E1F70E940CFB81E00F9479479F
:10DE800020E030E0A901F7016081718182819381F6
:10DE90000F94206D8823F1F08091270A81110CC026
:10DEA00080918E0290918F02019720914A163091B5
:10DEB0004B162817390774F080E090E0A0E7B2E431
:10DEC00089839A83AB83BC83BE016F5F7F4FC70199
:10DED0000F94351187E00F94C70E811103C0B6016E
:10DEE0000F94B22220E030E0A901F8016081718135
:10DEF000828193810F94206D882329F042E06B2D5D
:10DF0000C8010E94766D129A64E670E080E090E0AD
:10DF10000E94593E81E00F900F900F900F90DF917B
:10DF2000CF911F910F91FF90EF90DF90CF90BF9016
:10DF30000895CF92DF92EF92FF92CF93DF936B0120
:10DF40007C01D42FC091C30883E08093C30881E093
:10DF50008093C208C114D104E104F10431F00F949C
:10DF60003F52C60ED71EE81EF91E8091C2088823B4
:10DF700089F0C114D104E104F10421F48D2F0E9431
:10DF8000075FF3CF0F943F526C197D098E099F09EB
:10DF900097FDF4CF1092C208C093C308DF91CF91D0
:10DFA000FF90EF90DF90CF9008951F93CF93DF9372
:10DFB000D82FC62F0E944A5B61E08C2F0E94DF3968
:10DFC0000F943F52685370458F4F9F4F60939C064C
:10DFD00070939D0680939E0690939F061092A006D4
:10DFE0001091C30883E08093C30830E020E041EE45
:10DFF00055E46AEF7AE082E00E94664381E0809314
:10E00000C2088091C208882309F463C060E08C2FA5
:10E010000E94DF398091A006882309F456C040E0B1
:10E0200060E08AE00E94619B0E94D75780EE9AE0F0
:10E030000E945C4130E020E04AEC5AE061ED7AE079
:10E0400082E00E94664341E060E070E0CB010E9404
:10E05000996F30E020E050E040E06DEB7AE085E041
:10E060000E94664310929C0610929D0610929E0696
:10E0700010929F061092A0060F944B5260E080E031
:10E080000E94B16A8D2F0E944A5B0F943F526853E1
:10E0900070458F4F9F4F60939C0670939D068093B1
:10E0A0009E0690939F061092A00630E020E041EE7D
:10E0B00055E461EB7AE082E00E94664381E0809360
:10E0C000C20861E08C2F0E94DF3981E00E94075F67
:10E0D00098CF1093C308DF91CF911F910895CF92ED
:10E0E000DF92EF92FF920F931F93CF93DF93CDB701
:10E0F000DEB7A0970FB6F894DEBF0FBECDBF0E946B
:10E10000765887FDD1C0482F61E081E00E94619B75
:10E1100085E40E946E37882309F4D5C00E944437F5
:10E120006B017C0120E030E0A9010F94727687FF3B
:10E1300004C0F7FAF094F7F8F094F7FAF094F7F8CF
:10E14000F094C98ADA8AEB8AFC8A8CE0E0EAF2E091
:10E15000DE01119601900D928A95E1F78AE50E9401
:10E16000BC37882351F040E050E0BA018AE50E94B4
:10E17000423869877A878B879C8788E50E94BC37FD
:10E18000882351F040E050E0BA0188E50E9442380F
:10E1900069837A838B839C8389E50E94BC378823BB
:10E1A00051F040E050E0BA0189E50E9442386D83A9
:10E1B0007E838F83988785E50E946E37882309F4D4
:10E1C00089C00E9444376B017C0120E030E0A90146
:10E1D000C701B6010F94727687FF04C0F7FAF09476
:10E1E000F7F8F094F7FAF094F7F8F094CD8ADE8A15
:10E1F000EF8AF88E198E1A8E1B8E1C8E8CE40E946C
:10E200006E37882309F46FC00E9444376B017C018C
:10E2100020E030E0A901C701B6010F94727687FFB4
:10E2200004C0F7FAF094F7F8F094CD8EDE8EEF8EFE
:10E23000F8A262E070E082E40E948D39F82E8091AD
:10E24000A806811131C021E0AE014B5E5F4FBE01D7
:10E250006F5F7F4FCE0141960E94036F882321F1AB
:10E260006F2D81E00E94D56F82E50E94BC37882324
:10E2700009F442C00E94403740E050E060EA71E497
:10E280004D875E876F87788B2091A806222361F0E7
:10E290008C012F2DAE01435F5F4FBE01635E7F4F48
:10E2A000CE0149960E94156CA0960FB6F894DEBF79
:10E2B0000FBECDBFDF91CF911F910F91FF90EF90D7
:10E2C000DF90CF900895C12CD12C80E8E82E80E417
:10E2D000F82E33CFC0901406D0901506E0901606A5
:10E2E000F090170672CFC0901806D0901906E090F3
:10E2F0001A06F0901B068CCF90E080E0BDCFCF9245
:10E30000DF92EF92FF920F931F93CF93DF93CDB7DE
:10E31000DEB76C970FB6F894DEBF0FBECDBF8CE4AE
:10E320000E946E37882309F4C3C00E9444376B01F2
:10E330007C0120E030E0A9010F94727687FF04C0D1
:10E34000F7FAF094F7F8F094F7FAF094F7F8F094FD
:10E35000C98EDA8EEB8EFC8E8CE0E0EAF2E0DE0114
:10E36000119601900D928A95E1F788E50E94BC37DD
:10E370008823A1F040E050E0BA0188E50E944238CD
:10E380002091C7093091C8094091C9095091CA0923
:10E390000F94117469837A838B839C8389E50E942F
:10E3A000BC378823A1F040E050E0BA0189E50E9423
:10E3B00042382091C7093091C8094091C90950914C
:10E3C000CA090F9411746D837E838F8398878AE5C1
:10E3D0000E94BC37882351F040E050E0BA018AE542
:10E3E0000E94423869877A878B879C87F0906A17EA
:10E3F000F2FAFF24F0F840E061E080E00E94619BC7
:10E4000060E080E50E949C39E82E1D861E861F86EE
:10E41000188A8091A80681113CC02E2DAE01435F61
:10E420005F4FBE016F5F7F4FCE0149960E94036F21
:10E43000882379F180911C0681110F94135DFF20D0
:10E4400011F0EE2031F160E080E00E94D56F898DFF
:10E450009A8DAB8DBC8DB0588D8B9E8BAF8BB88F4A
:10E46000198A1A8A1B8A1C8A1D861E861F86188A8C
:10E470008091A806882369F010E000E020E0AE015A
:10E480004B5E5F4FBE016F5E7F4FCE010D960E94C7
:10E49000156C6C960FB6F894DEBF0FBECDBFDF9142
:10E4A000CF911F910F91FF90EF90DF90CF90089543
:10E4B000C12CD12C80E8E82E80E4F82E45CF2F9295
:10E4C0003F924F925F926F927F928F929F92AF9204
:10E4D000BF92CF92DF92EF92FF920F931F93CF9351
:10E4E000DF93CDB7DEB7E5970FB6F894DEBF0FBE6A
:10E4F000CDBF8DAB2091C3082CAB81E08093C308C6
:10E5000080914F058D3409F4C5C4843511F40C9401
:10E510008C86873409F091C180914D0590914E050C
:10E520008B31910509F4D9C108F079C18430910586
:10E5300008F030C1209173088230910508F48EC133
:10E54000213009F091C111E0029709F010E00E941A
:10E55000593819821A821B821C821D821E821F82D8
:10E56000188682E50E94BC37882309F48CC10E947A
:10E5700044376B017C0120E030E0A9010F94206D4D
:10E58000882309F4EAC04090D3095090D4096090E0
:10E59000D5097090D6098091D7099091D809A0919A
:10E5A000D909B091DA098CA79DA7AEA7BFA7809023
:10E5B000A8089090A908A090AA08B090AB088091F4
:10E5C000AC089091AD08A091AE08B091AF0888ABAF
:10E5D00099ABAAABBBABA5019401C301B2010F94E7
:10E5E000206D81110DC028A939A94AA95BA96CA584
:10E5F0007DA58EA59FA50F94206D882309F4ADC03D
:10E60000A3019201C501B4010F94117420E030E020
:10E6100040E05FE30F94866D68A779A78AA79BA760
:10E620002CA53DA54EA55FA568A979A98AA99BA996
:10E630000F94117420E030E040E05FE30F94866DAA
:10E640002B013C0120E030E0A901C701B6010F9485
:10E65000206D881F8827881F181709F40BC180E0D8
:10E6600090E0A0E8BFEB8CA79DA7AEA7BFA728A509
:10E6700039A54AA55BA5CA01B9010F94866D4B0166
:10E680005C01A3019201C301B2010F94866D9B014D
:10E69000AC01C501B4010F9412740F94C0764B0104
:10E6A0005C01AC019B01C701B6010F94117468AB0A
:10E6B00079AB8AAB9BABA5019401C701B6010F945E
:10E6C00012749B01AC0168A979A98AA99BA90F942E
:10E6D000866D6B017C0120E030E0A9010F94727619
:10E6E00087FDCDC0C701B6010F94C0766B017C01D8
:10E6F000C301B2019058A50194010F940C752CA58B
:10E700003DA54EA55FA50F94866DA70196010F94B8
:10E71000866D28A539A54AA55BA50F941274698357
:10E720007A838B839C83A501940168A579A58AA52A
:10E730009BA50F940C752CA53DA54EA55FA50F9428
:10E74000866DA70196010F94866DA30192010F9427
:10E7500012746D837E838F83988720E030E0A90157
:10E7600069817A818B819C810F94206D81119FC07A
:10E7700020E030E0A9016D817E818F8198850F9422
:10E78000206D811194C00E94D35785E091E10E94D1
:10E790005C416AC08531910509F466C08A319105F2
:10E7A00009F498C0049709F048C080E50E94BC377E
:10E7B000C12CD12C7601882321F00E94042A6B0100
:10E7C0007C0183E50E94BC37882361F00E944437B6
:10E7D00020E030E04AE754E40F94866D0F9485758D
:10E7E0006B017C010E940CFB8091DB13811105C041
:10E7F00060E08BE191E10E940CCA0F943F52C60E7B
:10E80000D71EE81EF91E0F943F526C197D098E0920
:10E810009F0997FF29C080E00E94075FF4CF8A32EA
:10E82000910509F4ACC160F48D31910509F4D4C0AF
:10E8300008F46CC04E9709F428C10F94B14714C076
:10E840008B35910509F47EC28C35910509F47EC2A1
:10E850008A35910591F71092DD0806C0213021F428
:10E860000E9459380F942816FDA9F111ABC40F94DA
:10E87000A052A8C480E090E0A0E8BFE3F4CEC12C91
:10E88000D12C760135CF89E40E94BC37882331F042
:10E890000E94443769837A838B839C838AE40E9435
:10E8A000BC37882309F459CF0E94443752CF412FF7
:10E8B000BE016F5F7F4F88EA98E00F9439530F9441
:10E8C0003F526093BA087093BB088093BC08909342
:10E8D000BD08CACF0E94DB4EC7CF87E00F945F2EE2
:10E8E0008111C2CF8CE0ECEAF2E0DE0111960190DA
:10E8F0000D928A95E1F770E060E080E50E94C937EB
:10E90000BE016F5F7F4F0F94B222AECF87E00F94AE
:10E91000C70E811106C060E08FE40E949C3981110E
:10E92000A3CF0E940CFB109240026091E2088CE49D
:10E930000E949C39E82E80E00E946D3C0F943F526B
:10E940006093BA087093BB088093BC089093BD088D
:10E950000F94AE0F81E080932D080F94931A8AE5EF
:10E960000E946E37F82E882369F081E00F94C70E5D
:10E97000182F82E00F94C70E11110C943E8811E0FD
:10E98000811101C010E088E50E946E37082F8111C7
:10E990000C94A18611110C94B1860C94A486012FBD
:10E9A000182F0C94B18660E070E080E890E40C943D
:10E9B000BA86A3019201C501B4010C94078760E0F7
:10E9C00086E391E10E940CCA0E94D75784E291E14C
:10E9D0000E945C410C94DF8714E00F943F526093D7
:10E9E000BA087093BB088093BC089093BD088091CF
:10E9F000E208811127C08EE40E946E37882321F03F
:10EA000087E491E10E94708887E00F945F2E811166
:10EA10001FC00E94C5658823D9F0115001F130E074
:10EA200020E04FE751E262E771E185E00E94664332
:10EA300061E085E691E10E941F438DE491E10E942F
:10EA40007088CBCF60E08FE40E949C39882399F2D4
:10EA50000E94374380E192E10E94708805CF61E017
:10EA600083E092E10E941F438EE891E10E9470884A
:10EA700061E08AE691E20E941F4340E070E060E0BE
:10EA80008FE791E10E940A5CEFCE0091E3161091AE
:10EA9000E416D8012D913D914D915C916091D3097F
:10EAA0007091D4098091D5099091D6090F94127470
:10EAB000AB01BC0188E50E94423869837A838B836D
:10EAC0009C83F80124813581468157816091D70963
:10EAD0007091D8098091D9099091DA090F94127434
:10EAE000AB01BC0189E50E9442386D837E838F8330
:10EAF0009887BE016B5F7F4FCE0101960E94213245
:10EB0000882309F4B1CE80E00E946D3C0F94AE0FD3
:10EB100061E085E40E949C39182F21E0482FBE0156
:10EB20006B5F7F4FCE0101960F94D3486B017C0140
:10EB3000AC019B010F940477811119C049815A815E
:10EB40006B817C8182E392E10E942F444D815E8142
:10EB50006F8178858DE292E10E942F44B701A60172
:10EB600088E292E10E942F448AE00E9423410F94A0
:10EB7000950F11110E94EA290F946B1975CE80919F
:10EB80007308813009F070CE89E40E94BC37082FE9
:10EB9000F12C882319F00E944037F82E8AE40E9455
:10EBA000BC37E82E882379F00E944037182F0023C5
:10EBB00009F4C0C0F4E0FF1508F0B9C08AE392E19F
:10EBC0000E945C4151CE10E00111F4CF80E1E3EDF1
:10EBD000F9E0A8EAB8E001900D928A95E1F70023E8
:10EBE00019F16F2DFF0C770B880B990B0F94276D84
:10EBF0002091890630918A0640918B0650918C06AF
:10EC00000F94866D20918106309182064091830693
:10EC1000509184060F9412746093A8087093A90809
:10EC20008093AA089093AB08EE2019F1612F110F81
:10EC3000770B880B990B0F94276D20918D063091DF
:10EC40008E0640918F06509190060F94866D20910C
:10EC500085063091860640918706509188060F946C
:10EC600012746093AC087093AD088093AE089093D3
:10EC7000AF0860E080E50E949C398823C1F1002341
:10EC8000D1F0E091E316F091E416208131814281C8
:10EC900053816091A8087091A9088091AA08909169
:10ECA000AB080F9411746093A8087093A90880931F
:10ECB000AA089093AB08EE20D1F0E091E316F09112
:10ECC000E41624813581468157816091AC087091AA
:10ECD000AD088091AE089091AF080F9411746093C5
:10ECE000AC087093AD088093AE089093AF0840E0F5
:10ECF00050E0BA0186E40E9442386B017C0120E0BA
:10ED000030E0A9010F9472761816C4F420E030E0C8
:10ED100040E752E4C701B6010F940C7569837A830A
:10ED20008B839C83CE0101960F94DB189DCDEE2042
:10ED300009F44CCF153008F449CF40CF60E070E0C3
:10ED4000CB01ECCF8FE08093DD088ECD80914C0518
:10ED5000882381F1893009F087CD68EBA62E62E027
:10ED6000B62E73EDC72E79E0D72EE12C00E010E02F
:10ED7000D5018D915D010E94BC37F82E882361F08A
:10ED8000133011F4082FFE2C0E944437F6016083E3
:10ED9000718382839383EF2C1F5FF4E0CF0ED11C2D
:10EDA000143031F7EE2009F457C00F94EA110F9494
:10EDB0006B195ACD58EBC52E52E0D52EF12CE12C13
:10EDC00000E010E0D6018D916D010E94BC37382E15
:10EDD0008823D9F10E9444374B015C01133059F06C
:10EDE000F701E953F64F20813181428153810F941D
:10EDF00011744B015C01F701ED52F64F2081318116
:10EE000042815381C501B4010F9411742B013C015F
:10EE10002DEB37E346E855EB0F94727687FD0AC079
:10EE20002DEB37E346E855E3C301B2010F94206DA3
:10EE300018165CF41330C1F48092DF099092E00957
:10EE4000A092E109B092E209032D1F5FB4E0EB0E3E
:10EE5000F11C143009F0B6CF002309F4A8CF8FEDD0
:10EE600099E00F94AF0CA3CFF701E350F74F5F0188
:10EE7000A301920160817181828193810F94127448
:10EE8000D5016D937D938D939C931397812F0F9450
:10EE9000A70EDBCF80914D0590914E058D379105E2
:10EEA00009F4FCC508F058C28E34910509F49BC6DC
:10EEB00008F021C18B31910509F4F4C508F0B1C007
:10EEC0008531910509F46BC508F07AC0813191054F
:10EED00009F424C508F044C0029708F0AECC80E5E0
:10EEE0000E94BC37C12CD12C7601882321F00E94CE
:10EEF000042A6B017C0183E50E94BC37882361F002
:10EF00000E94443720E030E04AE754E40F94866DD5
:10EF10000F9485756B017C010E940CFB8091540558
:10EF200090915505009709F4F3C40F942D35809105
:10EF30004D0590914E056BE572E1892B11F463E567
:10EF400072E130E020E041EE55E482E00E94664349
:10EF500040E0C701B6010E94996F0F94574784CCD7
:10EF60008231910511F40C944380449709F065CCEB
:10EF700080916A1783FF0BC58EE892E10E945C4185
:10EF800080916A1783FF17C08BE897E10E94B1E96F
:10EF90008BE1EBE8F7E1DE01119601900D928A9585
:10EFA000E1F770E060E0CE0101960E9421EECE0113
:10EFB00001960E94D9398FE792E10E945C4154CCBE
:10EFC0008831910509F400C5B0F48631910509F442
:10EFD000EAC4479709F031CC8091540590915505CA
:10EFE000FC012191222309F4E8C42032D1F7DF018A
:10EFF00011971C92F6CF8931910509F44FC54A97B4
:10F0000009F01BCC80916A1783FF2ECC83E50E9408
:10F01000BC37882309F428CC0E94252A0E943E2868
:10F0200023CC8132910509F4AFC508F03EC08E3182
:10F03000910509F499C568F48C31910509F48CC5E2
:10F040004D9709F0FACB80916A178E7F80936A17EB
:10F050000BCC8F31910509F49BC5809709F0EDCB5E
:10F0600080916A1782FD0E940CFB80916A1783FFD2
:10F07000FBCB60E080E50E949C39182F682F8091BF
:10F080005405909155050E942DED83E50E94BC37F3
:10F09000882321F00E94252A0E943E280E9428E110
:10F0A0001111E2CB0E94CC3EDFCB8B34910509F4E9
:10F0B00092C5B0F48033910509F489C5893491056E
:10F0C00009F0BBCB80E50E946E37882309F4CCCBD6
:10F0D0000E94352A853608F084E680935E05C4CB0D
:10F0E0008C34910509F47BC58D34910509F0A5CBCD
:10F0F0000E94DF3EB9CB8D36910509F435C608F084
:10F1000086C08C35910509F4C2C708F03FC083352D
:10F11000910509F4B0C778F48135910509F48EC7DB
:10F120008235910509F089CB8091DD088F7D806162
:10F130008093DD0899CB8435910509F4A4C7853502
:10F14000910509F07ACB83E50E946E37882309F494
:10F150008BCB0F943F526093BA087093BB08809397
:10F16000BC089093BD080E94443720E030E04AE795
:10F1700054E40F94866D0F94857560932E057093FB
:10F180002F0580933005909331056ECB8A3691051B
:10F1900009F448C698F58836910509F4B6C589364C
:10F1A000910509F04ACB0E947658182F87FD0AC0B6
:10F1B0008CE593E10E945C41812F0E94BEEF8AE0C2
:10F1C0000E9423412CA92093C308E5960FB6F8941A
:10F1D000DEBF0FBECDBFDF91CF911F910F91FF908A
:10F1E000EF90DF90CF90BF90AF909F908F907F90E7
:10F1F0006F905F904F903F902F9008958B369105C0
:10F2000009F44BC68C36910509F42ECB16CB833707
:10F21000910509F4DDC708F05DC08037910509F458
:10F2200023CB08F048C08E36910509F445C68F36C9
:10F23000910509F002CB83E50E946E37882331F0F7
:10F2400060E083E50E9436388093DB100E94D75738
:10F250008DE693E10E945C418091DB10882309F4E4
:10F260003EC610E000E020E08091DB1090E0B0E0CE
:10F27000A0E0002E04C0B695A795979587950A94AF
:10F28000D2F780FF12C0FF24F394F20E222319F06C
:10F290008CE20E942341F801EE0FFF1FED59FC4E56
:10F2A000859194910E945C412F2D0F5F1F4F053077
:10F2B0001105D1F61EC48137910509F413C68237B2
:10F2C000910509F0BACA0F94B7468AEF96E10E94F9
:10F2D00049F6CACA8737910509F4A8C770F585377A
:10F2E000910509F479C78637910509F0A6CA0091FE
:10F2F00054051091550594E0F12C40E0915009F42B
:10F3000084C7F8018081282F2B7F213409F076C72C
:10F310002181213309F079C7813409F484C7853408
:10F3200009F441E098012E5F3F4F89012F5F3F4F65
:10F33000F80180818032C9F3E1CF8837910509F463
:10F3400079C78937910509F078CA10922D08109273
:10F350002C080F94931A88CA8239E1E09E0711F4B1
:10F360000C94AA8408F0EBC08C3D910511F40C9428
:10F37000308208F072C0893C910509F4D0C708F0CA
:10F3800051C08B39910509F432C6B8F48C38910517
:10F3900009F4C7C58139910509F04FCA70E060E0F2
:10F3A00083E50E948D39823008F44DC70E94D357FF
:10F3B0008DEA93E10E945C4157CA8E3B910509F4A6
:10F3C000D7C5883C910509F038CA0E947658182F95
:10F3D00087FD4ACA0091FC0884E40E94BC37F82EDD
:10F3E0008823B9F00E9444374B015C0120E030E0F3
:10F3F000A9010F94206D882309F48FC724E012021D
:10F40000F0011124E850F74F80829182A282B382EA
:10F410000F2D602F83E50E949C398093FC080E9489
:10F4200016DC22CA8D3C910509F4C6C758F48B3C02
:10F43000910509F49EC78C3C910509F0FEC90E9414
:10F44000404412CA8E3C910509F4BAC7833D910528
:10F4500009F0F3C90E949B5807CA8D3221E0920738
:10F4600011F40C946A8308F044C08831A1E09A0733
:10F4700011F40C94CA82F0F48D3D910511F40C94B2
:10F4800073828A3F910509F0D8C983E40E946E37E0
:10F49000882321F00E9440370E940C2C6091590271
:10F4A00070915A028DE294E10E94B9498AE00E946B
:10F4B0002341DAC98232E1E09E0711F40C9466839D
:10F4C0008C32914009F0B9C964E071E083E50E9493
:10F4D000C9378C0168EE73E080E50E94C93789382E
:10F4E00023E1920710F088E893E1B8010E94339578
:10F4F000BBC9803321E0920711F40C94EC8368F4CB
:10F500008E32A1E09A0711F40C9460848F329140FE
:10F5100009F093C90E94C544A7C98039E1E09E075C
:10F5200011F40C94A6848139914009F086C9809128
:10F53000B90881113CCC81E00F943E1C38CC8C3052
:10F5400022E0920711F40C94C48508F0FDC0863EB9
:10F55000A1E09A0711F40C94408508F0C6C0843AE3
:10F56000E1E09E0711F40C94B284B8F48A3921E0EA
:10F57000920709F479C98D39914009F05EC983E594
:10F580000E946E37882311F40C9472860E94492AD7
:10F5900080931C060E94B93967C9853AA1E09A0791
:10F5A00011F40C94B6848C3A914009F046C987E076
:10F5B0000F945F2E811158C969E2C62E6DE2D62ED6
:10F5C000E3EDF9E0F9A7E8A79E012F5F3F4F19018E
:10F5D000790110E000E0C6010E941232A8A5B9A589
:10F5E0008D909D90AD90BD90B9A7A8A7A50194015D
:10F5F0000F9411742B013C01F70140825182628209
:10F60000738220E030E040EA51EC0F94727687FD7F
:10F610000AC020E030E040EA51E4C301B2010F9497
:10F62000206D181684F4F801E35BF24DE4911E1688
:10F6300054F4B7FAB094B7F8B094D7018D929D9274
:10F64000AD92BC921397F70181909190A190B190E7
:10F650007F0120E030E040EA51ECC501B4010F9495
:10F66000727687FF02C00C942B8520E030E040EAE0
:10F6700051E4C501B4010F94206D181614F40C94D4
:10F680002B850F5F1F4FF4E0CF0ED11C0330110507
:10F6900009F0A1CF59E0E52E59E0F52E10E0F10177
:10F6A00081919191A191B1911F01F7018193919362
:10F6B000A193B1937F01812F0F94A70E1F5F133089
:10F6C00071F70F946B1960E084EA94E10E940CCA10
:10F6D00063E972E084E690E00E9433956AEB72E0A1
:10F6E00084E690E00E943395BFC8863FE1E09E0724
:10F6F00011F40C94B68568F4843F21E0920711F46C
:10F700000C94B285853F914009F097C80F94492E1B
:10F71000ABC8873FA1E09A0711F40C94BA85883FE3
:10F72000914009F08AC881E0809391060F943D2EA4
:10F7300010929106882309F497C80E94D75780EE4B
:10F7400094E10E945C4190C88C36E3E09E0709F486
:10F750008BC808F08DC08D3B22E0920711F40C9409
:10F76000EF8508F076C08835A2E09A0711F40C9472
:10F77000D5858B35924009F060C80E947658082FD5
:10F7800087FD72C885E50E946E37882369F10E9463
:10F7900044374B015C01E02E002E000CFF0820E0F6
:10F7A00030E0A9010F94727687FF04C0B7FAB094D5
:10F7B000B7F8B09420E030E84BE354E4C501B4015D
:10F7C0000F947276970143E0220F331F4A95E1F7B9
:10F7D0002C5E394F181614F40C94D985D9018D92EA
:10F7E0009D92AD92BC9213978CE40E946E37882351
:10F7F00009F43AC80E9444376B017C01002E000CCA
:10F80000110B20E030E0A9010F94727687FF04C04D
:10F81000F7FAF094F7F8F09420E030E84BE354E482
:10F82000C701B6010F947276980193E0220F331F3F
:10F830009A95E1F72C5E394F181614F40C94E48570
:10F84000D9011496CD92DD92ED92FC9217970C940B
:10F8500034748E3BE2E09E0711F40C94F3858335FB
:10F86000934011F00C941D740E94C3490C9434749D
:10F87000873E23E0920711F40C946286C8F4843822
:10F88000A3E09A0711F40C94F785803A934011F0A5
:10F890000C941D74209154053091550590916A1770
:10F8A000926090936A17C9010E94E4EC0C9434743E
:10F8B000883EE3E09E0711F40C948886893E9340CD
:10F8C00011F00C941D740F94295E81110C94347402
:10F8D0000E94B1390F94E15D0F949A1F6D33710549
:10F8E0008105910520F08DE495E10E94708889E4FE
:10F8F00095E10E94708884EE80935E0585E395E132
:10F900000E945C4181E395E10E9470880C943474FC
:10F9100060E083E692E10E940CCA09CB8091500519
:10F9200084FD17C08091520587FD13C08091530557
:10F93000837079F460E086E792E10E940CCA5F98D8
:10F940008A988091080181708093060112980C9426
:10F95000347488E50E946E3781115F9889E50E94B2
:10F960006E3781118A988AE50E946E37882329F0C4
:10F970008091080181708093060185E40E946E37B2
:10F98000882311F40C94347412980C9434740E94EB
:10F99000D7578FE992E10E945C410C9434740E9425
:10F9A0004BE90C94347480916A1782FF02C00C9466
:10F9B00034740E943AE90C94347460E00E942DED96
:10F9C00010925E050C94347483E50E94BC37882342
:10F9D00021F00E94252A0E943E2884E50E94BC371F
:10F9E0008823A9F00E94252A6B017C010F944120F5
:10F9F000C0920C06D0920D06E0920E06F0920F0611
:10FA0000CD28CE28CF2819F081E08093DC088091A2
:10FA1000A8068823F9F080E090E0A0EAB1E48983A9
:10FA20009A83AB83BC831C8E1D8E1E8E1F8E18A2E4
:10FA300019A21AA21BA210E000E020E0AE014F5F65
:10FA40005F4FBE01645E7F4FCE0180960E94156CB1
:10FA50000C9434740E94A83E882381F00E9428E10F
:10FA60000E94CC3E83E599E00E94D9E810920D12E5
:10FA700010920E1210920F121092101261E087EB8A
:10FA800091E20E941F434FE751E269EA72E185E08B
:10FA90000F94CA480F9457470C9434740E947F7196
:10FAA0000C94347483E40E946E37882361F18FEBE9
:10FAB00092E10E945C418091D2188823F9F0BE0146
:10FAC0006F5F7F4F8FEC98E10E946CE8CE0101964A
:10FAD0000E941EE5CE0101960F94FB5D8091981364
:10FAE000882339F080E20E94234188E993E10E9453
:10FAF0001EE58AE00E9423410C94347485EB92E168
:10FB00000E945C41F6CF83E50E94BC37882301F157
:10FB10000E94352A182F8C3308F08CE38093280537
:10FB20000F943F526B017C01212F30E0A8EEB3E02F
:10FB30000F94B873C60ED71EE81EF91EC092240596
:10FB4000D0922505E0922605F09227050C94347496
:10FB50000E94E6E00C943474809154059091550510
:10FB60000E94E4EC0C94347480916A1783FD02C007
:10FB70000C9434740F9497478091540590915505D7
:10FB80000E947CEC0C9434740E94425E0C94347499
:10FB90000F949A1F6C8F7D8F8E8F9F8FBE016F5F2A
:10FBA0007F4FCE014C960E94C92FCE0101960F9433
:10FBB0002D350E94D757BE016F5F7F4F8EEC92E1CB
:10FBC0000E94385E8AE00E9423410C9434740E94A3
:10FBD000054B0C9434740E94CC3E0C9434740F94F6
:10FBE00094200C94347470E060E083E50E948D39B9
:10FBF0008E34910531F40E942DFA0F9457470C94DE
:10FC0000347489E393E10E945C4160911C08709117
:10FC10001D0880E393E10E941D4460911E087091CD
:10FC20001F0883E293E10E941D4460911C087091BB
:10FC30001D0880911E0890911F08681B790B809108
:10FC4000DC08815021E030E0823010F030E020E02C
:10FC5000621B730B88E193E10E941D448AE00E94BD
:10FC6000234180E193E10E945C41809120089091C2
:10FC70002108A0912208B09123088C8F9D8FAE8F10
:10FC8000BF8FBE016F5F7F4FCE014C960E94C92F80
:10FC9000BE016F5F7F4F83E093E10E94385E8091E9
:10FCA000240890912508A0912608B09127088C8FF0
:10FCB0009D8FAE8FBF8FBE016F5F7F4FCE014C9681
:10FCC0000E94C92FBE016F5F7F4F83EF92E10E94B8
:10FCD000385E20E030E04AE754E4609128087091F3
:10FCE000290880912A0890912B080F940C75AB017C
:10FCF000BC018BED92E10E942F448DE60E942341CE
:10FD00008AE00E9423410C9434748091DB1083FFBD
:10FD100002C00C9434740E94765887FF02C00C9481
:10FD2000347489E40E94BC37882311F40C94F18761
:10FD30000E94352A90E01816190614F481E090E02C
:10FD400026E0289FF001299FF00D1124EC58F74F71
:10FD5000808191810E948EFA61E080E00F94A6601C
:10FD60000F94BF600C9434748091DB1083FF02C049
:10FD70000C9434740E947658F82E87FF02C00C94BD
:10FD8000347489E40E94BC37882311F40C94FC87F6
:10FD90000E94352A90E01816190614F481E090E0CC
:10FDA00026E0289FF001299FF00D1124EC58F74F11
:10FDB0008081918110E00E948EFA61E081E00F94D1
:10FDC000A66020914C1630914D1680914A16909164
:10FDD0004B1682179307F4F48CE493E19F938F936F
:10FDE00087E593E19F938F931F920E94F1C90F9033
:10FDF0000F900F900F900F9001E00F94BF600023C1
:10FE000011F40C94347440E0612F8F2D0E94B6F1F0
:10FE10000C94347481E493E1112301F3012FEDCFAD
:10FE200010E0EBCF60E080E50E943638F82E31E03C
:10FE3000381710F40C94347481E40E946E3760918A
:10FE4000150A062F10E0811102C00FEF10E089E4BF
:10FE50000E94BC37882311F40C940E880E94352A26
:10FE600090E01816190614F481E090E026E0289F2F
:10FE7000F001299FF00D1124EC58F74F04811581F2
:10FE8000EF2DF0E0EB5EF54F0F3F110519F010F08C
:10FE90000FEF10E000830C94347460E080E50E9462
:10FEA0003638823010F00C943474E82FF0E0EB5EBA
:10FEB000F54F10820C9434748EE40E94BC37882372
:10FEC00011F40C9434740E94252A6093A611709347
:10FED000A7118093A8119093A9110C9434748FE505
:10FEE00093E10ECE83E50E94BC37882369F00E941F
:10FEF000352A8D3320F480931F020C9434748CE3E4
:10FF000080931F020C9434740E94D75760911F0293
:10FF100084E793E10E9427448AE00E9423410C94E5
:10FF200034748091DB1083FF02C00C94347489E434
:10FF30000E94BC37882311F40C941A880E94352A39
:10FF400090E01816190614F481E090E026E0289F4E
:10FF5000F001299FF00D1124EC58F74F8281938115
:10FF60000E94353761E080E00F94A6600C943474F1
:10FF70008091DB1083FF02C00C94347489E40E94EA
:10FF8000BC37882311F40C9425880E94352A90E010
:10FF90001816190614F481E090E026E0289FF0017D
:10FFA000299FF00D1124EC58F74F8281938110E0C6
:10FFB0000E94353760E081E00F94A6602091E90847
:10FFC0003091EA088091E7089091E808821793073A
:10FFD0001CF48AE893E102C08BE793E160E00E94A1
:10FFE0000CCA60E0812F0E9431F00C94347483E5D8
:10FFF0000E94BC37882311F40C9434740E94352A73
:020000021000EC
:10000000182F8C3308F08CE380932D050F943F520A
:100010006B017C01212F30E0A8EEB3E00F94B873A0
:10002000C60ED71EE81EF91EC0922905D0922A05D9
:10003000E0922B05F0922C050C9434740E947CF312
:100040000E941DFB0E94DF3E0E94E23E1092CE08FD
:100050001092CD081092CC0868EE73E080E090E03A
:100060000E94593E0E944C2660E089E993E10E947B
:100070000CCA0C9434748091DD088F7E806280936A
:10008000DD080C9434740E94D7370C9434740E94A9
:10009000765887FF02C00C9434748091500584FD1B
:1000A00009C08091520587FD05C08091530583707A
:1000B00009F489C028EBC22E22E0D22E3CEDE32EBB
:1000C00030E1F32E10E0D6018D916D010E94BC3716
:1000D000882309F465C0133009F06DC00E944437CD
:1000E0004B015C0120E030E040EA51E40F94206DC8
:1000F00087FF4EC0A50194016091FC107091FD1026
:100100008091FE109091FF100F940C752B013C0113
:10011000AC019B016091090A70910A0A80910B0A57
:1001200090910C0A0F94866D6093090A70930A0AE5
:1001300080930B0A90930C0AA301920160910C1119
:1001400070910D1180910E1190910F110F94866D89
:1001500060930C1170930D1180930E1190930F11F9
:100160006091F5097091F6098091F7099091F8096D
:100170000F94256DA30192010F94866D0F948575E0
:100180006093F5097093F6098093F7099093F80945
:100190008092FC109092FD10A092FE10B092FF1081
:1001A0001F5FF4E0EF0EF11C143009F08CCF0E94B9
:1001B000E8FA0C9434740E944437F701648B758B11
:1001C000868B978BEDCF81E00F941C470C94347491
:1001D0000E9483410C94347480915405909155058C
:1001E000009741F0DC012C91222321F00F942D3552
:1001F0000C9434740F9457470C943474803529F45C
:10020000818180538A3008F48DC841110E94D757EC
:10021000FF2021F08AEA93E10E945C41C8010E941C
:100220002A410C943474FF24F3947CC80F944F1A21
:100230000C94347481E080932D0880932C080F94E3
:10024000931A0C9434748C01112788E40E94BC37F3
:100250008823C1F00E9440378A3A91050CF44BC0C4
:100260000E944037843B91400CF048C00E944037C8
:1002700026E0209FF001219FF00D1124EC58F74F4C
:100280009183808382E40E94BC378823A9F00E9476
:1002900040370597B4F10E9440378D389105A4F599
:1002A0000E94403726E0209FF001219FF00D11248D
:1002B000EC58F74F9383828386E40E94BC378823EF
:1002C00011F40C9434740E94403797FD20C00E94B2
:1002D00040378F3F910509F0ECF40E94403726E04B
:1002E000209FF001219FF00D1124EC58F74F9583CA
:1002F00084830C9434748AEA90E0BACF83EB91E063
:10030000B7CF85E090E0CECF8CE890E0CBCF90E007
:1003100080E0E5CF8FEF90E0E2CF80E07EC80E94E2
:10032000765887FF02C00C94347408EB12E08CED11
:10033000E82E80E1F82E9CEBC92E92E0D92ED80150
:100340008D918D010E946E37882359F00E944437A9
:100350000F948575F70160837183828393830E9474
:100360009AFAF4E0EF0EF11CC016D10641F70C9496
:1003700034740E94765887FF02C00C94347418EBD2
:10038000E12E12E0F12E10E000E0D7018D917D0109
:100390000E946E37882349F00E944437F801E452E6
:1003A000FF4E64A375A386A397A30C5F1F4F003174
:1003B000110559F70C9434740E941E420C94347445
:1003C000B9E0EB2EB9E0FB2E10E088E5810F0E942A
:1003D0006E37882351F00E944437F70160837183A0
:1003E00082839383812F0F94A70E1F5FF4E0EF0E9B
:1003F000F11C133051F78091520587FF02C00C9415
:10040000D77680915305837011F00C94D776409184
:10041000090950910A0960910B0970910C098FEC40
:1004200093E10E942F4440910D0950910E09609173
:100430000F09709110098AE696E40E942F444091BA
:10044000110950911209609113097091140987E6FE
:1004500096E40E942F448AE00E9423410C94347455
:1004600082E40E946E37882341F080917B02909154
:100470007C02909321028093200282E50E946E37D5
:10048000882341F0809120029091210290937C0278
:1004900080937B0283E50E94BC37882331F00E9461
:1004A000403790937C0280937B028091500590911D
:1004B0005105A0915205B0915305892B8A2B8B2BA6
:1004C00011F00C94347460917B0270917C0286ED83
:1004D00093E10E94B94985E20E9423418AE00E948B
:1004E00023410C9434740E947658082F87FF02C071
:1004F0000C94347483E50E94BC37002E000C110B61
:100500007801EE0CFF1C882359F10E944037F70157
:10051000E35CFD4F91838083000F111F000F111FBB
:10052000980126573D4F7901BC01990F880B990B13
:100530000F94276D2AE037ED43E25CE30F94866D5C
:10054000085F194FD8012D913D914D915C910F9409
:10055000866DF70160837183828393830C94347476
:100560000E94D75785E40E94234180E3800F0E94B8
:100570002341F701E35CFD4F608171818AED93E1D6
:100580000E94B94985E20E9423418AE00E942341EA
:100590000C94347480E50E946E37882311F40C9417
:1005A00034740E9440378C01892B09F082C083E5A6
:1005B0000E946E37882391F00E9440378F3F980742
:1005C00031F484ED96E10E94E93E0C943474BC0150
:1005D00084ED96E10E94573F0C9434740E94D757E3
:1005E00070E060E085EE93E10E94B9498091D616F3
:1005F00058E5C52E52E0D52EC81AD10887FDD394F0
:10060000CC0CDD1CCC0CDD1C0D2C000CEE08FF0806
:100610008091D51678E8872E912C881A910887FD4D
:100620009394880C991C880C991C092C000CAA081E
:10063000BB088091D41690E08F3FC9F1FC01EE0F0A
:10064000FF1FE80FF91FE557F94E8181928133E0D2
:10065000880F991F3A95E1F7B0E0A0E044E0B59526
:10066000A795979587954A95D1F702969C012F5F9C
:100670003F4F032E000C440B550B281939094A092A
:100680005B09A4EBB0E00F94A573A70196012819AC
:1006900039094A095B090F948673B90182EE93E127
:1006A0000E94B9498AE00E9423410C94347480E08E
:1006B000DDCF0E94D357B8018CEF93E10E94B94976
:1006C0008DEE93E10E945C410C9434740E94DB57E0
:1006D0000C94347460E085E40E943638811174C053
:1006E00080E50E946E37882351F00E944437609362
:1006F0004F1670935016809351169093521689E4BA
:100700000E946E37882381F00E9444372CEA35EC32
:1007100047E25EE30F94866D609353167093541610
:10072000809355169093561684E40E946E37882362
:1007300081F00E9444372CEA35EC47E25EE30F94E7
:100740000C756093571670935816809359169093B2
:100750005A160E94D75740914F16509150166091EB
:100760005116709152168BE094E10E942F442CEAAE
:1007700035EC47E25EE36091531670915416809118
:100780005516909156160F940C75AB01BC0187E07D
:1007900094E10E942F442CEA35EC47E25EE360913D
:1007A0005716709158168091591690915A160F94B9
:1007B000866DAB01BC0183E094E10E942F448AE086
:1007C0000E9423410C9434740E94D3578FE094E12B
:1007D0000E945C410C94347480E50E946E3788233B
:1007E00051F00E9444376093EC087093ED088093B9
:1007F000EE089093EF0889E40E946E37882381F019
:100800000E9444372CEA35EC47E25EE30F94866D94
:100810006093F0087093F1088093F2089093F308C6
:1008200084E40E946E37882381F00E9444372CEACA
:1008300035EC47E25EE30F940C756093F408709317
:10084000F5088093F6089093F7080E94D7574091D7
:10085000EC085091ED086091EE087091EF0889E284
:1008600094E10E942F442CEA35EC47E25EE360916C
:10087000F0087091F1088091F2089091F3080F94BC
:100880000C75AB01BC0185E294E10E942F442CEA77
:1008900035EC47E25EE36091F4087091F5088091D1
:1008A000F6089091F7080F94866DAB01BC0181E2C8
:1008B00094E10E942F448AE00E9423410C943474F6
:1008C00083E50E946E37182F882369F00E94403715
:1008D0009C0190938F0280938E0291E0232B09F06C
:1008E00090E09093270A80E50E946E37882361F09C
:1008F00020918E0230918F02232B11F00E94492A01
:100900008093270A0C94347411110C9434740E944F
:10091000D75788E594E10E945C418091270A88239B
:1009200091F080E494E10E945C4160918E027091AC
:100930008F0287E494E10E94B94983E494E10E9424
:100940005C410C9434748CE394E1EDCF0E940CFB79
:100950000C9434740E9418320E94EA290F946B1987
:100960000C9434740E948A590C9434746FEF7FEFA6
:1009700089E40E948D39082F6FEF7FEF8AE40E948F
:100980008D39182F8AE50E94BC37D12C811107C000
:1009900081E50E94BC37D82E882309F467C3C02E96
:1009A00081E0800F863008F04EC0912E81E0810FEB
:1009B000863008F048C00E9444372B013C01F02EDD
:1009C00007FDF12C07FF02C004E0C02E812E17FDA9
:1009D000812C17FF02C014E0912EB5E03B2ECF14FE
:1009E00010F40C943474E82C3F9C500111249E1494
:1009F00040F10E2D10E020E030E0A901DD2069F08B
:100A0000F501E00FF11FEE0FFF1FEE0FFF1FE35E7A
:100A1000F94F20813181428153810A0D1B1D000F46
:100A2000111F000F111F035E194FC301B2010F9474
:100A30001274D8016D937D938D939C931397E394D7
:100A4000D6CFF394CCCF0E94D3578BE894E10E9489
:100A50005C410C9434740E94D35782EC94E10E9460
:100A60005C4161E084EB94E10E940CCA0E94789A98
:100A700068E270E088EC90E00E9433950C94347446
:100A800084E50E946E378823A1F010925F051092D2
:100A900060051092610510926205109263058FEF58
:100AA0000E944C2861E070E084E50E948D398093BB
:100AB000630583E50E946E37882321F00E9440374A
:100AC0000E944C2883E40E946E37882331F0809185
:100AD0002F02803210F40E94543A80E50E946E3753
:100AE000882331F00E944037803210F40E94543A3B
:100AF00085E50E946E37882311F40C9434740E94AB
:100B00004037803210F00C94347441E050E060E0E3
:100B100070E0082E04C0440F551F661F771F0A940B
:100B2000D2F7409550956095709500915F051091B2
:100B300060052091610530916205402351236223B5
:100B4000732340935F055093600560936105709334
:100B5000620590912F0289130C9434741092DA106C
:100B60000C9434740E94F3F60C9434740F94A21A0B
:100B70000C94347461E083E50E949C3991E08927EC
:100B80000F94F6260C94347480916A1782FF05C086
:100B9000806480936A170C94347483FD02C00C94B3
:100BA00034740F9497470C9434740E946F700C94B3
:100BB000347480E090E8ABE3B4E4F901808391837E
:100BC000A283B3830C94F47B80E090E8ABE3B4E4BD
:100BD000F90184839583A683B7830C9434740E94AF
:100BE0001C6B0C9434740E94236E0C943474A0908B
:100BF0000D0AB0900E0AC0900F0AD090100A8BE434
:100C00000E94BC37882339F10E9444377B018C0154
:100C100020E030E0A9010F94727687FD0AC020E041
:100C200030E040E251E4B701C8010F94206D18167E
:100C3000A4F48FE30E9423418BE40E94234186EFBA
:100C400094E10E945C418EEE94E10E945C418BEE47
:100C500094E10E945C41750186019701A801B501EC
:100C6000C6010F94206D882361F00E940CFBC70120
:100C7000D80180930D0A90930E0AA0930F0AB093A7
:100C8000100A8091500590915105A0915205B091A4
:100C90005305892B8A2B8B2B11F00C9434740E94F2
:100CA000D75740910D0A50910E0A60910F0A70912A
:100CB000100A8AE095E10E942F448AE00E942341B5
:100CC0000C94347481E0809373081092301460E0C7
:100CD00083E50E949C3981110C9434740F9438364A
:100CE0000C9434740E94D7578CE195E10E945C41CA
:100CF00080911C06882349F089E195E10E945C41BE
:100D00008AE00E9423410C94347485E195E1F6CF8A
:100D10000E94E2880C94347410914D050F943F5258
:100D20006093BA087093BB088093BC089093BD0889
:100D3000112311F40C943474812F0E9408EF0C9449
:100D40003474111107C011E089E50E946E378113D8
:100D50000C94CF74012FF11204C001E011E0FF24C4
:100D6000F39482E50E94BC37882311F40C94D37469
:100D70000E9444376CA37DA38EA39FA320E030E0A4
:100D8000A9010F94206D882381F0011105C0111174
:100D900003C0FF2009F413C160E0CE0184960F94D4
:100DA000E5100E94AC400E945B40002309F480C023
:100DB000112309F47AC01092D3091092D409109229
:100DC000D5091092D6091092D7091092D80910921D
:100DD000D9091092DA090F94EA1185E39DE20E9485
:100DE00012324B015C0189E39DE20E9412322B0119
:100DF0003C01AC019B01C501B4010F947276181639
:100E000014F00C94D974A5019401C301B2010F949C
:100E10000C759B01AC010F94866D20E030E040E83A
:100E20005FE30F9412740F94C07620E030E048E442
:100E300052E40F94866D68A379A38AA39BA320E054
:100E400030E040EC5FE3C301B2010F94866D90582F
:100E500069837A838B839C8320E030E040EC5FE3FE
:100E6000C501B4010F94866D90586C8F7D8F8E8F65
:100E70009F8FAE01405E5F4FBE016F5F7F4FCE011F
:100E80004C960F94A4100F94C41C1092D309109286
:100E9000D4091092D5091092D6091092D709109250
:100EA000D8091092D9091092DA0980E00F94B91D7F
:100EB000112319F081E00F94B91DFF2009F47FC0C0
:100EC00083E00F945F2E81117AC00F94EA11209174
:100ED000090930910A0940910B0950910C0960E011
:100EE00070E086EE92E40F9411742B013C01209186
:100EF0000D0930910E0940910F095091100960E0E1
:100F000070E086EE92E40F9411744B015C018091C5
:100F1000DB099091DC09A091DD09B091DE09809395
:100F2000B0089093B108A093B208B093B3080091B1
:100F3000E3161091E416D8012D913D914D915C91ED
:100F4000C301B2010F9411746093A8087093A908AB
:100F50008093AA089093AB08F801248135814681DB
:100F60005781C501B4010F9411746093AC0870935C
:100F7000AD088093AE089093AF0888EA98E00E948D
:100F80007924882311F40C94DF741C8E1D8E1E8E20
:100F90001F8E88E0E8EAF8E0DE01119601900D92DC
:100FA0008A95E1F7AE01445E5F4FBE016B5F7F4FF4
:100FB000CE0101960F94A41082E00F94B91D0F94F6
:100FC000EA1180912C0880932D088E2D0E946D3C93
:100FD0000F94950F83E0809389020F946B190C9402
:100FE000347483E50E94BC37882311F40C94B07EDE
:100FF0000E9440370C94AA7E83E50E94BC37182FCC
:10100000811108C082E50E94BC37082F882311F4A3
:101010000C94107F0E9440370C94DB7E83E50E9485
:10102000BC37882311F40C94407F0E94252A8B0141
:101030000C94407F83E50E94BC37882311F40C9404
:1010400034740E9440370C94B07F83E50E94BC3713
:10105000182F811107C082E50E94BC37882311F444
:101060000C9434740E9440370C94D87F0E94D3575C
:101070008BE694E10E945C410C943474882309F45B
:1010800062CE6BCEDF92EF92FF920F931F93CF93BE
:10109000DF93EC01E090C508F090C6088AE0D82EF6
:1010A0006AE070E0CE010F9460778C01009711F038
:1010B000FC011082CE010E94A83081E00E945F7284
:1010C0000115110519F0E801D992EACFC701DF91A6
:1010D000CF911F910F91FF90EF90DF900C94A8306B
:1010E0004F925F926F927F928F929F92AF92BF9238
:1010F000CF92DF92EF92FF920F931F93CF93DF93E4
:10110000CDB7DEB77C014DB65EB66090C508709075
:10111000C6088DB69EB66AE070E0C7010F945B6C9E
:101120006C018C010E191F09892B21F4C7010F9442
:101130006D6C8C01C80101962DB73EB7281B390B89
:101140000FB6F8943EBF0FBE2DBF8DB79EB7019668
:101150005C01A801B7010F948E6CF501E00FF11F3F
:101160001082C5010E94A83081E00E945F72C11404
:10117000D10451F076019FEFE91AF90A0FB6F894FD
:101180009EBE0FBE8DBEC5CF0FB6F8949EBE0FBEDD
:101190008DBEC3010E94A8300FB6F8945EBE0FBE8C
:1011A0004DBEDF91CF911F910F91FF90EF90DF9097
:1011B000CF90BF90AF909F908F907F906F905F90F7
:1011C0004F9008954F925F926F927F928F929F926D
:1011D000AF92BF92CF92DF92EF92FF920F931F9345
:1011E000CF93DF93CDB7DEB7C059D1090FB6F894CE
:1011F000DEBF0FBECDBF0E94C739882369F083E5EB
:101200000E946E37882301F120E040E070E060E04A
:1012100082EA9AE90E94DB97C057DF4F0FB6F89435
:10122000DEBF0FBECDBFDF91CF911F910F91FF9019
:10123000EF90DF90CF90BF90AF909F908F907F9076
:101240006F905F904F90089583E40E946E378823DB
:1012500019F00E94979AE0CF8090BC099090BD0948
:10126000A090BE09B090BF098091C50980FF05C05C
:101270009091DB1098609093DB108695817080933D
:10128000270A87EE90E10E94708880914B09909127
:101290004C099E012F5F3F4F7901009799F09F9372
:1012A0008F938EED90E19F938F933F932F930F94A5
:1012B000B76CC7010E9442880F900F900F900F905B
:1012C0000F900F908091490990914A09009799F0E9
:1012D0009F938F9385ED90E19F938F93FF92EF9271
:1012E0000F94B76CC7010E9442880F900F900F9027
:1012F0000F900F900F906E0131E8C30ED11C6091DA
:1013000028097091290980912A0990912B09860159
:1013100023E041E00F94ED679F938F9383EC90E17E
:101320009F938F93FF92EF920F94B76CC7010E9427
:1013300042888BEB90E10E94708887E08093B80828
:10134000809307060F900F900F900F900F900F90C3
:10135000809144098823F9F060914509709146090C
:10136000809147099091480923E041E00F94ED678F
:101370009F938F9382EB90E19F938F93FF92EF92D5
:101380000F94B76CC7010E9442880F900F900F9086
:101390000F900F900F9080914D098823A1F01F921C
:1013A0008F931F921F9285EA90E19F938F93FF92F4
:1013B000EF920F94B76CC7010E9442880FB6F89461
:1013C000DEBF0FBECDBF80914E098823A9F01F92CA
:1013D0008F931F9281E08F9385EA90E19F938F9383
:1013E000FF92EF920F94B76CC7010E9442880FB62C
:1013F000F894DEBF0FBECDBF40904F09509050090A
:10140000609051097090520920E030E0A901C301B9
:10141000B2010F94206D811104C08091C50982FF33
:1014200020C0860121E041E0C301B2010F94ED67C5
:101430009F938F938091C50982FB882780F91F9223
:101440008F9388E990E19F938F93FF92EF920F948F
:10145000B76CC7010E9442880FB6F894DEBF0FBE7A
:10146000CDBF60911A0970911B0980911C09909160
:101470001D098E010F581F4F23E041E00F94ED67C7
:10148000782E692E609116097091170980911809BC
:1014900090911909860123E041E00F94ED676F9266
:1014A0007F929F938F9387E890E19F938F93FF9212
:1014B000EF920F94B76CC7010E94428860911E0999
:1014C00070911F09809120099091210923E041E04A
:1014D0000F94ED678CE790E10E947088DF92CF92C5
:1014E00082E790E19F938F93FF92EF920F94B76CF6
:1014F000C7010E944288809127098F938091260915
:101500008F938BE690E19F938F93FF92EF920F94CE
:10151000B76CC7010E94428860912209709123092B
:10152000809124099091250923E041E00F94ED6713
:101530009F938F9381E690E19F938F93FF92EF9219
:101540000F94B76CC7010E9442888CE0ECE2F9E08E
:10155000A9E0B9E001900D928A95E1F78CE0E8E30B
:10156000F9E0ADEFB8E001900D928A95E1F780E0E7
:101570000F94A70E81E00F94A70E82E00F94A70EA0
:101580008091C4098093DD0881E080931C060E944D
:10159000B93983E599E09F938F9386E49DE39F9308
:1015A0008F93FF92EF920F94B76C0FB6F894DEBF53
:1015B0000FBECDBFC7010E9442888091C3098F939F
:1015C0008091C2098F938091C1098F938091C00946
:1015D0008F93BF92AF929F928F9283E590E19F93FA
:1015E0008F93FF92EF920F94B76CC7010E944288CD
:1015F0000FB6F894DEBF0FBECDBF0ECECF93DF93F4
:10160000C0911212C093E80981E6C89FE00111243D
:10161000CC5EDD4E8091DB1080FF05C00E94D75765
:10162000CE010E942A41CE010E94A83080E0DF91C5
:10163000CF910C945F728F929F92AF92BF92CF9294
:10164000DF92EF92FF92CF936B017C0120E030E0BC
:10165000A9010F94206D87FFA3C06DEB77E386E0AF
:1016600095EBA70196010F9412746B017C0120E0A9
:1016700030E040E251E40F94866D20E030E048EC29
:1016800052E40F94866D4B015C0120E030E040E2B3
:1016900051ECC701B6010F94206D181654F420E0E8
:1016A00030E048EC52E4C701B6010F94727687FD32
:1016B0008BC020E030E0A901C701B6010F94206D76
:1016C00087FF73C060E070E080EA90ECA5019401B0
:1016D0000F94127420E030E040E251E40F940C7556
:1016E0000F947E756B017C01F7FC64C020E137E24A
:1016F00040E050E00F948673CA01B9012AE030E05F
:1017000040E050E00F948673605D60939608C701D7
:10171000B60128EE33E040E050E00F9486739AE083
:10172000892E912CA12CB12CCA01B901A5019401DB
:101730000F948673605D60939708C701B60124E635
:1017400030E040E050E00F948673CA01B901A50172
:1017500094010F948673605D609398088EE2809385
:101760009908C701B601A50194010F948673C62F8D
:10177000CA01B901A50194010F948673605D60935D
:101780009A08C05DC0939B0886E998E0CF91FF90CE
:10179000EF90DF90CF90BF90AF909F908F90089583
:1017A0006DEB77E386E095E35CCF60E070E080EA84
:1017B00090E48CCFF094E094D094C094C11CD11CE0
:1017C000E11CF11C6DE2A1CF20E030E0A901C701CE
:1017D000B6010F94206D87FF6AC060E070E080EA78
:1017E00090ECA50194010F94127420E030E040E2E7
:1017F00051E40F940C750F947E754B015C0120E051
:1018000030E0A901C701B6010F94727687FD0BC0C5
:1018100020E030E040E251E4C701B6010F94206DB2
:1018200060E287FD13C0B7FC47C0C501B40128EED4
:1018300033E040E050E00F948673CA01B9012AE01A
:1018400030E040E050E00F948673605D609397084D
:10185000C501B40124E630E040E050E00F94867307
:101860008AE0C82ED12CE12CF12CCA01B901A701C4
:1018700096010F948673605D609398088EE2809362
:101880009908C501B401A70196010F948673C62F6C
:10189000CA01B901A70196010F948673605D609338
:1018A0009A08C05DC0939B0887E998E06FCF60E01D
:1018B00070E080EA90E495CFB094A09490948094E6
:1018C000811C911CA11CB11C6DE2C0CF60913D0236
:1018D00070913E02072E000C880B990B0F94276D18
:1018E0002AE037ED43E25CE30F94866D2091080611
:1018F0003091090640910A0650910B060F94866DAF
:1019000060938A0270938B0280938C0290938D0275
:101910000895E091A308E23030F4F0E0EB5EF54F7B
:10192000809191088083089580915F178823C1F08A
:10193000815080935F17EBE8F7E1882351F08150E5
:10194000990B2BE1289FF001299FF00D1124EF53F3
:10195000F84E8BE1A6EAB7E101900D928A95E1F786
:1019600020915F17211105C080916A1780628093D2
:101970006A1781E090E0A0E0B0E0211103C080E0B0
:1019800090E0DC018093890890938A08A0938B08EB
:10199000B0938C0810928E0881E08093880883E0D1
:1019A000809389020895CF93DF93EC01CB01BA01B4
:1019B0000F94276D29EC38EC48EC5EE30F940C751E
:1019C00020E030E040E05FE30F9412740F948575DF
:1019D0006883DF91CF9108958091590290915A02C6
:1019E0000C940C2CE091A30886E0E802F00111248D
:1019F000EC58F74F8091910890E095838483089587
:101A00008F929F92AF92BF92CF92DF92EF92FF920E
:101A1000CF936B017C0120E030E0A9010F94206D91
:101A200087FD9FC06DEB77E386E095E3A701960104
:101A30000F9412746B017C0120E030E040E251E42D
:101A40000F94866D20E030E048EC52E40F94866DF0
:101A50004B015C0120E030E0A901C701B6010F9401
:101A6000206D20E030E040EA50E487FF04C020E031
:101A700030E040EA50ECC501B4010F94127420E04C
:101A800030E040E251E40F940C750F947E756B01C9
:101A90007C018BE2F7FE09C0F094E094D094C094EE
:101AA000C11CD11CE11CF11C8DE280939508C7017B
:101AB000B60120E137E240E050E00F9486738AE0FF
:101AC000882E912CA12CB12CCA01B901A501940139
:101AD0000F948673605D60939608C701B60128EE87
:101AE00033E040E050E00F948673CA01B901A501CC
:101AF00094010F948673605D60939708C701B601E7
:101B000024E630E040E050E00F948673CA01B9014A
:101B1000A50194010F948673605D609398088EE22E
:101B200080939908C701B601A50194010F948673AB
:101B3000C62FCA01B901A50194010F948673605D97
:101B400060939A08C05DC0939B0885E998E0CF91A7
:101B5000FF90EF90DF90CF90BF90AF909F908F90CD
:101B600008956DEB77E386E095EB60CF8F929F92BF
:101B7000AF92BF92CF92DF92EF92FF926B017C0106
:101B800020E030E0A9010F94206D87FD6BC06DEB64
:101B900077E386E095E3A70196010F9412746B0139
:101BA0007C0120E030E040E251E40F94866D20E0BB
:101BB00030E040E251E40F94866D4B015C0120E07F
:101BC00030E0A901C701B6010F94206D20E030E09C
:101BD00040EA50E487FF04C020E030E040EA50ECE7
:101BE000C501B4010F94127420E030E040E251E4EA
:101BF0000F940C750F947E759B018BE237FF05C027
:101C000022273327261B370B8DE280939708C901C3
